:100000000C9487070C94D6070C94D6070C94D6074B
:100010000C94D6070C94D6070C94D6070C94D607EC
:100020000C94D6070C94A6170C94D6070C94D607FC
:100030000C94EF350C94D6070C94D6070C94D60785
:100040000C94D6070C94D6070C941B160C94D60768
:100050000C94EB0C0C94D6070C94B50C0C94D607AE
:100060000C94E31C0C94D6070C9493310C94D60793
:100070000C945F7B0C94D6070C945B760C94D6079B
:100080000C94D6070C94D6070C94D6070E1D131D9E
:10009000181D211D381D4F1D5F1D6F1D8C1D781FE4
:1000A0004F1D3A1E4B1E7A1E981EB51E0F1F6A1F4B
:1000B0004821DA2197221723802330243B269826D3
:1000C00005274F279A27E72738289228F1288B29D8
:1000D000262A202BBB31E23125329532AD32EE3269
:1000E000A133613461346134613461346134613429
:1000F000613461346134613418341A341F34373454
:1001000039340A0D426174743A0020256420436535
:100110006C6C732000204C6F77207761726E696E73
:1001200067206C6576656C3A2025642E2564000A8C
:100130000D466F756E6420424C2D4374726C3A20EC
:10014000002564000A0D0A0D2121204D4953534911
:100150004E4720424C2D4354524C3A2025642021D6
:1001600021000A0D3D3D3D3D3D3D3D3D3D3D3D3D7B
:100170003D3D3D3D3D3D3D3D3D3D3D3D3D3D3D3DAF
:100180003D3D3D3D3D3D3D000A0D43616C69627260
:100190006174696E67207072657373757265207320
:1001A000656E736F722E2E004F4B0A0D000A0D46BE
:1001B0006C696768742D74696D65202575206D699B
:1001C0006E2020546F74616C3A2575206D696E0045
:1001D0000A0D436F6E74726F6C3A2000486561645B
:1001E000696E67486F6C64004E6F726D616C202899
:1001F0004143432D4D6F646529000A0D3D3D3D3D52
:100200003D3D3D3D3D3D3D3D3D3D3D3D3D3D3D3D1E
:100210003D3D3D3D3D3D3D3D3D3D3D3D3D3D3D0A41
:100220000D00416E676C654E69636B2020202020B5
:100230002020416E676C65526F6C6C20202020205E
:1002400020204163634E69636B2020202020202002
:100250002020416363526F6C6C20202020202020DE
:1002600020205961774779726F202020202020209C
:1002700020204865696768742056616C7565202088
:1002800020204163635A202020202020202020208D
:1002900020204761732020202020202020202020A3
:1002A0002020436F6D706173732056616C756520FB
:1002B0002020566F6C74616765205B302E31565D6F
:1002C00020205265636569766572204C6576656CA1
:1002D00020204779726F20436F6D70617373202007
:1002E00020204D6F746F722031202020202020208C
:1002F00020204D6F746F722032202020202020207B
:1003000020204D6F746F7220332020202020202069
:1003100020204D6F746F7220342020202020202058
:1003200020204D6F746F7220352020202020202047
:1003300020204D6F746F7220362020202020202036
:100340002020313820202020202020202020202084
:100350002020576F757443616C635374617465201A
:100360002020536572766F2020202020202020201E
:100370002020486F7665726761732020202020203E
:10038000202043757272656E74205B302E31415DA2
:1003900020204361706163697479205B6D41685D01
:1003A00020204D6F746F72203720202020202020C5
:1003B00020204D6F746F72203820202020202020B4
:1003C00020204D6F746F72203920202020202020A3
:1003D00020204D6F746F722031302020202020208B
:1003E00020204932432D4572726F72202020202038
:1003F0002020424C204C696D697420202020202050
:1004000020204750535F4E69636B2020202020201E
:1004100020204750535F526F6C6C202020202020FA
:10042000202021212120494E434F4D504154494223
:100430004C4520212121002A002E000A0D20444194
:1004400043206F7220493243204552524F5221209F
:10045000436865636B204932432C203356726566CE
:100460002C2044414320616E6420424C2D43747221
:100470006C005B25695D005B25695D002B204D6983
:100480006B726F4B6F70746572202B0048573A5631
:1004900025642E25642053573A25642E2564256350
:1004A0000053657474696E673A25642025730048AB
:1004B00061726477617265204572726F7220313AA1
:1004C0002564202121004D697373696E6720424CB9
:1004D0002D4374726C3A25642121004D6978657250
:1004E000204572726F722100493243204552524FAB
:1004F00052212121004865696768743A202025351A
:100500006900536574706F696E743A2535690050DF
:10051000726573737572653A253569004F66667347
:1005200065743A202025356900486569676874203C
:10053000636F6E74726F6C0044495341424C454482
:100540000048656967687420636F6E74726F6C0031
:1005500044495341424C4544006163742E20626516
:100560006172696E67004E69636B3A20202020201B
:100570002025356900526F6C6C3A20202020202005
:1005800025356900436F6D706173733A2020202513
:100590003569004B313A25346920204B323A2534F5
:1005A0006920004B333A25346920204B343A2534F6
:1005B0006920004B353A25346920204B363A2534E2
:1005C0006920004B373A25346920204B383A2534CE
:1005D0006920004E693A2534692020526F3A25344B
:1005E00069200047733A253469202047693A253449
:1005F00069200050313A253469202050323A2534A0
:1006000069200050333A253469202050343A25348B
:100610006920004779726F202D2053656E736F72C9
:10062000004E69636B25346920282533692E2569BE
:100630002900526F6C6C25346920282533692E25DA
:10064000692900476965722534692028253369299D
:10065000004E69636B2025346920282533692E25D7
:10066000782900526F6C6C20253469202825336965
:100670002E257829005961772020253469202825E6
:10068000336929004E69636B20253469202825339E
:100690006929282533692900526F6C6C202534693B
:1006A00020282533692928253369290059617720B5
:1006B0002025346920282533692928253369290014
:1006C000414343202D2053656E736F72004E696362
:1006D0006B2025346920282533692900526F6C6C02
:1006E00020253469202825336929005A202020201C
:1006F00025346920282533692900566F6C74616799
:10070000653A2020202533692E253169560043752E
:100710007272656E743A2020202533692E25316966
:100720004100506F7765723A2020202020253469DF
:1007300057004469736368617267653A20253569BB
:100740006D41680052656365697665720052432D9C
:10075000525353493A202020202534690052432D1A
:100760005175616C6974793A202534690052432DC2
:100770004368616E6E656C733A25346900436F6D32
:10078000706173730048656164696E673A20202563
:1007900035690056616C75653A2020202025356941
:1007A0000053746172743A2020202025356900506E
:1007B0006F7469313A202025336900506F746932B3
:1007C0003A202025336900506F7469333A20202580
:1007D000336900506F7469343A2020253369005022
:1007E0006F7469353A202025336900506F7469367B
:1007F0003A202025336900506F7469373A2020254C
:10080000336900506F7469383A20202533690053EA
:100810006572766F202000536574706F696E742066
:100820002025336900506F736974696F6E3A202513
:1008300033690052616E67653A2533692D25336946
:100840000045787465726E436F6E74726F6C202011
:10085000004E693A2534692020526F3A25346920C8
:100860000047733A253469202047693A25346920C6
:100870000048693A253469202043663A25346920C6
:1008800000424C2D4374726C204572726F7273205B
:100890000025336420253364202533642025336408
:1008A000200025336420253364202533642025333C
:1008B00064200025336420253364202533642025FB
:1008C00033642000424C2054656D7065726174750C
:1008D0007265002533692025336920253369202579
:1008E00033692000253369202533692025336920A9
:1008F0002533692000253369202533692025336994
:10090000202533692000424C2D4374726C20666FA1
:10091000756E642000202563202020256320202080
:10092000256320202025632000202563202020250A
:1009300063202020256320202025632000202563BC
:100940002020202D2020202D2020202D200031307F
:1009500000313100313200466C696768742D54698A
:100960006D65202000546F74616C3A2535756D6992
:100970006E004163743A20202535756D696E00283C
:10098000726573657429000A0D47656E657261743E
:10099000696E672064656661756C74205061726170
:1009A0006D6574657220536574202564000A0D55C9
:1009B00073696E6720506172616D65746572205352
:1009C0006574202564000A0D47656E65726174695F
:1009D0006E672064656661756C74204D6978657218
:1009E000205461626C65000A0D4D697865722D4373
:1009F0006F6E6669673A20272573272028257520A2
:100A00004D6F746F727329000A0D3D3D3D3D3D3DB4
:100A10003D3D3D3D3D3D3D3D3D3D3D3D3D3D3D3D06
:100A20003D3D3D3D3D3D3D3D000A0D414343206E72
:100A30006F742063616C69627261746564210D0A70
:100A4000000A0D506C6561736520636F6E6E65639F
:100A500074205370656B7472756D2072656365697F
:100A600076657220666F722062696E64696E6720B7
:100A70004E4F572E2E2E006F6B2E0A0D0054696DAF
:100A8000656F75742E0A0D0000008F001E01AD0108
:100A90003B02CA025803E603740402058F051B06D5
:100AA000A7063307BE074808D2085B09E3096B0AAB
:100AB000F20A780BFD0B810C040D860D070E870ED4
:100AC000060F840F00107B10F5106E11E5115B12FC
:100AD000CF124213B31323149214FE146A15D315C4
:100AE0003B16A11605176717C81727188318DE18B5
:100AF00037198E19E319361A871AD61A231B6E1B5B
:100B0000B61BFD1B411C831CC31C001D3C1D751D19
:100B1000AB1DE01D121E421E6F1E9A1EC31EE91E53
:100B20000D1F2E1F4D1F691F841F9B1FB01FC31F4A
:100B3000D31FE11FEC1FF51FFB1FFF1F00200B0140
:100B40000000C76C00020101BA6D010302024E6E83
:100B500002040303AB6E03050404456F0406050598
:100B6000E16F05070606547006080707C6700709F7
:100B700008080971080A09095671090B0A0AA771C0
:100B80000A000B0BEC712532692E253169560025C0
:100B90003364256320253033646D005374617475AC
:100BA00073004552524F523A202532640025346971
:100BB000202532693A25303269002534696D256374
:100BC00000253369202533692025336920253369C1
:100BD00000253369202533692025336920253369B1
:100BE0000054656D706572617475726573202020A4
:100BF00020002563432020202020002532692E2557
:100C000031695620202533692E253169410025346C
:100C10006957202536696D4148002532756D2F735F
:100C2000205361743A2564200020203344004E6F25
:100C30004678004447505300486F6D653A25336449
:100C40006D202533642563004E6F204E6176694325
:100C500074726C210025336920253369202533699E
:100C60002025336900253369202533692025336920
:100C7000202533690043757272656E7473202020DD
:100C800020002533692E2531694120002533692054
:100C900025336920253369202533690025336920F0
:100CA0002533692025336920253369004D2053659C
:100CB00074506F696E74202020202020004D5365F1
:100CC0007450202020002533694E2025336952209E
:100CD000202B4E0025336947202020202B52202D29
:100CE0004E202D52002533693D486F76657267614D
:100CF00073002533693D48472F34202533693D472C
:100D00006173003E2533693D53657269616C706F94
:100D1000743100202533693D53657269616C706FD1
:100D2000743200202533693D53657269616C706FC0
:100D30007431003E2533693D53657269616C706F93
:100D40007432003E2533693D484400202533693D17
:100D5000485000202533693D4844003E2533693D15
:100D60004850000A0D7777772E4D696B726F4B6F85
:100D7000707465722E646520286329204869537950
:100D80007374656D7320476D6248000A0D74686561
:100D900020757365206F66207468697320736F66B1
:100DA0007477617265206973206F6E6C792070654D
:100DB000726D6974746564200A0D6F6E206F7269BC
:100DC00067696E616C204D696B726F4B6F707465F3
:100DD000722D48617264776172650041435420440A
:100DE000534C004A65746920736174656C6C697456
:100DF000005370656B7472756D20736174656C6CF3
:100E0000697420284C6F77207265736F6C757469F4
:100E10006F6E29005370656B7472756D2073617409
:100E2000656C6C6974202832303438290053706541
:100E30006B7472756D20736174656C6C6974004DB0
:100E4000756C74697369676E616C2050504D000A4F
:100E50000D52656365697665723A2000756E6B6E3A
:100E60006F776E2E205573696E672050504D2E2E71
:100E70002E006E6F7420737570706F7274656420CD
:100E8000627920686172647761726521000A0D3DA4
:100E90003D3D3D3D3D3D3D3D3D3D3D3D3D3D3D3D82
:100EA0003D3D3D3D3D3D3D3D3D3D3D3D3D3D3D3D72
:100EB0003D3D000A0D466C69676874436F6E74723D
:100EC0006F6C0A0D48617264776172653A25642E11
:100ED00025640A0D536F6674776172653A5625640E
:100EE0002E2564256320000A0D3D3D3D3D3D3D3DE1
:100EF0003D3D3D3D3D3D3D3D3D3D3D3D3D3D3D3D22
:100F00003D3D3D3D3D3D3D3D3D3D3D3D00001124D0
:100F10001FBECFEFD0E4DEBFCDBF11E0A0E0B1E057
:100F2000E4E2FCEF00E00BBF02C007900D92A23F8D
:100F3000B107D9F718E0A2EFB1E001C01D92AC39BA
:100F4000B107E1F77AEAE2E0F0E081E2809357004E
:100F5000D4907E010894E11CF11C20EF37EF41E0B2
:100F600050E087016FE0DA01C9012F5F3F4F4F4F1B
:100F70005F4FABBFFC018791F80181938F016150F6
:100F800067FFF1CFF7016EE081917827709561508E
:100F900067FFFACF8889781729F0F7E9DF1611F48F
:100FA0000000FECF0E9497080C94117E0C94000064
:100FB00080910406E82FFF27EE0FFF1FE55DF84F35
:100FC000808191818D5E9F4F14F01092030180818A
:100FD00091818A5B9F4FCCF4809103018823A9F40F
:100FE00081E08093030180915B048F5F80935B04B9
:100FF000853038F088EE93E09093220280932102AE
:1010000004C066E970E00E94833980915B049927EF
:101010009093D5058093D40508951F93CF93DF93C4
:10102000182F882389F082E091E09F938F938FEFB0
:1010300092E19F938F93E0912704F0912804099502
:101040000F900F900F900F9080912706823308F039
:1010500044C084EF91E00E942617EC01112329F08F
:10106000CE010E942F178823D9F3C2E0D0E026E5F5
:1010700030E080911D0190911E018217930730F09E
:101080002196255D3F4FC730D10598F38091270603
:101090009927C89F9001C99F300DD89F300D11240A
:1010A000209300011123D9F068EC70E08C2F0E948E
:1010B0008339DF93CF938AE091E09F938F938FEFF3
:1010C00092E19F938F93E0912704F0912804099572
:1010D0008DB79EB706968DBF02C080930001112385
:1010E00011F1809100016AE00E94647D892F9927A7
:1010F0009F938F93809100010E94647D99279F9315
:101100008F9385E191E09F938F938FEF92E19F936F
:101110008F93E0912704F091280409952DB73EB7ED
:10112000285F3F4F2DBFDF91CF911F910895CFEFE3
:10113000D0E4DEBFCDBF8824992414B815B807EEDB
:1011400013E00253104017FFFCCF85E180930201AA
:1011500081E887B93E9A8FEF88B98BE184B981E045
:1011600085B98EE38AB987E48BB9469A84B7877FBD
:1011700084BF80916000886180936000109260005D
:1011800084EC99E09093220280932102109216033E
:10119000109215031092300710922F071092180327
:1011A0001092170310921A031092190384EC94E022
:1011B000A0E0B0E08093950190939601A0939701F1
:1011C000B093980128980E948F170E9460170E9480
:1011D00007130E94D3350E94741B0E944A310E945B
:1011E000D2640E9486720E94927A809102018C30B1
:1011F00010F4299A01C0299878940E946430809153
:101200006B02826080936B0210926D020E94EB442D
:1012100084EF91E00E9426178C0180916B0280FD83
:1012200005C0C8010E942F178823B9F38FE291E00F
:101230009F938F93BFEFAB2EB2E1BB2EBF92AF92C5
:10124000E0912704F0912804099580EA9FE00E942C
:1012500026178C01C0E0D0E00F900F900F900F90F8
:10126000ADECEA2EA6E0FA2EF1E8CF2EF6E0DF2E66
:101270000E94EB4480916B0280FD05C0C8010E9472
:101280002F178823B9F3F60180811816ACF40BC030
:101290000E94EB4480916B0280FD05C0C8010E9452
:1012A0002F178823B9F3C8010E942F17882321F430
:1012B000F7018081882364F7F701808187FF18C0D8
:1012C0002196DF93CF93219781E491E09F938F93B1
:1012D000BF92AF92E0912704F09128040995809184
:1012E000F2018F5F8093F2018DB79EB706968DBF96
:1012F0002196E4E0F0E0CE0EDF1E88E090E0E80EFC
:10130000F91ECC30D10508F4B3CFC0E0D0E00AEC30
:1013100016E0E1E8EE2EE6E0FE2EF801838187FD7F
:101320001CC0F70180811816C4F42196DF93CF9377
:10133000219784E491E09F938F938FEF92E19F93A5
:101340008F93E0912704F0912804099582E080931F
:101350001F028DB79EB706968DBFF80183818078F6
:101360008383219684E090E0E80EF91E085F1F4F0A
:10137000CC30D10590F282E691E09F938F93CFEF2E
:10138000D2E1DF93CF93E0912704F09128040995EF
:10139000909102068091F2010F900F900F900F90A4
:1013A000981728F48091410480618093410488E873
:1013B00091E09F938F93DF93CF93E0912704F09177
:1013C0002804099588EE93E00E9426178C010E945C
:1013D0007A1B0F900F900F900F90C8010E942F174B
:1013E0008823D9F388EA91E09F938F93DF93CF937B
:1013F000E0912704F0912804099580E00E94453A85
:10140000809102010F900F900F900F908A3011F091
:10141000843110F0289801C0289A80ED97E09093CD
:1014200022028093210285E580935D048EE090E0A6
:101430000E94DC2E9927182F00278FE090E00E9451
:10144000DC2E080F111D1093F8010093F7018AE0BC
:1014500090E00E94DC2E9927182F00278BE090E067
:101460000E94DC2E080F111D1093F6010093F50168
:101470000F5F1F4F39F08091F7019091F8018F5F56
:101480009F4F41F41092F8011092F7011092F6016B
:101490001092F5018091F5019091F6019F938F9341
:1014A0008091F7019091F8019F938F938DEA91E0DD
:1014B0009F938F93DF93CF93E0912704F0912804BB
:1014C00009958DB79EB708968DBF80ED91E09F93EB
:1014D0008F93DF93CF93E0912704F091280409952F
:1014E000809110060F900F900F900F90E0912704BD
:1014F000F091280482FF07C08CED91E09F938F93B9
:10150000DF93CF9308C088EE91E09F938F938FEF86
:1015100092E19F938F9309950F900F900F900F90EA
:101520000E94BF2088E893E19093920180939101FB
:1015300081E080935C040E940D0880912A060E943D
:10154000F8798AEF91E09F938F93DF93CF93E091A7
:101550002704F0912804099580ED97E00E94261752
:101560008C018AEF90E00E942617EC0183E08093C3
:10157000AC050F900F900F900F90CE010E942F1787
:10158000882339F084E690E00E942617EC010E943F
:101590004E7B80912502882309F4DFC180910F01E1
:1015A000882309F4DAC11092250280915B04882314
:1015B00019F00E94D80702C00E947F470E94EB44A6
:1015C000209102012A3011F0243110F0289801C036
:1015D000289A80911B0390914104882339F08091CF
:1015E0001B03815080931B03977F0AC080916F007B
:1015F000806280936F0010922C0710922B079860E6
:101600009093410480919101909192010197909360
:101610009201809391018091910190919201892B87
:1016200029F080916C02882309F43EC080919101D9
:1016300090919201892B01F50E94703185E090E034
:1016400090939201809391018091E6059091E70536
:1016500001969093E7058093E6058091E702806804
:101660008093E702809141048160809341048091DE
:10167000AD0582608093AD058091080190910901CC
:101680008F5F9F4F19F5809112038823F9F080E155
:1016900097E2909322028093210280E890E0909359
:1016A00009018093080112C02A3011F0243110F092
:1016B000289801C0289A8091210290912202892BBA
:1016C00029F48091E7028F778093E70280912502C9
:1016D000882309F042C10E944B130E94290FC801C0
:1016E0000E942F17882309F434C10C5E1F4F80918C
:1016F0006C0290914104882339F0926090934104E8
:101700008091AD0582600CC09D7F909341048091D3
:10171000910190919201079728F08091AD058D7FFE
:101720008093AD058091910190919201079728F0E7
:10173000809141048E7F809341048091050188232C
:1017400021F081508093050125C080936704109299
:10175000F3021092F2021092F1021092F002109233
:10176000EF021092EE0280910801909109018F5FC3
:101770009F4F81F480911B03882361F488E99AE3E9
:10178000909322028093210280E09CE090930901D3
:10179000809308018091E801893C70F0815080932A
:1017A000E8018091E7028F7B8093E70280914104FA
:1017B0008B7F8093410435C080910908882309F10B
:1017C0008091E70280648093E70280914104846005
:1017D0008093410480910801909109018F5F9F4F90
:1017E00081F480911203882361F088E99AE3909351
:1017F00022028093210280E098EA9093090180936D
:1018000008011092F9031092F8031092F703109256
:10181000F6038FEF9FEF909337088093360810926E
:10182000E80180910001282F332780911D019091BC
:101830001E0182179307CCF48091E70280628093A7
:10184000E70280910801909109018F5F9F4FC1F4D9
:1018500080E797E1909322028093210280E093E059
:1018600090930901809308010BC08091210290910F
:101870002202892B29F48091E7028F7D8093E70271
:101880000E94D06884E08093200280911203882314
:1018900029F45AEA852E55E0952E12C08091F9015F
:1018A0008F5F8093F901813359F41092F90180918F
:1018B000F3019091F40101969093F4018093F30168
:1018C0000894811C911CF2E78F16FBE09F0609F03B
:1018D00040C0882499242091F7013091F8012F5FAE
:1018E0003F4F3093F8012093F7018091F5019091DB
:1018F000F60101969093F6018093F501832F9927C5
:10190000682F8EE090E00E94E42E8091F701909184
:10191000F8019070682F8FE090E00E94E42E809193
:10192000F5019091F601892F9927682F8AE090E0C0
:101930000E94E42E8091F5019091F6019070682F3D
:101940008BE090E00E94E42E84E190E00E94261754
:101950008C010E9420690E949D7280912002882340
:1019600009F00BCE0E94F36408CE1F920F920FB6BF
:101970000F9211248F939F93EF93FF938091070110
:101980008823E1F4809113029091140201969093C0
:10199000140280931302FC01E45FFA4FE081ED3002
:1019A00019F0803A910539F4109214021092130242
:1019B00081E080930701E093C60004C010921402F6
:1019C00010921302FF91EF919F918F910F900FBE94
:1019D0000F901F9018951F920F920FB60F9211241F
:1019E0002F933F934F935F936F937F938F939F9327
:1019F000AF93BF93CF93EF93FF9390E08091C60096
:101A000080930B0250911902503A10F090931A02F1
:101A100080910B028D3009F065C080911A028230EE
:101A200009F060C090931A02852F992786599B4F21
:101A3000FC01329740812091150230911602241B3F
:101A40003109DC0111978C91281B3109C9019F7064
:101A5000909316028093150246E0969587954A95D5
:101A6000E1F7982F935C909317022F733070235CEB
:101A7000209318028081981729F48C91281711F46B
:101A800091E006C090E0809108028F5F8093080289
:101A9000C0910A02CC2309F074C0992309F471C0E3
:101AA00081E080930A02580F509307025150E52FAE
:101AB000FF27E659FB4F8DE0808380916C048235CF
:101AC00009F05FC00E94BF2088E190E02CE00FB6D3
:101AD000F894A895809360000FBE20936000C09397
:101AE0001F024FC020911A02822F99278130910541
:101AF000F9F0823091051CF4892B21F040C0029747
:101B000011F13DC080910B02833239F480910A02B9
:101B1000882319F481E080931A0280910B0280934C
:101B20006A0481E08093190280910B02992722C0F8
:101B30002F5F20931A02E52FFF27E659FB4F809174
:101B40000B02808309C0E52FFF27E659FB4F8091E8
:101B50000B028083503A20F45F5F5093190202C059
:101B600010921A0220910B02809115029091160298
:101B7000820F911D909316028093150202C010925D
:101B80001A02FF91EF91CF91BF91AF919F918F91E9
:101B90007F916F915F914F913F912F910F900FBE69
:101BA0000F901F901895AC01A0E0B0E09D01A81720
:101BB000B90748F4ECE0F5E08191280F311D11964A
:101BC000A417B507C8F33F70FD01E45FFA4FC901E0
:101BD00056E0969587955A95E1F7835C8083119638
:101BE000FD01E45FFA4F2F733070822F835C808396
:101BF000A35FBA4F8DE08C931092070180910C0582
:101C00008093C6000895A0E0B0E0E9E0FEE00C9407
:101C1000DD7D2C859D850E85BB2483E280930C059C
:101C20009F5990930D0520930E0533E0E32EF12C80
:101C3000002309F49EC0CF84D888BE016D5E7F4F1B
:101C4000A989BA890150109709F493C01097B9F087
:101C5000F601EB0DF11DB3949081119791F40023DF
:101C600049F1FB016E5F7F4FDB01C080D1806E5F69
:101C70007F4F0D90BC91A02DBB24015002C090E07D
:101C800019C01097B9F0F601EB0DF11DB394408126
:101C9000119791F4002341F1FB016E5F7F4FDB014F
:101CA000C080D1806E5F7F4F0D90BC91A02DBB2472
:101CB000015002C040E018C01097B1F0F601EB0DE2
:101CC000F11DB3941081119781F4002371F0FB0191
:101CD0003296DB01CD90DC90BF016E5F7F4FA0811B
:101CE000B181BB24015001C010E0F701E45FFA4F5D
:101CF000892F86958695835C80830894E11CF11C6E
:101D0000F701E45FFA4F892F99278370907024E0E0
:101D1000880F991F2A95E1F755279A0194E0369587
:101D200027959A95E1F7822B835C80830894E11CC8
:101D3000F11CF701E45FFA4F4F705070440F551FCC
:101D4000440F551F812F992726E0969587952A9550
:101D5000E1F7842B835C80830894E11CF11CF7017C
:101D6000E45FFA4F1F73135C10830894E11CF11CAD
:101D70006ACFC7010E94D30DE9E00C94F97DA3E07E
:101D80007A2F409107024650442309F458C0E72FA8
:101D9000FF27E659FB4F80818D537F5FE72FFF2799
:101DA000E659FB4F20812D537F5FE72FFF27E65930
:101DB000FB4F30813D537F5FE72FFF27E659FB4FF5
:101DC00060816D537F5F9927880F991F880F991F36
:101DD000522F52955F70582B822F99278F709070D9
:101DE000F4E0880F991FFA95E1F7232F26952695A1
:101DF000282B832F992783709070E6E0880F991F16
:101E0000EA95E1F7682B41504F3FC9F0EA2FFF27D1
:101E1000E659FB4F5083AF5F41504F3F81F0EA2FAF
:101E2000FF27E659FB4F2083AF5F41504F3F39F00A
:101E3000EA2FFF27E659FB4F6083AF5FA5CF8DE602
:101E400094E09093060280930502A350A0930402AD
:101E50000895A2E0B0E0EFE2FFE00C94E37D809112
:101E60000A02882309F4C7C30E94BF0E80916B0445
:101E7000823609F081C280916C04992781379105DF
:101E800009F4C0C082379105C4F48D36910509F478
:101E900082C08E36910544F48B34910531F186363B
:101EA000910509F454C168C28E36910509F45BC0EE
:101EB0008037910509F49FC05FC28537910509F409
:101EC000E2C18637910544F48337910509F4DCC0FB
:101ED0008437910539F150C28737910509F410C252
:101EE0008937910509F46AC147C2E0910502F09172
:101EF00006028081918190932E0380932D0320917F
:101F00002B0330912C03821B930B845E9D4F68E65C
:101F100071E00E94847D845B904090932A038093BB
:101F200029032AC280910702A0910502B0910602FE
:101F3000853140F080E1E5E4F4E00D9001928A956E
:101F4000E1F70DC08D919D910D90BC91A02D8093D6
:101F5000450490934604A0934704B093480480EF4F
:101F6000809302024BC0809107018823E1F38DE446
:101F700090E09F938F9384E796E09F938F9381E007
:101F80008F938F938EE48F930E94030E8DB79EB72D
:101F900007968DBFF1C1A0910502B09106021C9178
:101FA000113081F48DE4E4E7F6E00D9001928A951A
:101FB000E1F70E94E42F1983809141048F7E809382
:101FC000410401C01982809107018823E1F381E077
:101FD00090E09F938F93CE0101969F938F9381E022
:101FE0008F938F938DE48F930E94030EADB7BEB78E
:101FF0001796ADBFC1C181E080930D028FEF809332
:102000000501BAC1E0910502F091060280818F3F7F
:1020100039F40E944730E0910502F0910602808376
:10202000E0910502F09106028081882311F481E09D
:1020300003C0863010F085E08083E0910502F091C6
:10204000060280810E94FA2EE0910502F0910602BC
:1020500080818983809107018823E1F380E790E004
:102060009F938F9383E096E09F938F9381E090E01E
:102070009F938F93CE0101969F938F9382E08F93CE
:1020800081E08F9381E571C12091050230910602B4
:10209000D9018C918150853008F040C0F9018181CF
:1020A0008435E1F52F5F3F4F80E7E3E0F6E0D901AB
:1020B0000D9001928A95E1F7F90182910E94632FB8
:1020C000809142069927AA27BB27BC01CD0124ECA9
:1020D00039E040E050E00E94457DDC01CB01809377
:1020E000B5019093B601A093B701B093B801809168
:1020F00043069927AA27BB27BC01CD010E94457D35
:10210000DC01CB018093B1019093B201A093B301A4
:10211000B093B4010E944730898301C01982809135
:1021200007018823E1F381E090E09F938F93CE0134
:1021300001969F938F9381E08F938F9383E58F9385
:102140000E94030E8DB79EB707968DBF26C0E09103
:102150000502F0910602E0818E2F8150853018F43F
:102160008E2F0E94FA2E0E944730898380910701AA
:102170008823E1F381E090E09F938F93CE01019655
:102180009F938F9381E08F938F9386E48F930E9428
:10219000030EADB7BEB71796ADBF8091120388236B
:1021A00029F46EE670E089810E94833980E00E9404
:1021B0000D0880912A060E94F879DEC0E0910502A0
:1021C000F09106028081992787FD909590934607AC
:1021D000809345078181992787FD909590934807C3
:1021E000809347078281992787FD909590934A07AE
:1021F000809349078381992787FD909590934C0799
:1022000080934B078481992787FD909590934E0783
:1022100080934D078581992787FD9095909350076E
:1022200080934F078681992787FD90959093520759
:10223000809351078781992787FD90959093540744
:10224000809353078085992787FD90959093560733
:10225000809355078185992787FD9095909358071E
:10226000809357078285992787FD909590935A0709
:10227000809359078385992787FD909590935C07F4
:1022800080935B0779C0E0910502F091060280819E
:102290000E942C358A83882319F481E0898301C048
:1022A0001982809107018823E1F388E090E09F93F1
:1022B0008F9382EC96E09F938F9321E030E03F93E1
:1022C0002F9380910502909106029F938F933F93E5
:1022D0002F93CE0102969F938F933F932F93CE011E
:1022E000820F931F9F938F9384E08F9381E08F934E
:1022F00085E58F930E94030EEDB7FEB773963BC042
:10230000809104028930C0F12091050230910602CB
:102310002F5F3F4F88E0A2ECB6E0F90101900D92EB
:102320008A95E1F7D9018E910E9482348A838823AD
:1023300019F481E0898301C0198280910701882303
:10234000E1F321E030E03F932F93CE0102969F937B
:102350008F933F932F93CE01820F931F9F938F9361
:1023600082E08F9381E08F9387E58F930E94030E25
:10237000EDB7FEB73B96EDBF80916C04992784368C
:10238000910509F4CDC085369105ACF481369105EF
:1023900009F481C0823691052CF48B34910509F43F
:1023A0005DC021C18236910509F482C08336910552
:1023B00009F491C018C18C36910509F4FFC08D361F
:1023C00091054CF48736910509F40AC188369105C8
:1023D00009F4C4C008C18437910529F086379105F6
:1023E00009F4FAC000C180910702A0910502B091E2
:1023F0000602803140F080E1E5E4F4E00D900192C6
:102400008A95E1F70DC08D919D910D90BC91A02D05
:102410008093450490934604A0934704B0934804E6
:10242000809107018823E1F31F92809104018F932B
:1024300084E58F930E94030E8AEF809302028FEF50
:102440008093050180EA9FE00E9426179093FB018C
:102450008093FA010F900F900F90C5C0E091050294
:10246000F09106028081918190932E0380932D0339
:1024700020912B0330912C03821B930B845E9D4F84
:1024800068E671E00E94847D845B904090932A030B
:1024900080932903A8C0E0910502F0910602808193
:1024A00080930601803298F08FE1809306010FC07F
:1024B000A0910502B09106028BE0EDE5F4E00D90ED
:1024C00001928A95E1F7809166048093EE058FEF83
:1024D0008093050188C08091FE019091FF01892BB6
:1024E00089F4E0910502F0910602E081EE2351F0BB
:1024F0008AE0E89FC00111240E94261790933804B7
:1025000080933704E0910502F091060290818AE001
:10251000989FC00111249093FF018093FE0115C084
:102520008FEF80930501E0910502F0910602908102
:102530008AE0989FC00111249093010280930002C9
:10254000892B19F081E080930F0280EA9FE00E94BE
:1025500026179093FB018093FA0145C08FEF80937B
:102560000501E0910502F0910602908197FD08C0F7
:1025700082E080930C021092FD011092FC011AC0BF
:10258000909580916402892B8093640291818AE006
:10259000989FC00111249093FD018093FC0184E079
:1025A00080930C0280EA9FE00E9426179093FB0123
:1025B0008093FA0181E08093100215C08FEF809321
:1025C0000501E0910502F091060280818093650289
:1025D00081E08093110207C081E080930E0203C066
:1025E00081E08093120210920A0210920602109269
:1025F000050210920402E3E0CE5F0C94FF7D982F59
:102600008091C00085FFFCCF9093C60008950F9382
:102610001F9388E18093C1008091C0008260809305
:10262000C0008091C10080688093C1008091C1008A
:1026300080648093C10000E010E00093C5008AE24E
:1026400090E08093C40080910002909101020E946A
:10265000261790933A04809339048CED90E00E9401
:102660002617909369048093680410923B0480E5D8
:1026700080933C0486E080933F048BE080933D048C
:1026800010923E0410930602009305021092040279
:102690001F910F910895A0E1B0E0E1E5F3E10C9402
:1026A000E07D80910701882309F4C1C28091FA017D
:1026B0009091FB010E942F17882361F01092FD0179
:1026C0001092FC0110920102109200021092FF0180
:1026D0001092FE018091FC019091FD01892B41F047
:1026E00080910A0590910B050E942F17882329F4E9
:1026F00080911002882309F460C08091070188232B
:1027000009F45BC080910C0200E211E08430A8F073
:102710000E94D32080E590E09F938F931F930F93A7
:1027200081E08F938F9388E48F930E94030E2DB7DF
:102730003EB7295F3F4F2DBF34C01092660282E240
:1027400094E09F938F9388EC90E29F938F93E09116
:102750002704F0912804099584E190E09F938F93DA
:102760001F930F9381E090E09F938F938CE092E012
:102770009F938F9382E08F9381E08F9388E48F9370
:102780000E94030E80910C02982F8F5F80930C02A1
:102790002DB73EB7215F3F4F2DBF943010F0109200
:1027A0000C028091FC019091FD010E9426179093EC
:1027B0000B0580930A051092100280911102882364
:1027C00051F180910701882331F10E94D32080E5E7
:1027D00090E09F938F9380E291E09F938F9321E00D
:1027E00030E03F932F938FE191E09F938F933F933E
:1027F0002F9385E692E09F938F9383E08F9381E000
:102800008F938CE48F930E94030E109211028DB768
:102810009EB70F968DBF80910E028823D1F08091D4
:1028200007018823B1F08AE090E09F938F938BE3B8
:1028300094E09F938F9381E08F938F9386E58F939E
:102840000E94030E10920E022DB73EB7295F3F4F34
:102850002DBF809112028823D9F08091070188232F
:10286000B9F08BE090E09F938F938DE594E09F9378
:102870008F9381E08F93809104018F9387E48F93EE
:102880000E94030E109212028DB79EB707968DBF5D
:1028900080916804909169040E942F17882309F49D
:1028A00061C080910701882309F45CC080911F06F4
:1028B0009927880F991F880F991F7C010027F7FC23
:1028C0000095102F80916F0390917003A091710378
:1028D000B0917203BC01CD01A80197010E94B97D9E
:1028E00030935604209355048091670390916803B8
:1028F000A0916903B0916A03BC01CD01A8019701C1
:102900000E94B97D30935804209357048091FC02B3
:10291000809359048091FB0280935A0488E090E0F0
:102920009F938F9385E594E09F938F9381E08F939E
:1029300083E08F938BE68F930E94030E80915B045C
:102940002DB73EB7295F3F4F2DBF853018F086E089
:1029500080935B0483E690E00E94261790936904BD
:10296000809368048091000290910102892B41F0CC
:102970008091390490913A040E942F17882321F402
:1029800080910F02882339F180910701882319F182
:102990000E944F3882E490E09F938F938CEA95E0F9
:1029A0009F938F9381E08F938F9384E48F930E9402
:1029B000030E10920F028DB79EB707968DBF8091C0
:1029C000000290910102009731F00E942617909327
:1029D0003A04809339048091FE019091FF01892B84
:1029E00009F4B8C080913704909138040E942F17E1
:1029F000882309F4AFC080910701882309F4AAC095
:102A000080911F069927880F991F880F991F7C01B5
:102A10000027F7FC0095102F80916F0390917003B1
:102A2000A0917103B0917203BC01CD01A80197017F
:102A30000E94B97D30932A04209329048091670372
:102A400090916803A0916903B0916A03BC01CD0124
:102A5000A80197010E94B97D30932C0420932B0488
:102A60002091F1073091F2074091F3075091F4075C
:102A7000DA01C90163E0880F991FAA1FBB1F6A957D
:102A8000D1F7820F931FA41FB51F820F931FA41F9E
:102A9000B51F209195013091960140919701509179
:102AA0009801BC01CD010E94B97D30932E04209382
:102AB0002D048091370390913803A0913903B09190
:102AC0003A0339E0B595A795979587953A95D1F74B
:102AD00080932F048091330390913403A0913503A8
:102AE000B091360329E0B595A795979587952A95D6
:102AF000D1F78093300480913F0390914003A091DF
:102B00004103B091420309E0B595A7959795879544
:102B10000A95D1F7809331048EE090E09F938F93D4
:102B200089E294E09F938F9381E08F938F9383E466
:102B30008F930E94030E8091FE019091FF010E94ED
:102B4000261790933804809337042DB73EB7295F3A
:102B50003F4F2DBF809106018F3F71F1992714E0FF
:102B6000880F991F1A95E1F78E5D9D4F40E150E067
:102B7000BC01CE0101960E94987B80E190E09F937A
:102B80008F93CE0101969F938F9381E090E09F9366
:102B90008F9386E091E09F938F9382E08F9381E003
:102BA0008F9381E48F930E94030E8FEF8093060131
:102BB0008DB79EB70B968DBF8091EE058823D1F01F
:102BC000809107018823B1F081E090E09F938F937B
:102BD0008EEE95E09F938F9381E08F938F9382E4A5
:102BE0008F930E94030E1092EE052DB73EB7295F1A
:102BF0003F4F2DBF80910D028823C9F080910701BE
:102C00008823A9F084E390E09F938F938BE297E071
:102C10009F938F9381E08F938F9380E58F930E9492
:102C2000030E10920D028DB79EB707968DBFE6E09A
:102C3000C05F0C94FC7D1F920F920FB60F9211246F
:102C40002F933F935F936F937F938F939F93AF9354
:102C5000BF93EF93FF9320E080912002882329F017
:102C60008091200281508093200280910A04882361
:102C700019F0815080930A0480912802815080933A
:102C800028028F3F09F05BC089E080932802809181
:102C900026029091270201969093270280932602A4
:102CA00080910A018F5F817080930A01882319F453
:102CB00081E080932502349903C081E0809329024A
:102CC0008091210290912202892B21F18091210291
:102CD000909122020B9750F0809121029091220254
:102CE0000A97909322028093210204C0109222023C
:102CF00010922102809121029091220220910801DC
:102D00003091090182239323892B11F021E008C01F
:102D100020E006C08FEF9FEF909309018093080198
:102D200080910201222331F08A3011F45A9A07C0AF
:102D3000479A05C08A3011F45A9801C0479880918B
:102D40002902882309F472C02091E801222309F0A6
:102D50006DC08091100683FF69C086B19927FC0180
:102D6000E071F07084FF14C08091230290912402DE
:102D700001969093240280932302809123029091E4
:102D80002402895E934008F451C0209329024EC06A
:102D90008091230290912402892B09F443C08091F1
:102DA0002302909124028A569140E0F580912302FB
:102DB0009091240269E270E00E94707D809123026C
:102DC00090912402860F971F9093240280932302F0
:102DD00080912302909124020B9750F0809123025E
:102DE000909124020A9790932E0380932D0304C0A0
:102DF000F0932E03E0932D0380912D0390912E03E9
:102E000020912B0330912C03821B930B845E9D4FEA
:102E100068E671E00E94847D845B904090932A0371
:102E2000809329031092240210922302FF91EF91C4
:102E3000BF91AF919F918F917F916F915F913F91E2
:102E40002F910F900FBE0F901F9018952091260282
:102E500030912702280F391FC9010196089520914A
:102E6000260230912702821B930B892F9927869582
:102E7000807490700895CF93DF930E942617EC0121
:102E8000CE010E942F178823D9F3DF91CF910895A7
:102E9000CF93DF930E942617EC0109C080910F01A8
:102EA000882329F090930F018FEC80937A00CE0154
:102EB0000E942F17982F882389F3DF91CF910895CF
:102EC0009FB7F8945F983E9A469A8091B0008F70B1
:102ED0008093B0008091B00083608093B0008091B7
:102EE000B1008B738093B1008091B1008B608093AF
:102EF000B1001092B2008FEF8093B3008091B000C8
:102F000080688093B000809170008A7F8093700009
:102F1000809170008260809370009FBF08958AE066
:102F200090E00E942617909331028093300282E055
:102F300085BD83EA84BD17BC84EB88BD86E086BD71
:102F400080916E00816080936E0008951F920F92B1
:102F50000FB60F9211242F933F934F935F936F936C
:102F60007F938F939F93AF93BF93CF93DF93EF9311
:102F7000FF938091020190912A02843108F011C1DF
:102F8000992309F06AC38091B00086FFECC080915C
:102F9000B0008F7B8093B00089EA93E090932C027D
:102FA00080932B0280910B0190910C019C01220FC8
:102FB000331F280F391F8091A1019927880F991F6E
:102FC000880F991F280F391F37FF02C02D5F3F4F11
:102FD000C901959587959595879590930C01809358
:102FE0000B0190931E0280931D02809165066091F3
:102FF000310620916F03309170034091710350911D
:10300000720380FF2CC0772788279927EA01D9010E
:1030100057FF04C0A158BF4FCF4FDF4FE7E0D59512
:10302000C795B795A795EA95D1F79D01AE010E9486
:10303000457D9B01AC0197FF04C0215C3F4F4F4F82
:103040005F4F66E055954795379527956A95D1F777
:1030500080911D0290911E02820F931F2BC0772733
:1030600088279927EA01D90157FF04C0A158BF4F0B
:10307000CF4FDF4F27E0D595C795B795A7952A95F0
:10308000D1F79D01AE010E94457D9B01AC0197FFE8
:1030900004C0215C3F4F4F4F5F4FF6E05595479579
:1030A00037952795FA95D1F780911D0290911E02D0
:1030B000821B930B90931E0280931D028091320617
:1030C000282F3327220F331F220F331F80911D0219
:1030D00090911E02821793077CF080913306282F6F
:1030E0003327220F331F220F331F80911D0290912F
:1030F0001E022817390724F430931E0220931D0264
:1031000020912B0230912C0280911D0290911E0281
:10311000280F391F2050324030932C0220932B026D
:1031200080911D0290911E0297FD039695958795BB
:103130009595879590931E0280931D0245E02D3D45
:10314000340718F08CED95E005C02757314030F476
:1031500087E791E090932C0280932B0280912B02C1
:1031600090912C0243C28091B00080648093B000A3
:1031700080913806282F33278DED96E0289FA001F7
:10318000299F500D389F500D1124CA0120912D0206
:1031900030912E02821B930B90932C0280932B0272
:1031A00059C2992309F059C28091B00086FF23C209
:1031B0008091B0008F7B8093B000E0912F02EE23CE
:1031C000F1F480913806282F33278DED96E0289F63
:1031D000A001299F500D389F500D1124CA01209144
:1031E0002D0230912E02821B930B90932C02809320
:1031F0002B0210922E0210922D02469A2BC289EABF
:1032000093E090932C0280932B028E2F992783308A
:10321000910509F4A4C1843091053CF481309105F5
:1032200061F0029709F4D2C0AAC18430910509F473
:1032300099C1059709F4A0C1A2C180910B01909199
:103240000C019C01220F331F280F391F8091A1010F
:103250009927880F991F880F991F280F391F37FF4B
:1032600002C02D5F3F4FC90195958795959587952C
:1032700090930C0180930B0190931E0280931D028A
:10328000809165066091310620916F033091700343
:10329000409171035091720380FF2CC077278827DB
:1032A0009927EA01D90157FF04C0A158BF4FCF4F5A
:1032B000DF4F27E0D595C795B795A7952A95D1F704
:1032C0009D01AE010E94457D9B01AC0197FF04C0AA
:1032D000215C3F4F4F4F5F4FA6E05595479537957F
:1032E0002795AA95D1F780911D0290911E02820F19
:1032F000931F27C077278827992757FF04C0215895
:103300003F4F4F4F5F4FF7E05595479537952795BE
:10331000FA95D1F70E94457D9B01AC0197FF04C04F
:10332000215C3F4F4F4F5F4FE6E0559547953795EE
:103330002795EA95D1F780911D0290911E02821B7C
:10334000930B90931E0280931D0280913206282FCA
:103350003327220F331F220F331F80911D029091BC
:103360001E02821793077CF080913306282F3327A3
:10337000220F331F220F331F80911D0290911E02D6
:103380002817390724F430931E0220931D028091E0
:103390002B0290912C0220911D0230911E02820F6F
:1033A000931F8050924090932C0280932B02809127
:1033B0001D0290911E0297FD039695958795959510
:1033C000879590931E0280931D02ECC080910D01A1
:1033D00090910E019C01220F331F280F391F8091FD
:1033E000A0019927880F991F880F991F280F391F4F
:1033F00037FF02C02D5F3F4FC90195958795959581
:10340000879590930E0180930D0190931C028093F9
:103410001B028091650660913506A0916703B0910B
:103420006803C0916903D0916A0381FF2AC077279E
:10343000882799279D01AE01D7FF04C021583F4F2F
:103440004F4F5F4FA7E05595479537952795AA951C
:10345000D1F70E94457D9B01AC0197FF04C0215C20
:103460003F4F4F4F5F4FF6E055954795379527955E
:10347000FA95D1F780911B0290911C02820F931F45
:1034800029C07727882799279D01AE01D7FF04C05F
:1034900021583F4F4F4F5F4FE7E055954795379580
:1034A0002795EA95D1F70E94457D9B01AC0197FFD6
:1034B00004C0215C3F4F4F4F5F4F76E055954795D5
:1034C000379527957A95D1F780911B0290911C0230
:1034D000821B930B90931C0280931B0280913606F3
:1034E000282F3327220F331F220F331F80911B02F7
:1034F00090911C02821793077CF080913706282F49
:103500003327220F331F220F331F80911B0290910C
:103510001C022817390724F430931C0220931B0245
:1035200080912B0290912C0220911B0230911C0261
:10353000820F931F8050924090932C0280932B0215
:1035400080911B0290911C0297FD0396959587959B
:103550009595879590931C0280931B0223C08091C0
:10356000BF0702C0809199079927880F991F880F7C
:10357000991F87559E4F12C08091C707F5CFFF272F
:10358000EE0FFF1FE55DF84F20813181220F331FC1
:1035900080912B0290912C02820F931F90932C020A
:1035A00080932B0280912B0290912C0255E08D3D4F
:1035B000950718F08CED95E005C08757914030F4E1
:1035C00087E791E090932C0280932B0220912B02AD
:1035D00030912C022C5B304030932C0220932B0234
:1035E00080912D0290912E02820F931F90932E02B4
:1035F00080932D022FC08091B00080648093B00032
:103600008CEB90E090932C0280932B0280912D0202
:1036100090912E0284549F4F90932E0280932D02FE
:1036200080911F02882321F080911B03853B20F4A9
:1036300080911F02823011F4469801C0469A809111
:103640002F028F5F80932F0290913806981710F405
:1036500010922F0281E080932A0220912B02309158
:103660002C0241E02F37340730F08FEF8093B30006
:103670002F5F30400FC02F3F3105C9F0C0F0A901C6
:103680004F5F50404F37510550F480E88093B300AE
:103690002058304030932C0220932B0212C08FEF21
:1036A0008093B30050932C0240932B020AC0809168
:1036B0002B028093B30010922C0210922B021092D6
:1036C0002A02FF91EF91DF91CF91BF91AF919F912E
:1036D0008F917F916F915F914F913F912F910F90BB
:1036E0000FBE0F901F90189510927C008FEC809366
:1036F0007A000895CF93DF931092360286E987BD52
:1037000083E090E00E94DC2EC82F863E08F4C65F5E
:10371000C8BD84E690E00E94481780911301909103
:1037200014018152934010F0C0EF02C0C530F8F090
:10373000C8BD82E390E00E94481787E394E09F931E
:103740008F938FEF92E19F938F93E0912704F091F5
:103750002804099580911301909114010F900F9006
:103760000F900F908152934010F4C550DFCF6C2F13
:1037700083E090E00E94E42ECF3018F0CCE8D0E057
:1037800002C0C0E0D0E0CA3FD105F8F4C7BD82E373
:1037900090E00E94481789E394E09F938F938FEF06
:1037A00092E19F938F93E0912704F091280409956B
:1037B00080911301909114010F900F900F900F9032
:1037C0008052934010F02196DECFC093FF05809188
:1037D000100680FF09C08C2F8A508B3E28F0809104
:1037E0004004806480934004C7BD8CE291E00E9455
:1037F0004817DF91CF910895EF92FF921F93CF93D7
:1038000010E080ED97E00E9426177C01CCE8133091
:1038100019F4CB3008F0C9E010E080914602909195
:1038200047028C5F934024F48091120181500AC0BA
:1038300080914602909147028750944034F08091E5
:1038400012018F5F8093120101C011E08091440248
:10385000909145028C5F934024F480911101815036
:103860000AC080914402909145028750944034F000
:10387000809111018F5F8093110101C01F5F8091C2
:103880004202909143028C5F934024F48091100196
:1038900081500AC080914202909143028750944027
:1038A000C4F0809110018F5F8093100113C08BE3EF
:1038B00094E09F938F938FEF92E19F938F93E0918A
:1038C0002704F091280409950F900F900F900F9006
:1038D0005FC01F5F82E18093700280916B028E7FD8
:1038E00080936B0285EA8093BC00809112018A303C
:1038F00040F4809140048160809340048AE080938A
:10390000120180911201863F40F080914004816055
:103910008093400485EF80931201809111018A30D9
:1039200040F4809140048260809340048AE0809358
:10393000110180911101863F40F080914004826026
:103940008093400485EF80931101809110018A30AB
:1039500040F4809140048460809340048AE0809326
:10396000100180911001863F40F0809140048460F6
:103970008093400485EF809310018091700288232A
:1039800039F0C7010E942F17882309F090CFF5CF97
:1039900010920F018FEC80937A0080910F018823A1
:1039A000E1F3CA3020F48AE090E00E944817C15049
:1039B00009F02DCF86E490E00E944817CF911F9127
:1039C000FF90EF9008951F920F920FB60F9211245F
:1039D000AF92BF92CF92DF92EF92FF920F931F931D
:1039E0002F933F934F935F936F937F938F939F9307
:1039F000AF93BF93EF93FF9380914F02282F33270C
:103A0000442755278F5F80934F02F90122313105FA
:103A100008F08CC3EA5BFF4F0C940B7E809178001A
:103A20009091790046C080917800909179002CC1E6
:103A30008091780090917900909352028093510286
:103A400057C180917803909179032091780030914B
:103A50007900821B930B9093F0058093EF05809182
:103A6000EF059091F00590935C0280935B025EC13C
:103A7000809178009091790020917A0330917B03B6
:103A8000821B930B9093FE058093FD058091FD05AD
:103A90009091FE0590935E0280935D0249C38091F0
:103AA0005502909156022091780030917900820F52
:103AB000931F909356028093550281E03AC3809100
:103AC0005302909154022091780030917900820F36
:103AD000931F909354028093530284E02AC38091F1
:103AE0001D0190911E019C01220F331F280F391FC9
:103AF000809178009091790063E070E00E94707D81
:103B0000260F371F369527953695279530931E013A
:103B100020931D0185E00DC380917800909179007C
:103B20004091740350917503841B950B90933D0253
:103B300080933C0280913C0290913D02029704F1F7
:103B400022E04E3E520784F4209150022B5F2093D6
:103B5000500225508091E8029091E902845F9140E3
:103B600018F4215F2093500280915002853684F131
:103B70004F5F5F4F5093750340937403845626C084
:103B800080913C0290913D028F5F9F4F0CF532E097
:103B900047325307ECF020915002255020935002F9
:103BA0002B5F8091E8029091E902845F914018F4C4
:103BB0002F5020935002809150028C394CF4415088
:103BC000504050937503409374038C598093500276
:103BD00081E080933B0280917800909179009093EE
:103BE000F6058093F50580913C0290913D029C0181
:103BF000442737FD4095542F80912F039091300337
:103C0000A0913103B0913203820F931FA41FB51FFF
:103C100080932F0390933003A0933103B09332032A
:103C200020912F03309130034091310350913203A2
:103C300057FF04C021503C4F4F4F5F4F0AE055954E
:103C40004795379527950A95D1F780912F03909145
:103C50003003A0913103B0913203821B930BA40B6C
:103C6000B50B80932F0390933003A0933103B0934F
:103C700032032EC18091530290915402209178001A
:103C800030917900820F931F9093540280935302D6
:103C900010924E0250C2809102018A3071F48091DC
:103CA0007800909179002091510230915202820F58
:103CB000931F01969695879517C040915102509198
:103CC0005202843158F02091780030917900240F0D
:103CD000351F8FEF97E0821B930B06C08091780011
:103CE00090917900840F951F909343028093420234
:103CF00086E01FC28091780390917903209178002B
:103D000030917900821B930B9093F0058093EF051F
:103D10008091EF059091F00520915B0230915C025B
:103D2000820F931F909341028093400287E001C26B
:103D3000809178009091790020917A0330917B03F3
:103D4000821B930B9093FE058093FD058091FD05EA
:103D50009091FE0520915D0230915E02820F931FCB
:103D600090933F0280933E02E3C12091550230912F
:103D700056028091780090917900280F391F309376
:103D8000560220935502809102018A3019F4220FC5
:103D9000331F04C0220F331F220F331F30935602EC
:103DA000209355022091550230915602C90137FDEA
:103DB0000796A3E095958795AA95E1F7909347021A
:103DC000809346028091570290915802820F931F70
:103DD00097FD019695958795909358028093570289
:103DE0002091840330918503821B930B90931C01D7
:103DF00080931B0120914C0230914D0280911B0158
:103E000090911C01280F391F37FF02C02F5F3F4FD1
:103E10003595279530934D0220934C024ECE20913C
:103E20005302309154028091780090917900280FCC
:103E3000391F3093540220935302809102018A303B
:103E400019F4220F331F04C0220F331F220F331F18
:103E50003093540220935302209153023091540224
:103E6000C90137FD079663E0959587956A95E1F757
:103E700090934502809344028091590290915A0296
:103E8000820F931F97FD01969595879590935A02FF
:103E9000809359022091820330918303821B930BFC
:103EA00090931A018093190120914A0230914B029C
:103EB0008091190190911A01280F391F37FF02C014
:103EC0002F5F3F4F3595279530934B0220934A0241
:103ED00083E02FC110924F0281E080930F01809107
:103EE0003202909133020196909333028093320212
:103EF0008091780090917900909314018093130140
:103F00008091130190911401AA27BB27A0905F0212
:103F1000B0906002C0906102D0906202A80EB91EFB
:103F2000CA1EDB1EA0925F02B0926002C0926102C4
:103F3000D0926202809163028F5F8093630282312C
:103F400008F4F6C08091150190911601A091170117
:103F5000B09118017C018D0123E0EE0CFF1C001FC5
:103F6000111F2A95D1F7E81AF90A0A0B1B0BEA0C64
:103F7000FB1C0C1D1D1D80913602992787FD909515
:103F8000A92FB92FBC01CD0126EC34E240E050E06E
:103F90000E94457DDC01CB01E81AF90A0A0B1B0BD4
:103FA000D801C7010496A11DB11DB7FF05C0D801F6
:103FB000C7010B96A11DB11D13E0B595A795979567
:103FC00087951A95D1F78093150190931601A093C8
:103FD0001701B09318018091F7059091F8057C01C5
:103FE0000027F7FC0095102F809115019091160184
:103FF000A0911701B0911801E81AF90A0A0B1B0BDE
:10400000E0920D03F0920E0300930F031093100340
:1040100020913702309138024091390250913A0292
:1040200057FF04C0215F3F4F4F4F5F4FF4E055955E
:10403000479537952795FA95D1F78091370290915A
:104040003802A0913902B0913A02821B930BA40B63
:10405000B50B8093370290933802A0933902B09346
:104060003A028091370290913802A0913902B091C2
:104070003A028E0D9F1DA01FB11F809337029093AF
:104080003802A0933902B0933A02809134029091A1
:104090003502AC01E5E0440F551FEA95E1F7481BF6
:1040A000590B8091370290913802A0913902B0915A
:1040B0003A02B7FF03C00F96A11DB11D74E0B5957C
:1040C000A795979587957A95D1F720910D03309113
:1040D0000E03281B390B63E0220F331F6A95E1F7AB
:1040E000240F351F37FF02C0215E3F4F45E0359555
:1040F00027954A95E1F73093350220933402D60193
:10410000C501D7FE03C00196A11DB11DB595A795A8
:104110009795879580935F0290936002A0936102C8
:10412000B093620289E08093630202C010924F0252
:1041300082E080934E0280914E0280937C008091B9
:104140004F02882319F08FEC80937A00FF91EF9152
:10415000BF91AF919F918F917F916F915F914F919F
:104160003F912F911F910F91FF90EF90DF90CF9093
:10417000BF90AF900F900FBE0F901F90189590E2D8
:10418000E0E2F1E08FE49193815087FFFCCF089546
:1041900090916602E0E2F1E0E90FF11D80839F5FFC
:1041A000909366020895EF92FF920F931F93CF931F
:1041B000DF932091640220FF0AC08091650288236A
:1041C00011F0815002C080911F018093650221FF90
:1041D0000CC09091650280911F01981719F41092FC
:1041E000650203C09F5F90936502822F992780FF2D
:1041F00004C081FF02C0109265020E94BF2080911E
:104200006502282F3327C8ECEC2EC0E2FC2EC091AB
:104210002704D09128048A3098F481E180936602C3
:104220003F932F9382E794E09F938F93FF92EF92B7
:10423000FE0109952DB73EB72A5F3F4F2DBF11C034
:1042400080E1809366023F932F9387E794E09F93EA
:104250008F93FF92EF92FE0109958DB79EB7069658
:104260008DBF20916502822F9927AA27BB27FC01C9
:10427000429710F00C94802BE85AFF4FB8ECEB2ECD
:10428000B0E2FB2EC0912704D09128040C940B7E41
:10429000109266028CE794E09F938F9308EC10E2F3
:1042A000FF92EF92FE01099584E1809366020F90E0
:1042B0000F900F900F9087E690E09F938F9380E58B
:1042C00090E09F938F931F921F92809102016AE06A
:1042D0000E94647D892F99279F938F93809102017B
:1042E0000E94647D99279F938F938CE894E09F931D
:1042F0008F93FF92EF92E0912704F09128040995A3
:1043000088E2809366022DB73EB7225F3F4F2DBFF4
:1043100085E796E09F938F930E94473099279F935C
:104320008F9381EA94E09F938F93FF92EF92E091B5
:104330002704F091280409958DB79EB708968DBF84
:1043400090914004992351F08CE380936602892F69
:1043500099279F938F938FEA94E085C690916C0282
:10436000992371F08CE380936602892F99279F939C
:104370008F9386EC94E09F938F931F930F9391C03C
:104380008091410484FF07C08CE3809366028BED2B
:1043900094E00C94122B80919101909192010697D8
:1043A00010F00C94892B8CE38093660288EE94E0E5
:1043B0000C94122B80911006A8ECEA2EA0E2FA2EA3
:1043C000C0912704D091280480FF74C01092660227
:1043D00080910D0390910E03A0910F03B0911003F3
:1043E000BC01CD0125E030E040E050E00E94B97D05
:1043F0003F932F9385EF94E09F938F93FF92EF92DB
:10440000FE01099584E1809366022DB73EB72A5FCD
:104410003F4F2DBF8091090390910A03A0910B0398
:10442000B0910C03BC01CD0125E030E040E050E04C
:104430000E94B97D3F932F9382E095E09F938F93E5
:10444000FF92EF92E0912704F0912804099588E209
:10445000809366028DB79EB706968DBF809113013B
:10446000909114019F938F938FE095E09F938F938A
:10447000FF92EF92E0912704F091280409958CE3D4
:10448000809366022DB73EB72A5F3F4F2DBF87B599
:1044900099279F938F938CE195E09F938F93FF9241
:1044A000EF92E0912704F091280409958DB79EB70B
:1044B00006962FC71092660289E295E09F938F932C
:1044C000FF92EF92FE01099584E1809366020F90BE
:1044D0000F900F900F9088E395E09F938F93FF923A
:1044E000EF92E0912704F0912804099588E28093E7
:1044F00066020F900F900F900F9081E495E09F93CC
:104500008F93FF92EF92E0912704F0912804099590
:104510008CE3809366020F900F900F900F9080E5D0
:1045200095E09F938F93FF92EF920C94162B10922D
:10453000660289E595E09F938F9308EC10E2FF9265
:10454000EF92FE01099584E1809366020F900F902F
:104550000F900F9080916F0390917003A091710361
:10456000B0917203B7FF04C081509C4FAF4FBF4F53
:10457000FAE0B595A79597958795FA95D1F7BF93EA
:10458000AF939F938F9386E695E09F938F931F93AE
:104590000F93E0912704F0912804099588E2809315
:1045A00066022DB73EB7285F3F4F2DBF809167034E
:1045B00090916803A0916903B0916A03B7FF04C0AA
:1045C00081509C4FAF4FBF4FEAE0B595A7959795A7
:1045D0008795EA95D1F7BF93AF939F938F9385E724
:1045E00095E09F938F931F930F93E0912704F09191
:1045F000280409958CE3809366028DB79EB70896D0
:104600008DBF80912D0390912E039F938F9384E80B
:1046100095E09F938F931F930F93E0912704F09160
:10462000280409952DB73EB72A5F3F4F0DC710925A
:10463000660280912F07909130079F938F9380910E
:104640002D0790912E079F938F9383E995E09F9379
:104650008F93FF92EF92FE01099584E180936602A9
:104660008DB79EB708968DBF809133079091340720
:104670009F938F9380913107909132079F938F93EF
:1046800083EA95E09F938F93FF92EF92E091270446
:10469000F0912804099588E2809366022DB73EB711
:1046A000285F3F4F2DBF80913707909138079F9328
:1046B0008F9380913507909136079F938F9383EB6B
:1046C00095E09F938F93FF92EF92E0912704F091F2
:1046D000280409958CE3809366028DB79EB70896EF
:1046E0008DBF80913B0790913C079F938F93809162
:1046F000390790913A079F938F9383EC95E0A2C07E
:104700001092660280910506E82FFF27EE0FFF1F2B
:10471000E55DF84F808191819F938F93809104068E
:10472000E82FFF27EE0FFF1FE55DF84F8081918195
:104730009F938F9383ED95E09F938F93FF92EF92DA
:10474000FE01099584E1809366028DB79EB70896B5
:104750008DBF80910706E82FFF27EE0FFF1FE55D55
:10476000F84F808191819F938F9380910606E82F67
:10477000FF27EE0FFF1FE55DF84F8081918188587C
:104780009F4F9F938F9383EE95E09F938F93FF921C
:10479000EF92E0912704F0912804099588E2809334
:1047A00066022DB73EB7285F3F4F2DBF80910906A7
:1047B000E82FFF27EE0FFF1FE55DF84F8081918105
:1047C00082599F4F9F938F9380910806E82FFF2770
:1047D000EE0FFF1FE55DF84F8081918182599F4F59
:1047E0009F938F9383EF95E09F938F93FF92EF9228
:1047F000E0912704F091280409958CE380936602E8
:104800008DB79EB708968DBF80910B06E82FFF27C6
:10481000EE0FFF1FE55DF84F8081918182599F4F18
:104820009F938F9380910A06E82FFF27EE0FFF1FBB
:10483000E55DF84F8081918182599F4F9F938F93BF
:1048400083E096E09F938F93FF92EF92E09127048D
:10485000F091280409952DB73EB7285F3F4FF4C566
:104860001092660283E196E09F938F9308EC10E22A
:10487000FF92EF92FE010995809102010F900F9037
:104880000F900F908A3009F0A1C084E180936602F6
:1048900080918403909185039C0197FF02C0295F5A
:1048A0003F4F287F821B930B9F938F9380918403AC
:1048B0009091850397FD079673E0959587957A9576
:1048C000E1F79F938F93209184033091850337FF05
:1048D00002C0295F3F4F63E0359527956A95E1F760
:1048E0008091460290914702821B930B9F938F9376
:1048F00081E296E09F938F931F930F93E09127049B
:10490000F0912804099588E2809366028DB79EB7DE
:104910000A968DBF80918203909183039C0197FF3B
:1049200002C0295F3F4F287F821B930B9F938F9379
:10493000809182039091830397FD079653E09595AC
:1049400087955A95E1F79F938F9320918203309139
:10495000830337FF02C0295F3F4F43E0359527951A
:104960004A95E1F78091440290914502821B930B96
:104970009F938F9382E396E09F938F931F930F9360
:10498000E0912704F091280409958CE38093660256
:104990002DB73EB7265F3F4F2DBF8091800390918A
:1049A00081039F938F938091800390918103209145
:1049B000420230914302821B930B9F938F9383E4B7
:1049C00096E09F938F931F930F93A3C38B3019F09F
:1049D000843108F4ADC084E1809366028091840341
:1049E000909185039C0197FF02C0215F3F4F207F7C
:1049F000821B930B97FD0196959587959F938F93B7
:104A0000809184039091850397FD0F9624E09595FE
:104A100087952A95E1F79F938F9320918403309196
:104A2000850337FF02C0295F3F4F83E03595279507
:104A30008A95E1F78091460290914702821B930B81
:104A40009F938F9381E596E09F938F931F930F938E
:104A5000E0912704F0912804099588E2809366028A
:104A60002DB73EB7265F3F4F2DBF809182039091B7
:104A700083039C0197FF02C0215F3F4F207F821B71
:104A8000930B97FD0196959587959F938F938091B2
:104A900082039091830397FD0F96B4E095958795D7
:104AA000BA95E1F79F938F9320918203309183030E
:104AB00037FF02C0295F3F4FA3E035952795AA95A0
:104AC000E1F78091440290914502821B930B9F93E2
:104AD0008F9383E696E09F938F931F930F93E091BC
:104AE0002704F091280409958CE3809366028DB722
:104AF0009EB70A968DBF809180039091810397FDA8
:104B00000196959587959F938F93809180039091BF
:104B100081032091420230914302821B930B9F93A9
:104B20008F9385E796E09F938F931F930F938ECE7D
:104B30008D3009F0EEC584E1809366028091120108
:104B400099279F938F93809184039091850397FD7C
:104B50000F96E4E095958795EA95E1F79F938F93FB
:104B6000209184033091850337FF02C0295F3F4FB6
:104B700073E0359527957A95E1F7809146029091FB
:104B80004702821B930B9F938F9384E896E09F9339
:104B90008F931F930F93E0912704F09128040995B8
:104BA00088E2809366028DB79EB70A968DBF80918A
:104BB000110199279F938F93809182039091830392
:104BC00097FD0F9664E0959587956A95E1F79F9319
:104BD0008F93209182033091830337FF02C0295FB6
:104BE0003F4F53E0359527955A95E1F78091440260
:104BF00090914502821B930B9F938F9388E996E0D7
:104C00009F938F931F930F93E0912704F0912804B3
:104C100009958CE3809366022DB73EB7265F3F4F20
:104C20002DBF8091100199279F938F9380918003CE
:104C30009091810397FD0196959587959F938F930A
:104C40008091800390918103209142023091430230
:104C5000821B930B9F938F938CEA96E09F938F9385
:104C60001F930F93E0912704F091280409958DB7C5
:104C70009EB70A964EC31092660280EC96E09F9310
:104C80008F93FF92EF92FE01099584E18093660273
:104C90000F900F900F900F9080917A0390917B036B
:104CA0009F938F9380913E0290913F029F938F93A9
:104CB0008DEC96E09F938F93FF92EF92E091270403
:104CC000F0912804099588E2809366022DB73EB7DB
:104CD000285F3F4F2DBF80917803909179039F9378
:104CE0008F9380914002909141029F938F938CED1E
:104CF00096E09F938F93FF92EF92E0912704F091BB
:104D0000280409958CE3809366028DB79EB70896B8
:104D10008DBF80917403909175039F938F938091C1
:104D20003C0290913D029F938F938BEE96E08ACD4B
:104D30001092660280911D0190911E016AE070E060
:104D40000E94847D9F938F9380911D0190911E01FD
:104D50006AE070E00E94847D7F936F938AEF96E013
:104D60009F938F93FF92EF92FE01099584E18093C8
:104D700066028DB79EB708968DBF809168089091A6
:104D800069086AE070E00E94707D9F938F93809124
:104D90006808909169086AE070E00E94707D7F93D6
:104DA0006F938EE097E09F938F93FF92EF92E09145
:104DB0002704F0912804099588E2809366022DB7B4
:104DC0003EB7285F3F4F2DBF80916A0890916B08D6
:104DD0009F938F9382E297E09F938F93FF92EF923E
:104DE000E0912704F091280409958CE380936602F2
:104DF0008DB79EB706968DBF80916C0890916D0817
:104E00009F938F9382E397E02EC11092660284E411
:104E100097E09F938F93FF92EF92FE01099584E1B3
:104E2000809366020F900F900F900F9080912B0748
:104E300090912C079F938F938DE497E09F938F938E
:104E4000FF92EF92E0912704F0912804099588E2FF
:104E5000809366028DB79EB706968DBF80911B0327
:104E600099279F938F938DE597E09F938F93FF9260
:104E7000EF92E0912704F091280409958CE3809348
:104E800066022DB73EB72A5F3F4F2DBF80912A079C
:104E9000992701979F938F938DE697E0FECA109212
:104EA00066028DE797E09F938F93FF92EF92FE014A
:104EB000099584E1809366020F900F900F900F90F8
:104EC0008091290390912A039F938F9385E897E01F
:104ED0009F938F93FF92EF92E0912704F091280423
:104EE000099588E2809366022DB73EB72A5F3F4F4F
:104EF0002DBF80912D0390912E039F938F9383E973
:104F000097E09F938F93FF92EF92E0912704F091A7
:104F1000280409958CE3809366028DB79EB70696A8
:104F20008DBF80912B0390912C039F938F9381EAE7
:104F300097E099C01092660280911C0399279F9375
:104F40008F938FEA97E09F938F93FF92EF92FE01EA
:104F5000099584E1809366028DB79EB706968DBF52
:104F600080911D0399279F938F938BEB97E09F93DD
:104F70008F93FF92EF92E0912704F0912804099516
:104F800088E2809366022DB73EB72A5F3F4F2DBF60
:104F900080911E0399279F938F9387EC97E09F93AF
:104FA0008F93FF92EF92E0912704F09128040995E6
:104FB0008CE3809366028DB79EB706968DBF809175
:104FC0001F0399279F938F9383ED97E04CC0109216
:104FD00066028091200399279F938F938FED97E02E
:104FE0009F938F93FF92EF92FE01099584E1809346
:104FF00066028DB79EB706968DBF809121039927D3
:105000009F938F938BEE97E09F938F93FF92EF92F6
:10501000E0912704F0912804099588E280936602C4
:105020002DB73EB72A5F3F4F2DBF809122039927AE
:105030009F938F9387EF97E09F938F93FF92EF92C9
:10504000E0912704F091280409958CE3809366028F
:105050008DB79EB706968DBF8091230399279F93A6
:105060008F9383E098E09F938F93FF92EF92D5CA3E
:10507000109266028FE098E09F938F93FF92EF92D9
:10508000FE01099584E1809366020F900F900F90C6
:105090000F908091A10199279F938F9387E198E0CA
:1050A0009F938F93FF92EF92E0912704F091280451
:1050B000099588E2809366028DB79EB706968DBFEC
:1050C00080911D0290911E029F938F9385E298E03C
:1050D0009F938F93FF92EF92E0912704F091280421
:1050E00009958CE3809366022DB73EB72A5F3F4F48
:1050F0002DBF8091330699279F938F93809132061D
:1051000099279F938F9383E398E09F938F93FF92C8
:10511000EF92E0912704F091280409958DB79EB78E
:105120000896F7C01092660281E498E09F938F93EF
:10513000FF92EF92FE01099584E1809366020F9041
:105140000F900F900F9080916104992787FD9095A3
:105150009F938F9380916004992787FD90959F93EB
:105160008F9381E598E09F938F93FF92EF92E09168
:105170002704F0912804099588E2809366022DB7F0
:105180003EB7285F3F4F2DBF80916204992787FD6E
:1051900090959F938F938091630499279F938F930A
:1051A00081E698E09F938F93FF92EF92E09127041E
:1051B000F091280409958CE3809366028DB79EB721
:1051C00008968DBF8091670499279F938F93809154
:1051D0006404992787FD90959F938F9381E798E0CA
:1051E00031CB1092660281E898E09F938F93FF92F3
:1051F000EF92FE01099584E1809366020F900F9073
:105200000F900F908091E50699278F7790709F936C
:105210008F938091DD0699278F7790709F938F935E
:105220008091D50699278F7790709F938F93809167
:10523000CD0699278F7790709F938F9381E998E09F
:105240009F938F93FF92EF92E0912704F0912804AF
:10525000099588E2809366028DB79EB70C968DBF44
:105260008091050799278F7790709F938F938091F6
:10527000FD0699278F7790709F938F938091F50605
:1052800099278F7790709F938F938091ED06992740
:105290008F7790709F938F9382EA98E09F938F937C
:1052A000FF92EF92E0912704F091280409958CE396
:1052B000809366022DB73EB7245F3F4F2DBF80918C
:1052C000250799278F7790709F938F9380911D0763
:1052D00099278F7790709F938F93809115079927C7
:1052E0008F7790709F938F9380910D0799278F7779
:1052F00090709F938F9383EB98E09F938F93FF928F
:10530000EF92E0912704F091280409958DB79EB79C
:105310000C968DBFFEC11092660284EC98E09F93BC
:105320008F93FF92EF92FE01099584E180936602CC
:105330000F900F900F900F908091E906992787FDAD
:1053400090959F938F938091E106992787FD909583
:105350009F938F938091D906992787FD90959F936E
:105360008F938091D106992787FD90959F938F9376
:1053700083ED98E09F938F93FF92EF92E091270443
:10538000F0912804099588E2809366022DB73EB714
:10539000245F3F4F2DBF80910907992787FD909586
:1053A0009F938F9380910107992787FD90959F93F5
:1053B0008F938091F906992787FD90959F938F93FE
:1053C0008091F106992787FD90959F938F9384EEA6
:1053D00098E09F938F93FF92EF92E0912704F091D2
:1053E000280409958CE3809366028DB79EB70C96CE
:1053F0008DBF80912907992787FD90959F938F9363
:1054000080912107992787FD90959F938F93809195
:105410001907992787FD90959F938F938091110786
:10542000992787FD90959F938F9385EF98E09F93A1
:105430008F93FF92EF92E0912704F0912804099551
:105440002DB73EB7245F3F4F2DBF63C11092660258
:1054500086E099E09F938F9308EC10E2FF92EF9221
:10546000FE01099584E1809366020F900F900F90E2
:105470000F908091E506881F8827881F97E0899FF5
:10548000C00111248D969F938F938091DD06881F14
:105490008827881F96E0899FC00111248D969F93CD
:1054A0008F938091D506881F8827881F95E0899F54
:1054B000C00111248D969F938F938091CD06881FF4
:1054C0008827881F9927880F991F880F991F8D9605
:1054D0009F938F9385E199E09F938F93FF92EF9233
:1054E000E0912704F0912804099588E280936602F0
:1054F0008DB79EB70C968DBF80910507881F8827B2
:10550000881F9BE0899FC00111248D969F938F93E4
:105510008091FD06881F8827881F9AE0899FC00117
:1055200011248D969F938F938091F506881F88276D
:10553000881F99E0899FC00111248D969F938F93B6
:105540008091ED06881F8827881F992723E0880F00
:10555000991F2A95E1F78D969F938F9389E299E0A1
:105560009F938F93FF92EF92E0912704F09128048C
:1055700009958CE3809366022DB73EB7245F3F4FB9
:105580002DBF80910D07881F8827881F9CE0899F69
:10559000C00111248D969F938F938DE399E09F9383
:1055A0008F93FF92EF92E0912704F09128040995E0
:1055B000809115072DB73EB72A5F3F4F2DBF87FF5C
:1055C00012C080E4809366028EE499E09F938F93EB
:1055D000FF92EF92E0912704F091280409950F9033
:1055E0000F900F900F9080911D0787FF12C084E4E9
:1055F0008093660281E599E09F938F931F930F93A9
:10560000E0912704F091280409950F900F900F90D6
:105610000F908091250787FF7CC088E48093660205
:1056200084E599E09F938F931F930F93E091270454
:10563000F091280409950F900F900F900F9069C07A
:105640001092660287E599E09F938F93FF92EF9205
:10565000FE01099584E1809366020F900F900F90F0
:105660000F908091F5019091F6019F938F9385E6BD
:1056700099E09F938F93FF92EF92E0912704F0912E
:105680002804099588E2809366028DB79EB7069636
:105690008DBF8091F7019091F8019F938F9382E7DE
:1056A00099E09F938F93FF92EF92E0912704F091FE
:1056B0002804099589E4809366022DB73EB72A5FD6
:1056C0003F4F2DBF8FE799E09F938F93FF92EF920B
:1056D000E0912704F09128040995809164020F90CD
:1056E0000F900F900F9083FF14C01092F80110924A
:1056F000F70160E070E08EE090E00E94F52E09C0B6
:1057000080911F01281719F4215020931F01109236
:10571000650210926402E6E0CDB7DEB70C94FC7D22
:10572000F999FECF92BD81BDF89A80B59927089569
:10573000F999FECF1FBA92BD81BD60BD0FB6F89436
:10574000FA9AF99A0FBE08954AEA20E030E0261747
:10575000370740F4FC018191480F2F5F3F4F261718
:105760003707C8F3842F99270895EAEA40E050E00C
:105770004617570778F49C01F999FECF32BD21BD39
:10578000F89A80B5E80F4F5F5F4F2F5F3F4F461786
:10579000570790F38E2F9927089581E0809306068E
:1057A00082E08093050683E08093040684E0809382
:1057B000070685E08093080686E08093090687E067
:1057C00080930A0688E080930B0689E080930C069C
:1057D0008AE080930D068BE080930E068CE0809328
:1057E0000F0608951F93CF93DF9384E580930306FC
:1057F00080910201843150F08AE080932306109258
:1058000045068BE180931F068EE40AC083E08093F7
:10581000230680E2809345068EE180931F0685E58E
:1058200080934206809343068AE68093100683E0C5
:1058300080936606AEE1A09311068FEF8093130666
:10584000EFE0E0931406A093120610921606F8E01B
:10585000F093170680E4809318061092190684E1ED
:10586000809315068EE080931A06B0E1B0931B0674
:105870001CE010931C06F0931D0686EE80931E0616
:1058800080E88093200650E55093210686E98093B6
:105890002206509324068093250676E07093260610
:1058A00081E2809327068DE2809328069AE5909303
:1058B000290680E280932B0610922C0610922D066A
:1058C00010922E0610922F0610924706109248064C
:1058D0001092490610924A0634E63093300648E2A8
:1058E0004093310661E0609365061092320627EF1F
:1058F00020933306709338068DE7809339068093A2
:105900003A0680933B063093340640933506109256
:1059100036062093370682E380933C0690933D063B
:1059200080933E061092640690933F065093400683
:1059300060934106B0934406309346068FE580930A
:105940004B0683EF80934D068AEA80934F0680933F
:105950005006E0934C06E0934E068EEF809351067E
:1059600030935206909353069093540690935506A5
:105970008BE48093560680935706809358061092C6
:10598000590670935A06F0935B0690935C06A093B9
:105990005D0630935E0630935F0682E0809360067A
:1059A00060932A061092620610926306A7E6B6E09C
:1059B000E0E7F1E0ED01019009921A95E1F760E767
:1059C00070E0CD01845690400E94A42B8093730612
:1059D000DF91CF911F910895CF93DF9384E580935A
:1059E000030680910201843150F08AE080932306FF
:1059F000109245068BE180931F068EE40AC083E077
:105A00008093230680E2809345068EE180931F06F3
:105A100085E580934206809343068AE680931006CC
:105A200083E0809366067EE1709311068FEF80938A
:105A300013069FE0909314067093120610921606B8
:105A400068E06093170680E48093180610921906A8
:105A5000909315068AE080931A0680E180931B06D6
:105A600056E050931C0660931D0686EE80931E063A
:105A700080E8809320062AE52093210688E780931A
:105A8000220620932406809325065093260681E261
:105A9000809327068DE28093280620932906E0E272
:105AA000E0932B0610922C0610922D0610922E06D3
:105AB00010922F061092470610924806109249063F
:105AC00010924A0644E64093300638E2309331069D
:105AD000F1E0F09365061092320697EF909333064B
:105AE000509338068DE78093390680933A06809369
:105AF0003B06409334063093350610923606909359
:105B0000370682E380933C0620933D0680933E0651
:105B10001092640620933F0680E5809340068CE354
:105B200080934106E09344069BE4909346068FE5FC
:105B300080934B0683EF80934D068AEA80934F064D
:105B40008093500684E180934C0680934E068EEF3E
:105B50008093510640935206209353062093540697
:105B600020935506909356069093570690935806A7
:105B70001092590650935A0660935B0620935C0678
:105B800070935D0640935E0640935F0682E08093CB
:105B90006006F0932A061092620610926306A7E64A
:105BA000B6E08CE0E7E7F1E0ED01019009928A951B
:105BB000E1F760E770E0CD01845690400E94A42B8D
:105BC00080937306DF91CF910895CF93DF9384E59F
:105BD0008093030680910201843150F08AE0809323
:105BE0002306109245068BE180931F068EE40AC0BF
:105BF00083E08093230680E2809345068EE18093C4
:105C00001F0685E580934206809343068AE68093CB
:105C1000100683E0809366066EE1609311068FEFB5
:105C2000809313069FE090931406609312061092DF
:105C3000160678E07093170680E480931806109299
:105C400019069093150670931A0690E190931B061F
:105C500056E050931C0670931D0686EE80931E0638
:105C600080E88093200634E63093210688E780930D
:105C7000220630932406809325065093260681E25F
:105C8000809327068DE2809328062AE52093290633
:105C900090932B0610922C0610922D0610922E0631
:105CA00010922F061092470610924806109249064D
:105CB00010924A063093300648E240933106E1E004
:105CC000E09365061092320697EF90933306509357
:105CD00038068DE78093390680933A0680933B0619
:105CE000309334064093350610923606909337066B
:105CF00082E380933C0620933D0680933E061092FB
:105D0000640620933F0680E58093400696E49093D6
:105D1000410680E280934406909346068FE5809387
:105D20004B0683EF80934D068AEA80934F0680935B
:105D3000500660934C0660934E068EEF809351069A
:105D40003093520620935306209354062093550611
:105D50008BE48093560680935706809358061092E2
:105D6000590650935A0670935B0620935C06609325
:105D70005D0630935E0630935F0682E08093600696
:105D8000E0932A061092620610926306A7E6B6E038
:105D90008CE0EFE7F1E0ED01019009928A95E1F7DF
:105DA00060E770E0CD01845690400E94A42B809360
:105DB0007306DF91CF910895F999FECF92BD81BD11
:105DC000F89A80B599270895F999FECF1FBA92BD28
:105DD00081BD60BD0FB6F894FA9AF99A0FBE089586
:105DE00060E97BE20E94D37B089548E95BE20E9470
:105DF0000D7C0895EF92FF920F931F93CF93C82FBE
:105E00008150853008F0C3E081E7C89F80011124EC
:105E100083EFE82E8FEFF82EE00EF11E60E770E0C2
:105E2000C7010E94B52B682F98012D593F4F8FB3A2
:105E30009927AC014270507081FDF9CF32BD21BD70
:105E4000F89A80B5861711F0CA0121C08FB399273F
:105E50009C012270307081FDF9CFF2BCE1BCF89A50
:105E600080B5843511F0C90112C081E7C89FC00117
:105E700011240D9720E93BE241E750E0BC0183E0AB
:105E800096E00E94AE7B0E94116981E090E0CF9184
:105E90001F910F91FF90EF900895282F863010F0FA
:105EA00025E003C0882309F421E0F999FECF1FBA49
:105EB00082E090E092BD81BD20BD0FB6F894FA9AC1
:105EC000F99A0FBE0895CF93C82F809103068435A9
:105ED00009F042C0C63010F0C5E003C0CC2309F47D
:105EE0003BC060E770E083E096E00E94A42B8093C3
:105EF000730681E7C89FC001112428E93BE241E70E
:105F000050E063E076E00D970E94EB7B28E93BE2EE
:105F10004CE050E064E076E080E590E00E94EB7BAE
:105F20006CE070E084E096E00E94A42B282FF999A1
:105F3000FECF1FBA8CE590E092BD81BD20BD0FB6AB
:105F4000F894FA9AF99A0FBE8C2F0E944D2F0E9456
:105F5000116981E090E002C080E090E0CF91089567
:105F60006DE470E088EE93E00E94B52B482F8FB36C
:105F700099279C012270307081FDF9CF85E394E070
:105F800092BD81BDF89A80B5841779F48FB39927B3
:105F90009C012270307081FDF9CF88EE93E092BDB4
:105FA00081BDF89A80B5813011F0C901089520E9CA
:105FB0003BE24EE450E068EE73E084E796E00E9436
:105FC000AE7B81E090E00895809174068130A9F461
:105FD0006DE470E084E796E00E94A42B8093C106F4
:105FE00028E93BE24EE450E064E776E088EE93E097
:105FF0000E94EB7B81E090E0089580E090E00895BE
:10600000CF93DF9381E080937406E4E7F6E08FE0BE
:10601000158616861786108A8150349687FFF8CF2A
:1060200080E4809381068093820610928306809399
:1060300084068093850690EC9093860610928706DE
:10604000809388068093890610928A0690938B0627
:1060500090938C0680938D0610928E0680938F0607
:1060600090939006A5E7B6E087E0E9E8F1E0ED015E
:10607000019009928A95E1F76DE470E0CD010197F6
:106080000E94A42B8093C106DF91CF910895F999C6
:10609000FECF82E090E092BD81BDF89A80B5282FB6
:1060A000863078F023E0322FF999FECF1FBA82E0D4
:1060B00090E092BD81BD30BD0FB6F894FA9AF99A7E
:1060C0000FBE822F99270895DF92EF92FF920F93D0
:1060D0001F93CF93FF24DF2CEF2C81E090E00E94F0
:1060E000DC2E843539F031E0E32E64E581E090E088
:1060F0000E94E42E6CE070E080E590E00E94B52BF9
:10610000C82FF999FECF8CE590E092BD81BDF89A39
:1061100080B58C1711F421E0D22EC1E001E010E02F
:10612000EE2029F48C2F0E94FA2E8823C1F591E0ED
:10613000F92E1F930F9387E899E09F938F938FEF2A
:1061400092E19F938F93E0912704F09128040995A1
:106150008DB79EB706968DBF0230110549F003300A
:1061600011054CF40130110531F40E94F22B05C0E9
:106170000E94EC2C02C00E94E52DDD2059F020E9A0
:106180003BE24CE050E060E570E084E096E00E9485
:10619000AE7B02C00E94CD2B8C2F0E94632FCF5F5D
:1061A0000F5F1F4FC63008F4BBCFFF2019F083E00C
:1061B0000E944D2F0E944730C82F0E94FA2E8C2F2C
:1061C00099279F938F938DEA99E09F938F930FEF79
:1061D00012E11F930F93E0912704F0912804099591
:1061E0008DB79EB706968DBFEE2021F40E94B02F8A
:1061F000882399F486EC99E09F938F931F930F93D4
:10620000E0912704F091280409950E9400300E9433
:10621000E42F0F900F900F900F901092020690E0D5
:10622000E1E8F6E0CFE08081349618160CF49F5F29
:10623000C150C7FFF8CF90930206892F99279F93EB
:106240008F9385E796E09F938F9387EE99E09F93D6
:106250008F931F930F93E0912704F09128040995E1
:106260008DB79EB708968DBF88E09AE09F938F9375
:106270001F930F93E0912704F091280409950F9044
:106280000F900F900F90CF911F910F91FF90EF9073
:10629000DF9008959FB7F8943998389A88B1836051
:1062A00088B98091B9008C7F8093B9008AE280938D
:1062B000B8001092700210926E0210926D02EAEC19
:1062C000F6E08BE010821182128213821482158212
:1062D000168217828150389687FFF4CF9FBF0895AA
:1062E0001092700284E98093BC0010926E021092AA
:1062F0006D0280E88093BC001092BD001092BA003D
:106300001092BB001092B9001092B8000E944A315E
:106310001092BB0085E88093BC0080916B02826084
:1063200080936B0208951F920F920FB60F92112463
:106330002F933F934F935F938F939F93EF93FF938D
:1063400080917002282F3327442755278F5F809331
:106350007002F9012731310508F0B3C2E659FF4F49
:106360000C940B7E80916E028C3090F480916E02C2
:106370008F5F80936E0280916E02E82FFF27EE0FF1
:10638000FF1FEE0FFF1FEC58F94F8585181654F7C5
:1063900080916E028C3070F010926A021092690245
:1063A00010926E0285E08093700280916D02880FDA
:1063B0008D5A04C080916E02880F8E5A8093BB0064
:1063C00085E874C280916E02E82FFF2783E0EE0F0C
:1063D000FF1F8A95E1F7E653F94F81818093BB0057
:1063E00085E88093BC0080916E02E82FFF27EE0FB6
:1063F000FF1FEE0FFF1FEE0FFF1FE653F94F8081C7
:1064000080FF91C080916E02E82FFF27EE0FFF1FE3
:10641000EE0FFF1FEE0FFF1FE653F94F8281882317
:1064200029F080910206873008F45FC280916902EA
:1064300090916A02892B09F058C28091670290916D
:106440006802892B09F051C26EC080916E0221E072
:1064500030E002C0220F331F8A95E2F78091670275
:106460009091680228233923232B79F080916E02C2
:10647000E82FFF27EE0FFF1FEE0FFF1FEE0FFF1F8E
:10648000E653F94F80E184830DC080916E02E82FBE
:10649000FF27EE0FFF1FEE0FFF1FEE0FFF1FE6534C
:1064A000F94F148280916E02E82FFF2753E0EE0F20
:1064B000FF1F5A95E1F7E653F94F8481282F3327C0
:1064C00043E0220F331F4A95E1F780916E02E82FD7
:1064D000FF2793E0EE0FFF1F9A95E1F7E653F94F80
:1064E00082818770822B8093BB0085E88093BC00FB
:1064F00020916E0281E090E002C0880F991F2A95DA
:10650000E2F72091690230916A0282239323892B5A
:1065100051F082EC96E0909374028093730288E0CD
:1065200080937502E2C184E080C1E0917302F09132
:10653000740281918093BB0085E88093BC00F09346
:106540007402E0937302809175028150809375020A
:10655000882309F4CAC183E068C18091B9008033FF
:1065600051F580917102882329F480916E028F5F2A
:106570008093710280916E02E82FFF2783E0EE0F77
:10658000FF1F8A95E1F7E653F94F838199278F77AB
:1065900090708F3791057CF480916E02E82FFF2771
:1065A000EE0FFF1FEE0FFF1FEE0FFF1FE653F94F19
:1065B00083818F5F83831092700284E98093BC0093
:1065C0008AE090E0909392018093910180916E0215
:1065D0008F5F80936E021092700262C18091B90049
:1065E0008034A9F180916D02E82FFF27EE0FFF1F85
:1065F000EE0FFF1FEE0FFF1FE653F94F83818F77DA
:10660000838380916D028F5F80936D0280916D0214
:106610008C30A0F010926D02109268021092670206
:10662000809172028F5F809372028C3038F01092EA
:10663000720280916B028D7F80936B0280916B025E
:10664000816080936B021092700284E971C0809126
:106650006D02E82FFF27EE0FFF1FEE0FFF1FEE0F5B
:10666000FF1FE653F94F83818068838380916D0219
:10667000E82FFF27EE0FFF1FEE0FFF1FEE0FFF1F8C
:10668000E653F94F808180FF2FC080916D02E82F83
:10669000FF2753E0EE0FFF1F5A95E1F7E653F94F3E
:1066A00084819927009751F04097D9F582EC96E0C4
:1066B000909374028093730288E031C080916D02E0
:1066C000992743E0880F991F4A95E1F78153994F25
:1066D000909374028093730290916D028091720284
:1066E0009817E1F483E01BC080916D02992733E095
:1066F000880F991F3A95E1F78153994F909374024F
:106700008093730280916B0281FD06C090916D02AF
:1067100080917202981711F482E001C081E08093A9
:10672000750280917502813011F485E801C085EC15
:106730008093BC008091710280936C021092710270
:10674000D4C0E0917302F09174028091BB00808309
:1067500080917302909174020196909374028093D9
:10676000730280917502815080937502823010F01F
:1067700085EC58C0813011F485E854C080916B02DB
:1067800081FF2DC08091E70280FD1DC080916D02C8
:10679000E82FFF2723E0EE0FFF1F2A95E1F7E653CE
:1067A000F94F86818A3F79F480916D02E82FFF27A7
:1067B00093E0EE0FFF1F9A95E1F7E653F94F8081C2
:1067C000816080830CC080916D02E82FFF2783E0F9
:1067D000EE0FFF1F8A95E1F7E653F94F1082809183
:1067E0006D028F5F80936D0280916D028C30A0F0FE
:1067F00010926D02109268021092670280917202EC
:106800008F5F809372028C3038F010927202809108
:106810006B028D7F80936B021092700284E98093EB
:10682000BC0049C08093BC0086E0809370025DC0CC
:1068300088E9C4CD80916F02880F805FBFCD8091C1
:106840006F0299278130910561F0823091051CF427
:10685000892B21F04AC0029739F047C0809112017C
:10686000ADCD80911101AACD80911001A7CD80E816
:10687000A5CD1092700284E98093BC008AE090E07C
:10688000909392018093910180916F02823088F4FD
:1068900080916F028F5F80936F0282E1809370021C
:1068A00080916B028E7F80936B0285EA8093BC009F
:1068B0001CC010926F0280916B02816080936B020A
:1068C00014C01092700284E98093BC0080916B0226
:1068D000816080936B028AE090E0909392018093B4
:1068E000910110926E0210926D02FF91EF919F91B3
:1068F0008F915F914F913F912F910F900FBE0F900D
:106900001F9018951F93CF93DF93182F8091120338
:10691000882321F480910202882319F081E090E01D
:1069200097C01D3008F092C01123B1F0E12FFF276E
:1069300023E0EE0FFF1F2A95E1F7E653F94F359755
:106940008081359688230CF081C03897808180FD46
:1069500003C083E090E07CC08091C206823019F0D1
:1069600084E090E075C067E070E082EC96E00E9401
:10697000A42B9091C906891719F085E090E068C0B2
:1069800080ED97E00E942617EC0180916B0280FD5C
:1069900005C0CE010E942F178823B9F3112319F4E3
:1069A0008FEF90E00BC0212F33272150304081E042
:1069B00090E002C0880F991F2A95E2F790936A022F
:1069C00080936902A1E0B0E0EAECF6E040E050E03C
:1069D0006BE0CD01042E02C0880F991F0A94E2F7E4
:1069E0002091690230916A0282239323892B11F04E
:1069F0001182128261504F5F5F4F389667FFE9CF77
:106A000010926E021092700280916B028E7F8093C2
:106A10006B0285EA8093BC0080916B0280FD05C00B
:106A2000CE010E942F178823B9F3809169029091BB
:106A30006A02892B29F0CE010E942F17882311F3B7
:106A40008091690290916A02009711F082E090E0D3
:106A5000DF91CF911F9108950F931F93CF93DF93F1
:106A6000982F80911203882321F4809102028823B9
:106A700019F081E090E092C09D30A0F4992319F4C0
:106A800086E090E08BC0C92FDD27FE0133E0EE0FDA
:106A9000FF1F3A95E1F7E653F94F35978081359618
:106AA00087FD03C082E090E079C03897808180FD47
:106AB00003C083E090E072C080ED97E00E9426174B
:106AC0008C0180916B0280FD05C0C8010E942F17C8
:106AD0008823B9F3219721E030E0C90102C0880F73
:106AE000991FCA95E2F79093680280936702D901D3
:106AF000EAECF6E040E050E06BE0CD01042E02C08D
:106B0000880F991F0A94E2F720916702309168027A
:106B100082239323892B11F01182128261504F5FDF
:106B20005F4F389667FFE9CF10926D021092C20650
:106B30001092C9061092700280916B028E7F809332
:106B40006B0285EA8093BC0080916B0280FD05C0DA
:106B5000C8010E942F178823B9F380916702909192
:106B60006802892B29F0C8010E942F17882311F38E
:106B70008091C206823019F084E090E00FC067E097
:106B800070E082EC96E00E94A42B9091C9068917D0
:106B900019F085E090E002C080E090E0DF91CF91B5
:106BA0001F910F91089589E1AFE5B7E0EBE2F7E0BF
:106BB00011821082329611961C921E92129681506A
:106BC00087FFF6CF10928103109280031092830307
:106BD00010928203109285031092840308951F92ED
:106BE0000F920FB60F9211240F931F932F933F9381
:106BF0004F935F936F937F938F939F93AF93BF93C5
:106C0000CF93DF93EF93FF938091660682FDCFC011
:106C10004091860050918700809177029091780290
:106C2000481B590B809186009091870090937802C1
:106C300080937702CA018D549440A0917902B0915B
:106C40007A02835F9A4178F48091790280932A07CF
:106C5000149714F01092930181E090E090937A02DF
:106C60008093790207C2AD30B1050CF003C2CA01AE
:106C70008B5F9040845B914008F074C0425D51404E
:106C8000FD01EA0FFB1FE55DF84F80819181FA015C
:106C9000E81BF90BCF01F7FF03C0909581959F4F3B
:106CA00006975CF480911B03883C20F480911B03C1
:106CB000865F01C088EC80931B03FD01EA0FFB1F78
:106CC000E55DF84F808191819C01220F331F280FD1
:106CD000391F240F351F37FF02C02D5F3F4FE901D9
:106CE000D595C795D595C795CA0101968C179D076F
:106CF00014F4219706C041505040C417D5070CF436
:106D0000219680911B03833CE0F08D010A0F1B1F2D
:106D1000F801E55DF84F808191819E01281B390BB8
:106D2000C90163E070E00E94847DCB01880F991F48
:106D3000860F971F015A184FD80111969C938E9376
:106D400007C0AA0FBB1FA15AB84F11961C921E92E2
:106D5000E0917902F0917A02EE0FFF1FE55DF84FA6
:106D6000D183C0832091790230917A022F5F3F4F07
:106D700030937A022093790280910201843108F0E5
:106D800079C12530310511F45D9A01C05D9880917B
:106D9000790290917A028630910511F45C9A01C0D3
:106DA0005C98079711F45B9A65C15B9863C1409149
:106DB00086005091870080917B0290917C02481B55
:106DC000590B809186009091870090937C0280936C
:106DD0007B02CA018D5494406091E502835F9A4121
:106DE00008F07AC06093760280917602843008F4CD
:106DF00053C090912A0780917602981709F04CC0F1
:106E00005091E6025B3008F43FC01092930110925B
:106E1000E50240E05F31C0F0E42FFF27EE0FFF1FD7
:106E20009F012F543D4FDF01A55DB84F8D919C917F
:106E3000D9018D939C93DF01A15AB84F8D919C91FC
:106E4000E553FD4F91838083E42FFF27EE0FFF1F53
:106E50009F01255D384FDF01A358BD4F8D919C9157
:106E6000D90111969C938E93DF01A956BD4F8D9148
:106E70009C91E15AF84F91838083842F8F5F482F34
:106E80008D3040F28093E5028091E6028F3FB9F0A9
:106E90008F5F8093E60213C08091E602853620F072
:106EA0008AE08093E60202C01092E602809102011D
:106EB0008A3011F0843110F0289A01C0289881E0BE
:106EC0008093E50280911203882309F0D3C080915A
:106ED000760280932A07CEC06D3008F0A3C0CA01A5
:106EE0008B5F9040845B914008F07EC0425D5140D2
:106EF000E62FFF27EE0FFF1FE358FD4F80819181A2
:106F0000FA01E81BF90BCF0105960B97B0F48091BD
:106F1000E6028A3120F080911B03865F05C08B302A
:106F200028F080911B038E5F80931B0380911B03CD
:106F3000893C18F088EC80931B03E62FFF27EE0FA7
:106F4000FF1FE358FD4F808191819C01220F331F69
:106F5000280F391F240F351F37FF02C02D5F3F4F09
:106F6000E901D595C795D595C795CA0101968C17A6
:106F70009D0714F4219706C041505040C417D5070F
:106F80000CF4219680911B038E3BD8F0E62FFF274F
:106F9000EE0FFF1FDF01A358BD4F8D919C919E0105
:106FA000281B390BC90163E070E00E94847DCB018E
:106FB000880F991F860F971FE956FD4F9183808395
:106FC00008C0E62FFF27EE0FFF1FE956FD4F118285
:106FD00010828091E502E82FFF27EE0FFF1FE35894
:106FE000FD4FD183C08309C0809102018A3011F026
:106FF000843110F0289A01C02898809102018431D0
:1070000088F48091E502853011F45D9A05C05D98A1
:10701000863011F45C9A05C05C98873011F45B9A55
:1070200001C05B988091E502843120F48F5F8093EA
:10703000E50220C08431F1F4809102018A3011F020
:10704000843110F0289A01C028988EE18093E502DF
:107050002CE0CFE5D7E0A1EBB2E0EBE2F7E08D91D9
:107060009D919183808332961982188222962150B5
:1070700027FFF5CFFF91EF91DF91CF91BF91AF91B6
:107080009F918F917F916F915F914F913F912F9140
:107090001F910F910F900FBE0F901F901895EF92B8
:1070A000FF920F931F9380911F069927880F991FB6
:1070B000880F991F7C010027F7FC0095102F809105
:1070C0006F0390917003A0917103B0917203BC01A2
:1070D000CD01A80197010E94B97D3093AF0520939F
:1070E000AE058091670390916803A0916903B09108
:1070F0006A03BC01CD01A80197010E94B97D3093BC
:10710000B1052093B0058091E5079091E60797FDC2
:10711000039695958795959587959093B30580935C
:10712000B2058091F5079091F60797FD0396959526
:107130008795959587959093B5058093B405809133
:107140008003909181032091420230914302821B7F
:10715000930B9093B7058093B60580910D039091A2
:107160000E03A0910F03B0911003BC01CD0125E0E7
:1071700030E040E050E00E94B97D3093B9052093A3
:10718000B80580913C0290913D029093BB0580939D
:10719000BA0580912D0390912E039093BF058093A3
:1071A000BE0580911D0190911E019093C1058093B1
:1071B000C00580911B0399279093C3058093C20556
:1071C0008091F1079091F207A091F307B091F40735
:1071D000209195013091960140919701509198012D
:1071E000BC01CD010E94B97D3093C5052093C40533
:1071F0008091CB0699279093C7058093C60580910F
:10720000D30699279093C9058093C8058091DB0622
:1072100099279093CB058093CA058091E30699271F
:107220009093CD058093CC058091EB0699279093A0
:10723000CF058093CE058091F30699279093D105D1
:107240008093D0058091FB0699279093DF0580936A
:10725000DE058091030799279093E1058093E0056F
:1072600080910B0799279093E3058093E205809125
:10727000130799279093E5058093E40580911D02FB
:1072800090911E029093D7058093D605809168084F
:10729000909169089093DB058093DA0580916C08E2
:1072A00090916D089093DD058093DC0580916E08C8
:1072B00099279093E9058093E8058091F8039091D0
:1072C000F9039093EB058093EA058091F603909182
:1072D000F7039093ED058093EC058091400488239B
:1072E00021F480914104882321F08091AD058160D3
:1072F00003C08091AD058E7F8093AD051F910F91E6
:10730000FF90EF9008951F93CF93DF93182FEB0119
:10731000809112038823A1F411501F3F89F0D0936C
:107320002202C09321028091210290912202892B96
:10733000D1F7CE018C0F9D1F0E943B17115078F79B
:10734000DF91CF911F910895CF93DF938091020138
:107350008D3011F40E94FC1B10927A00809146023D
:10736000909147029093AC078093AB0780914402C1
:107370009091450290939D0780939C0780914202D3
:10738000909143029093EB078093EA0720913E028D
:1073900030913F02C901880F991F880F991F820FF2
:1073A000931F820F931F9093E6078093E507209128
:1073B000400230914102C901880F991F880F991F1F
:1073C000820F931F820F931F9093F6078093F50708
:1073D0008FEC80937A00ACE1B3E0C8E0D6E097E0B0
:1073E0008991E82FFF27EE0FFF1FE55DF84F019011
:1073F000F081E02DE259FF4F1E161F061CF0E0E061
:10740000F0E005C0EF3FF10514F0EFEFF0E08C91F4
:10741000282F3327E217F30714F4815004C02E17E6
:107420003F0714F48F5F8C939150119697FFD8CF3C
:10743000809142069927AA27BB27BC01CD0124ECE5
:1074400039E040E050E00E94457DDC01CB018093B3
:10745000B5019093B601A093B701B093B8018091A4
:1074600043069927AA27BB27BC01CD010E94457D71
:10747000DC01CB018093B1019093B201A093B301E1
:10748000B093B401DF91CF910895A0E0B0E0EBE4B8
:10749000FAE30C94DA7D882EC0E0D0E07E016E0124
:1074A00010924004469AD0937B03C0937A03D09302
:1074B0007903C0937803D0937503C0937403D0937A
:1074C0008503C0938403D0938303C0938203D09336
:1074D0008103C093800310929E0110929D0110922F
:1074E00036020E94A43984E690E00E9448170E9468
:1074F000A4398091100680FF10C0809113019091F3
:107500001401875B934038F480911301909114012A
:107510008E5E924010F40E947A1B0FE18AE090E0A8
:107520000E9448178091420290914302C80FD91FD0
:107530008091460290914702E80EF91E8091440224
:1075400090914502C80ED91E015007FFE7CF970161
:10755000205F3F4F369527953695279530938503C5
:1075600020938403C60140969695879596958795B6
:1075700090938303809382036096F5E0D695C79538
:10758000FA95E1F7D0938103C093800390937F0332
:1075900080937E0330937D0320937C03882009F43D
:1075A00041C08091E5079091E60797FF03C0909551
:1075B00081959F4F6CE070E00E94847D9B017093E9
:1075C0007B0360937A038091F5079091F60797FF0C
:1075D00003C0909581959F4F6CE070E00E94847D80
:1075E00070937903609378038091F5059091F60587
:1075F0009093750380937403B90184E090E00E9436
:10760000F52E609178037091790386E090E00E94F6
:10761000F52E609174037091750388E090E00E94EC
:10762000F52E65C084E090E00E94F02E90937B03DD
:1076300080937A0386E090E00E94F02E9093790385
:107640008093780388E090E00E94F02E9C01909354
:1076500075038093740380917A0390917B0381502A
:10766000984050F48091780390917903815098402C
:1076700018F421503440D8F189E29AE09F938F9317
:107680008FEF92E19F938F93E0912704F09128046C
:1076900009958091E5079091E60797FF03C09095C3
:1076A00081959F4F6CE070E00E94847D70937B0316
:1076B00060937A038091F5079091F60797FF03C0D6
:1076C000909581959F4F6CE070E00E94847D70934F
:1076D0007903609378038091F5059091F605909376
:1076E0007503809374030F900F900F900F9010927A
:1076F000AC071092AB0710929D0710929C07109256
:10770000EB071092EA0784E690E00E944817809108
:107710003E0290913F029C01220F331F220F331F24
:10772000280F391F280F391F3093E6072093E507EC
:1077300080914002909141028C01000F111F000FB7
:10774000111F080F191F080F191F1093F607009338
:10775000F50780911F06C82EDD24EE24FF24442760
:1077600037FD4095542FC701B6010E94457D4B015E
:107770005C0160936F037093700380937103909327
:1077800072039801442737FD4095542FC701B60175
:107790000E94457DDC01CB018093670390936803D1
:1077A000A0936903B0936A0380924B0390924C03B9
:1077B000A0924D03B0924E038093430390934403F1
:1077C000A0934503B093460310923F0310924003E9
:1077D000109241031092420380911501909116017D
:1077E000A0911701B09118019093F8058093F705C7
:1077F000109235021092340210922F03109230032F
:10780000109231031092320380912D0390912E0338
:1078100090932C0380932B030E94A86482E390E052
:107820009093220280932102809142069927AA27F1
:10783000BB27BC01CD0124EC39E040E050E00E94C0
:10784000457DDC01CB018856954CAF4FBF4F8093EF
:10785000B5019093B601A093B701B093B8018091A0
:1078600043069927AA27BB27BC01CD010E94457D6D
:10787000DC01CB018856954CAF4FBF4F8093B101CF
:107880009093B201A093B301B093B40110929A0106
:107890001092990180912D0390912E03AA2797FDB4
:1078A000A095BA2F209195013091960140919701B2
:1078B00050919801BC01CD010E94457DDC01CB01B6
:1078C0008093F1079093F207A093F307B093F40726
:1078D000109226031092250381E0809301010E94FB
:1078E00011698091E70284608093E7028FEF8093B3
:1078F00063081092640880E280936508CCE1D3E0CD
:10790000A8E0B6E007E08D91E82FFF27EE0FFF1FFC
:10791000E55DF84F8081918182598993015007FF7D
:10792000F2CF84E680931B0380911F02882311F01D
:10793000469A579A80918403909185038056994086
:10794000815C9B4228F080914004816080934004D8
:10795000809182039091830380569940815C9B4281
:1079600028F08091400482608093400480918003DD
:10797000909181038C5291408957954028F08091D5
:10798000400484608093400480917A0390917B034B
:107990008C529140835C914028F080914004886033
:1079A0008093400480917803909179038C529140A8
:1079B000835C914028F08091400480618093400472
:1079C000809174039091750380509240835591404B
:1079D00028F080914004806280934004ECE0CDB7B1
:1079E000DEB70C94F67DA3E1B0E0E9EFFCE30C9484
:1079F000D47D809180039091810320914202309147
:107A00004302821B930B9093EB078093EA078091CC
:107A10004C0290914D0297FD07969C0153E03595DD
:107A200027955A95E1F73093AC072093AB078091E7
:107A30004A0290914B0297FD079643E095958795F2
:107A40004A95E1F790939D0780939C073093B70781
:107A50002093B6079093AF078093AE078091E50718
:107A60009091E607AC01440F551F480F591F209114
:107A70003E0230913F02C901880F991F880F991F5C
:107A8000820F931F820F931F480F591F57FF02C089
:107A90004D5F5F4F55954795559547955093E60730
:107AA0004093E5078091F5079091F607AC01440FEC
:107AB000551F480F591F2091400230914102C901C2
:107AC000880F991F880F991F820F931F820F931F92
:107AD000480F591F57FF02C04D5F5F4F559547959F
:107AE000559547955093F6074093F50720913E0230
:107AF00030913F02C901880F991F880F991F820F8B
:107B0000931F820F931F9C01442737FD4095542FEC
:107B100080915F0390916003A0916103B091620333
:107B2000820F931FA41FB51F80935F039093600380
:107B3000A0936103B093620320914002309141020F
:107B4000C901880F991F880F991F820F931F820FF9
:107B5000931F9C01442737FD4095542F80915B0370
:107B600090915C03A0915D03B0915E03820F931F1F
:107B7000A41FB51F80935B0390935C03A0935D03E8
:107B8000B0935E038091C0079091C10720913E029F
:107B900030913F02820F931F9093C1078093C007DB
:107BA0008091ED079091EE072091400230914102C3
:107BB000820F931F9093EE078093ED0780917603D9
:107BC0009091770301969093770380937603809149
:107BD000F5059091F6052091740330917503821B91
:107BE000930B9C01442737FD4095542F80915703F8
:107BF00090915803A0915903B0915A03820F931F9B
:107C0000A41FB51F8093570390935803A093590363
:107C1000B0935A038FEC80937A0010920F01209159
:107C20004703309148034091490350914A03298703
:107C30003A874B875C8729543B46414050402CF0A3
:107C400028E43BE641E050E00DC089859A85AB858C
:107C5000BC85885B9449AE4FBF4F4CF428EB34E9A8
:107C60004EEF5FEF2D833E834F83588708C0898591
:107C70009A85AB85BC858D839E83AF83B887209121
:107C80004F033091500340915103509152032D877F
:107C90003E874F87588B29543B46414050402CF03B
:107CA00028E43BE641E050E00DC08D859E85AF8520
:107CB000B889885B9449AE4FBF4F4CF428EB34E948
:107CC0004EEF5FEF29833A834B835C8308C08D8539
:107CD0009E85AF85B88989839A83AB83BC83A09145
:107CE000EA07B091EB07BB8BAA8BFD01CF01AA2756
:107CF00097FDA095BA2FA0903F03B0904003C0908D
:107D00004103D0904203A80EB91ECA1EDB1EA092EA
:107D10003F03B0924003C0924103D0924203E090EF
:107D2000F107F090F2070091F3071091F407E80EC5
:107D3000F91E0A1F1B1FE092F107F092F207009351
:107D4000F3071093F407F0910203F98BFF2309F076
:107D500098C180910103882309F093C18091100696
:107D600086FF8FC180919C0790919D07AA2797FD60
:107D7000A095BA2FBC01CD0129813A814B815C814C
:107D80000E94457D9B01AC0197FF04C02150384FF4
:107D90004F4F5F4F6BE055954795379527956A95FF
:107DA000D1F780919D01682E772488249924CA01F7
:107DB000B901A40193010E94457DDC01CB018093B0
:107DC000900390939103A0939203B0939303B7FF12
:107DD00004C08150904FAF4FBF4F1C012D013CE0BC
:107DE00055944794379427943A95D1F7209290036D
:107DF0003092910340929203509293038091AB078B
:107E00009091AC07AA2797FDA095BA2FBC01CD0190
:107E10002D813E814F8158850E94457D97FF04C08A
:107E20006150784F8F4F9F4F2BE0959587957795B1
:107E300067952A95D1F7A40193010E94457DDC0145
:107E4000CB018093940390939503A0939603B093F2
:107E50009703B7FF04C08150904FAF4FBF4F9C01B5
:107E6000AD018CE055954795379527958A95D1F7C3
:107E70002093940330939503409396035093970374
:107E8000809190039091910390939407809393072E
:107E9000809194039091950390939807809397070E
:107EA000221933094409550920939403309395030B
:107EB0004093960350939703E20EF31E041F151F81
:107EC000E092F107F092F2070093F3071093F407A2
:107ED00080919C018823B1F457FF04C02F5F3F4F6E
:107EE0004F4F5F4F5595479537952795A21AB30A7F
:107EF000C40AD50AA0923F03B0924003C092410346
:107F0000D09242032A893B8979010027F7FC00952A
:107F1000102F8091940390919503A0919603B091B6
:107F20009703E80EF91E0A1F1B1FC801B70129811C
:107F30003A814B815C810E94457D9B01AC0197FF9A
:107F400004C02150384F4F4F5F4FBBE055954795C8
:107F500037952795BA95D1F780919E01A82EBB241D
:107F6000CC24DD24CA01B901A60195010E94457DFA
:107F7000DC01CB018093880390938903A0938A034B
:107F8000B0938B03B7FF04C08150904FAF4FBF4FEA
:107F90003C014D01ACE09594879477946794AA9541
:107FA000D1F7609288037092890380928A0390923D
:107FB0008B03C801B7012D813E814F8158850E94F6
:107FC000457D97FF04C06150784F8F4F9F4FFBE076
:107FD0009595879577956795FA95D1F7A6019501BF
:107FE0000E94457DDC01CB0180938C0390938D032F
:107FF000A0938E03B0938F03B7FF04C08150904FBE
:10800000AF4FBF4FAC01BD01ECE07595679557953B
:108010004795EA95D1F740938C0350938D03609375
:108020008E0370938F032A893B8937FF03C03095F5
:1080300021953F4F21343105E4F1D401C30197FE6E
:1080400007C0B095A095909581959F4FAF4FBF4FBA
:1080500081389105A105B10584F4DB01CA0177FFE0
:1080600007C0B095A095909581959F4FAF4FBF4F9A
:1080700081389105A105B105E4F081E080932703E3
:1080800018C01092980710929707109294071092B8
:10809000930710928C0310928D0310928E0310920E
:1080A0008F03109288031092890310928A03109212
:1080B0008B0380918C0390918D03A0918E03B091DE
:1080C0008F03BC01CD0124E630E040E050E00E9487
:1080D000B97DE0908803F0908903E21AF30AF092E8
:1080E000AA07E092A9078091880390918903A09143
:1080F0008A03B0918B03BC01CD0124E630E040E05F
:1081000050E00E94B97DDA01C90120918C033091C1
:108110008D038C01021B130B10939F0700939E0786
:108120008091950190919601A0919701B09198014D
:10813000BC01CD0128E631E040E050E00E94457DE1
:108140002091F1073091F2074091F3075091F40725
:10815000261737074807590764F0261B370B480BCB
:10816000590B2093F1073093F2074093F307509394
:10817000F4072091F1073091F2074091F3075091F5
:10818000F40757FF0CC0260F371F481F591F2093B5
:10819000F1073093F2074093F3075093F40760918F
:1081A0009C0770919D076E0D7F1D9B01442737FD35
:1081B0004095542F8091430390914403A09145032F
:1081C000B0914603820F931FA41FB51F80934303F2
:1081D00090934403A0934503B09346038091070313
:1081E00090910803681B790BCB01AA2797FDA095F6
:1081F000BA2F29853A854B855C85820F931FA41F72
:10820000B51F8093470390934803A0934903B0930D
:108210004A03C090B101D090B201E090B301F09058
:10822000B401C816D906EA06FB06C4F488EA91E64A
:10823000A0E0B0E08C199D09AE09BF098093470307
:1082400090934803A0934903B0934A038093430358
:1082500090934403A0934503B0934603222733270A
:10826000A9012C193D094E095F098091470390919E
:108270004803A0914903B0914A0382179307A407CA
:10828000B507B4F4D701C601885A9146A040B04062
:108290008093470390934803A0934903B0934A0304
:1082A0008093430390934403A0934503B093460304
:1082B0006091AB077091AC07600F711F9B01442761
:1082C00037FD4095542F80914B0390914C03A09122
:1082D0004D03B0914E03820F931FA41FB51F8093CF
:1082E0004B0390934C03A0934D03B0934E038091A6
:1082F000050390910603681B790BCB01AA2797FD14
:10830000A095BA2F2D853E854F855889820F931FE2
:10831000A41FB51F80934F0390935003A093510364
:10832000B0935203E090B501F090B6010091B7010F
:108330001091B801E816F9060A071B07C4F488EA89
:1083400091E6A0E0B0E08E199F09A00BB10B8093DD
:108350004F0390935003A0935103B0935203809323
:108360004B0390934C03A0934D03B0934E032227ED
:108370003327A9012E193F09400B510B80914F0360
:1083800090915003A0915103B0915203821793072B
:10839000A407B507B4F4D801C701885A9146A04094
:1083A000B04080934F0390935003A0935103B09338
:1083B000520380934B0390934C03A0934D03B093CF
:1083C0004E0380913F0390914003A0914103B091EF
:1083D00042038093530390935403A0935503B093A7
:1083E000560380914F0390915003A0915103B09197
:1083F000520380936F0390937003A0937103B09323
:1084000072038091470390914803A0914903B09172
:108410004A038093670390936803A0936903B09322
:108420006A0380914B0390914C03A0914D03B0914E
:108430004E0380936B0390936C03A0936D03B093F2
:108440006E038091430390914403A0914503B09142
:1084500046038093630390936403A0936503B093F2
:10846000660380911B0190911C0197FD079633E0F4
:10847000959587953A95E1F79093AC078093AB0774
:108480008091190190911A0197FD079623E0959527
:1084900087952A95E1F790939D0780939C0780919B
:1084A0004602909147020F9734F488E19CEF909335
:1084B000AC078093AB0780914602909147020797E3
:1084C00034F480E398EF9093AC078093AB0720914E
:1084D00002012A30A9F48091460290914702835FFD
:1084E000934034F088EE93E09093AC078093AB0711
:1084F00080914602909147028A5F9340DCF014C05D
:108500008091460290914702815D974034F088EE59
:1085100093E09093AC078093AB07809146029091D3
:108520004702805E974034F080ED97E09093AC076F
:108530008093AB0780914402909145020F9734F4E9
:1085400088E19CEF90939D0780939C078091440263
:1085500090914502079734F480E398EF90939D073C
:1085600080939C072A30A9F480914402909145029F
:10857000835F934034F088EE93E090939D0780935F
:108580009C0780914402909145028A5F9340DCF001
:1085900014C08091440290914502815D974034F06F
:1085A00088EE93E090939D0780939C07809144020E
:1085B00090914502805E974034F080ED97E0909373
:1085C0009D0780939C07E091A801EE2309F4B7C0B2
:1085D00040911B0150911C01809198039091990347
:1085E000481B590B50939F0340939E0320911B01FE
:1085F00030911C01280F391F37FF02C02F5F3F4FFA
:108600003595279530939903209398034138510568
:108610001CF080E890E005C040585F4F34F480E8DB
:108620009FEF90939F0380939E038E2F9927A09195
:108630009E03B0919F03A89FA001A99F500DB89FD2
:10864000500D112457FF02C0415F5F4F14E0559554
:1086500047951A95E1F78091AB079091AC07840F8D
:10866000951F9093AC078093AB07609119017091AF
:108670001A0180919A0390919B03681B790B709368
:108680009D0360939C034091190150911A01480F7A
:10869000591F57FF02C04F5F5F4F55954795509345
:1086A0009B0340939A03613871051CF080E890E0C9
:1086B00005C060587F4F34F480E89FEF90939D038E
:1086C00080939C032E2F332780919C0390919D03D0
:1086D000829FB001839F700D929F700D1124AB019A
:1086E00077FF02C0415F5F4FE4E055954795EA95FB
:1086F000E1F780919C0790919D07840F951F9093BF
:108700009D0780939C07A29FC001A39F900DB29FDD
:10871000900D11249C0180911B0190911C01820FEE
:10872000931F90931C0180931B01809119019091DC
:108730001A01860F971F90931A01809319010091D7
:10874000AE071091AF078091930790919407101690
:1087500011065CF59C0197FF04C022273327281BD4
:10876000390BC901AA2797FDA095BA2F20919C012A
:10877000332744275527BC01CD010E94457D9B012D
:10878000AC0197FF04C0215C3F4F4F4F5F4F76E035
:1087900055954795379527957A95D1F78091A907F3
:1087A0009091AA07820F931F27C097FF03C090954F
:1087B00081959F4FAA2797FDA095BA2F20919C01E4
:1087C000332744275527BC01CD010E94457D9B01DD
:1087D000AC0197FF04C0215C3F4F4F4F5F4F66E0F5
:1087E00055954795379527956A95D1F78091A907B3
:1087F0009091AA07821B930B9093AA078093A907D5
:10880000E090B607F090B70780919707909198078E
:108810001E141F045CF59C0197FF04C02227332718
:10882000281B390BC901AA2797FDA095BA2F2091C3
:108830009C01332744275527BC01CD010E94457D6B
:108840009B01AC0197FF04C0215C3F4F4F4F5F4F2E
:1088500096E055954795379527959A95D1F780914C
:108860009E0790919F07820F931F27C097FF03C019
:10887000909581959F4FAA2797FDA095BA2F20919B
:108880009C01332744275527BC01CD010E94457D1B
:108890009B01AC0197FF04C0215C3F4F4F4F5F4FDE
:1088A00086E055954795379527958A95D1F780911C
:1088B0009E0790919F07821B930B90939F07809335
:1088C0009E078091100687FF44C09989992309F07B
:1088D00040C0809101038823E1F5A1E0EA16A1E000
:1088E000FA064CF08091AB079091AC078E0D9F1D5E
:1088F000805091400DC0B0E0EB16BFEFFB0664F472
:108900008091AB079091AC078E0D9F1D80509F4FBB
:108910009093AC078093AB07E1E001301E074CF069
:1089200080919C0790919D07800F911F80509140EE
:108930000CC0FFEF00301F0764F480919C079091FA
:108940009D07800F911F80509F4F90939D078093AC
:108950009C07ACE1B3E068E076E057E0FB01819171
:10896000BF01E82FFF27EE0FFF1FE55DF84F0190D5
:10897000F081E02DE259FF4FEF3FF10521F01CF0AF
:10898000EFEFF0E004C0F7FF02C0E0E0F0E04C9150
:10899000242F3327E217F307B1F0CF01821B930B8B
:1089A00097FD079613E0959587951A95E1F7242F83
:1089B000280F2C93822F9927E817F90714F42150D8
:1089C00001C02F5F2C935150119657FFC7CFE2E1A2
:1089D000CD5E0C94F07D80911203882301F5809187
:1089E000E7028C7F8093E702A5E4B4E0EAECF6E0CE
:1089F0009BE080910202882309F48C938D918183FE
:108A000012829150389697FFF4CF8091020288230A
:108A100059F08091020281508093020205C080913A
:108A2000E70281608093E70210926E02109270025A
:108A300080916B028E7F80936B0285EA8093BC00ED
:108A4000089580911206883F38F0EFEFF0E0E81BC0
:108A5000F109E45EFC4F80818093AE018091AE010C
:108A6000882329F0843618F084E68093AE01809143
:108A70001406883F38F0EFEFF0E0E81BF109E45E00
:108A8000FC4F80818093AC018091AC01882329F058
:108A9000843618F084E68093AC0180912106883FEB
:108AA00038F0EFEFF0E0E81BF109E45EFC4F808165
:108AB0008093A7018091A7018B3010F48AE002C057
:108AC0008F3F11F48093A70180914C06883F38F0C6
:108AD000EFEFF0E0E81BF109E45EFC4F808180934A
:108AE000C2078091C207823010F481E002C08F3F3C
:108AF00011F48093C20780914E06883F38F0EFEF63
:108B0000F0E0E81BF109E45EFC4F80818093E80708
:108B10008091E807823010F481E002C08F3F11F4A9
:108B20008093E80780913906883F38F0EFEFF0E056
:108B3000E81BF109E45EFC4F80818093BF078091C0
:108B40003A06883F38F0EFEFF0E0E81BF109E45E09
:108B5000FC4F80818093990780913B06883F38F0D5
:108B6000EFEFF0E0E81BF109E45EFC4F80818093B9
:108B7000C70790911306983F18F49093AD0109C070
:108B8000EFEFF0E0E91BF109E45EFC4F8081809398
:108B9000AD01983F18F49093AD0109C0EFEFF0E0FC
:108BA000E91BF109E45EFC4F80818093AD01809167
:108BB0001606883F38F0EFEFF0E0E81BF109E45EBD
:108BC000FC4F80818093AB0180911806883F38F07C
:108BD000EFEFF0E0E81BF109E45EFC4F8081809349
:108BE000A90180912006883F38F0EFEFF0E0E81B04
:108BF000F109E45EFC4F80818093AA0180912206F6
:108C0000883F38F0EFEFF0E0E81BF109E45EFC4F3D
:108C100080818093A60180912306883F38F0EFEF92
:108C2000F0E0E81BF109E45EFC4F80818093A8012D
:108C300080912406883F38F0EFEFF0E0E81BF1095F
:108C4000E45EFC4F80818093A50180912506883FDA
:108C500038F0EFEFF0E0E81BF109E45EFC4F8081B3
:108C60008093A40180912B06883F38F0EFEFF0E06D
:108C7000E81BF109E45EFC4F80818093A2018091A2
:108C80002C06883F38F0EFEFF0E0E81BF109E45ED6
:108C9000FC4F80818093FC0280912D06883F38F044
:108CA000EFEFF0E0E81BF109E45EFC4F8081809378
:108CB000FB0280912E06883F38F0EFEFF0E0E81BD2
:108CC000F109E45EFC4F80818093FA0280912F06C7
:108CD000883F38F0EFEFF0E0E81BF109E45EFC4F6D
:108CE00080818093F90280914706883F38F0EFEF4A
:108CF000F0E0E81BF109E45EFC4F80818093F8020C
:108D000080914806883F38F0EFEFF0E0E81BF1096A
:108D1000E45EFC4F80818093F70280914906883F92
:108D200038F0EFEFF0E0E81BF109E45EFC4F8081E2
:108D30008093F60280914A06883F38F0EFEFF0E02A
:108D4000E81BF109E45EFC4F80818093F50280917D
:108D50003006883F38F0EFEFF0E0E81BF109E45E01
:108D6000FC4F80818093A10180913406883F38F0C8
:108D7000EFEFF0E0E81BF109E45EFC4F80818093A7
:108D8000A00180913C06883F38F0EFEFF0E0E81B4F
:108D9000F109E45EFC4F808180939F0180913F0642
:108DA000883F38F0EFEFF0E0E81BF109E45EFC4F9C
:108DB000808180939E0180914006883F38F0EFEFDC
:108DC000F0E0E81BF109E45EFC4F808180939D0197
:108DD00080914106883F38F0EFEFF0E0E81BF109A1
:108DE000E45EFC4F808180939C0180914606883F21
:108DF00038F0EFEFF0E0E81BF109E45EFC4F808112
:108E000080939B0180916106883F38F0EFEFF0E09E
:108E1000E81BF109E45EFC4F80818093F8078091A4
:108E2000A201282F33272F5F3F4F8CE398E2B9012F
:108E30000E94847D7093B0016093AF0180911E0603
:108E40008093E90780911D068093B0079091630697
:108E5000933320F181E08093F402983F58F0EFEFD4
:108E6000F0E0E91BF109E45EFC4F8081823310F4ED
:108E70001092F402809136089091370897FF08C04D
:108E80008091F402882321F080914004806803C01F
:108E9000809140048F778093400402C01092F402C6
:108EA000809136089091370897FF1DC0809112037A
:108EB0008823C9F08091F4028823A9F080910801E9
:108EC000909109018F5F9F4F71F488E99AE3909325
:108ED00022028093210280E094EA9093090180931A
:108EE00008011092F4028091F402882339F08091F5
:108EF0009E01823D18F4825E80939E010895A5E351
:108F0000B0E0E5E8F7E40C94D47D0E94F33C3091A6
:108F100002013C3010F4299A01C02998E090130313
:108F2000F0901403F9A2E8A28091B00799270A965D
:108F3000E816F90614F499A388A380911B038436DC
:108F400008F05CC08091B4039091B503009731F0B4
:108F500001979093B5038093B40307C01092120356
:108F60008091E7028F7E8093E7023A3011F034312E
:108F700010F0289A01C028988091E8029091E902A7
:108F8000895E9340C0F180912806282F332739A3AA
:108F900028A38091E70280618093E7028091040614
:108FA000A82FBB27AA0FBB1FFD01E15AF84F118262
:108FB000108280910506282F3327220F331FC90105
:108FC000815A984FFC0111821082A55DB84F11960D
:108FD0001C921E92255D384FD90111961C921E924B
:108FE00080910706E82FFF27EE0FFF1FE55DF84F82
:108FF00011821082AAC210921203A7C280911B0391
:109000008D3808F4A2C28091E7028F7E8093E70238
:109010009091290682E3989FC00111249093B50393
:109020008093B403E8A1F9A1B9978CF08091120361
:10903000882369F08091E8029091E902FFEF8F3F69
:109040009F0729F001969093E9028093E8028091AE
:10905000E8029091E9028F3F910509F038F51092EE
:109060003703109238031092390310923A0310928A
:10907000330310923403109235031092360310928A
:10908000A0031092A1031092A2031092A3031092C6
:109090003F031092400310924103109242038A3F13
:1090A000910549F481E08093BA0305C08091E702FD
:1090B00082608093E70280910606E82FFF27EE0F7B
:1090C000FF1FE55DF84F80819181813591050CF49A
:1090D00041C120911203222309F03CC1809107066F
:1090E000E82FFF27EE0FFF1FE55DF84F808191818C
:1090F0008C3491050CF406C18091B6038F5F809388
:10910000B603893C08F426C13C3010F4299801C00C
:10911000299A109212031092B6031092E90210924B
:10912000E80230910406E32FFF27EE0FFF1FE55DF5
:10913000F84F8081918187349105B4F480910506C0
:10914000E82FFF27EE0FFF1FE55DF84F808191812B
:109150000190F081E02DF7FF03C0F095E195FF4FFE
:10916000E734F1050CF478C041E020910506A22F08
:10917000BB27AA0FBB1FA55DB84F8D919C9111977E
:109180008734910544F0E32FFF27EE0FFF1FE55DC5
:10919000F84F808191818D919C918734910574F075
:1091A00080910406E82FFF27EE0FFF1FE55DF84FC3
:1091B00080819181873491050CF042E0E22FFF27F6
:1091C000EE0FFF1FE55DF84F808191818634910598
:1091D00074F480910406E82FFF27EE0FFF1FE55D72
:1091E000F84F80819181873491050CF043E0E22FA4
:1091F000FF27EE0FFF1FE55DF84F808191818A5BAD
:109200009F4F74F480910406E82FFF27EE0FFF1F95
:10921000E55DF84F80819181873491050CF044E041
:10922000E22FFF27EE0FFF1FE55DF84F8081918150
:109230008A5B9F4F74F480910406E82FFF27EE0F9E
:10924000FF1FE55DF84F80819181863491050CF414
:1092500045E0842F0E944D2F80910506E82FFF27BF
:10926000EE0FFF1FE55DF84F808191810190F08145
:10927000E02DF7FF03C0F095E195FF4F7E97BCF41A
:1092800080910406E82FFF27EE0FFF1FE55DF84FE2
:10929000808191818A5B9F4F54F481E080935B04CD
:1092A00088EE93E0909322028093210253C00E94A3
:1092B00047300E94FA2E80E00E940D0880912A0615
:1092C0000E94F8798091100680FF10C080911301F0
:1092D00090911401875B934038F480911301909131
:1092E00014018E5E924010F40E947A1B10921F02AD
:1092F00080E00E94453A81E08093B90380931F0289
:10930000579A1FC080819181855B9F4F0CF580919A
:10931000B6038F5F8093B603893CE0F03C3010F4D5
:10932000299801C0299A109212031092B603109244
:10933000E9021092E80281E00E94453A81E08093C0
:10934000B9030E94473068E770E00E94833902C089
:109350002093B60380910606E82FFF27EE0FFF1F2C
:10936000E55DF84F808191818B5A9F4F0CF0EDC0E5
:1093700020911203E0910706222309F0CAC0FF27BB
:10938000EE0FFF1FE55DF84F80819181855B9F4F58
:109390000CF0BCC08091B7038F5F8093B703893C0A
:1093A00008F4D3C02093B70380914004882309F0C8
:1093B000A6C08091B903882309F4A1C081E090E0A0
:1093C0009093E9028093E80281E080931203109267
:1093D000A0031092A1031092A2031092A303109273
:1093E0003F031092400310924103109242031092E7
:1093F0003B0310923C0310923D0310923E03809178
:109400001F06E82EFF24002711278091E507909181
:10941000E6079C01442737FD4095542FC801B7014A
:109420000E94457DDC01CB0180934F039093500354
:10943000A0935103B09352038091F5079091F607E2
:109440009C01442737FD4095542FC801B7010E9465
:10945000457DDC01CB018093470390934803A093A3
:109460004903B0934A0380916F0390917003A091D8
:109470007103B091720380934B0390934C03A093BC
:109480004D03B0934E038091670390916803A091C0
:109490006903B0916A038093430390934403A093BC
:1094A0004503B0934603109237031092380310928D
:1094B000390310923A03109233031092340310923E
:1094C0003503109236038091E70288608093E702AB
:1094D000909162068FE0989F9001112480912D0356
:1094E00090912E03820F931F68E671E00E94847DA5
:1094F00097FD0196959587958093730326C08CED13
:1095000095E090932202809321021FC02093B7031D
:109510001CC0FF27EE0FFF1FE55DF84F8081918192
:109520008C34910584F08091B8038F5F8093B803E9
:10953000893C58F0109212031092B8031092E9027D
:109540001092E80202C01092B803809193018150FA
:1095500080939301809193018F3F21F08091E702E6
:1095600084FF82C30E9421458091C3039091C4036C
:109570009C01220F331F280F391FA0900406AA2D2B
:10958000BB27AA0FBB1FFD01E55DF84F90901A069F
:10959000492D552780819181849FF001859FF00D91
:1095A000949FF00D11242E0F3F1F37FF02C02D5F37
:1095B0003F4FB9017595679575956795A15AB84F55
:1095C00080911B06082F11278D919C91809F70011F
:1095D000819FF00C909FF00C11246E0D7F1D7093F5
:1095E000C4036093C3038091C5039091C6039C019B
:1095F000220F331F280F391FB0900506AB2DBB2754
:10960000AA0FBB1FFD01E55DF84F80819181849F0A
:10961000F001859FF00D949FF00D11242E0F3F1F38
:1096200037FF02C02D5F3F4FA901559547955595CE
:109630004795A15AB84F8D919C91809F7001819F51
:10964000F00C909FF00C11244E0D5F1D5093C6033B
:109650004093C5039E012F5F3F4F8FE1E0ECF1E0A7
:10966000D90101900D928A95E1F78091F402882347
:1096700009F448C0CB0177FD0396DC01B595A795A9
:10968000B595A795CA0157FD0396FC01F595E79599
:10969000F595E7958091E901682F772767FD70952B
:1096A0006A9F90016B9F300D7A9F300D112480913D
:1096B000FC03482F552747FD50954E9FC0014F9FF3
:1096C000900D5E9F900D1124280F391F37FF02C0A7
:1096D000295F3F4F03E0359527950A95E1F73093D1
:1096E0001A03209319036E9F90016F9F300D7E9F88
:1096F000300D11244A9FC0014B9F900D5A9F900D31
:10970000112444C080916206082F1127DE01A00FAA
:10971000B11FFD0197819093E901020F131FD8013A
:109720008C918093FC03A92FBB27A7FDB095A69F22
:109730009001A79F300DB69F300D1124E82FFF2711
:10974000E7FDF095E49FC001E59F900DF49F900D1B
:109750001124280F391F37FF02C0295F3F4F13E044
:10976000359527951A95E1F730931A03209319033D
:10977000A49F9001A59F300DB49F300D1124E69F4A
:10978000C001E79F900DF69F900D1124281B390B07
:1097900037FF02C0295F3F4FF3E035952795FA95D3
:1097A000E1F7309318032093170380910706E82F01
:1097B000FF27EE0FFF1FE55DF84F808191819095A7
:1097C00081959F4F909316038093150383309105E5
:1097D00014F0029705C0BFEF8E3F9B0734F402964A
:1097E000909316038093150304C0109216031092F1
:1097F00015038091F8039091F9032091F4033091BF
:10980000F503820F931FC0901903D0901A03C81A52
:10981000D90AD0921A03C09219038091F60390914D
:10982000F7032091F2033091F303820F931F00910D
:10983000170310911803081B190B109318030093BA
:10984000170380910606E82FFF27EE0FFF1FE55D47
:10985000F84FE080F180E8E7F0E0EE0EFF1EF092B6
:109860001403E09213038091A7019927AA2797FD7B
:10987000A095BA2FBC01CD010E94B97CDC01CB01BF
:1098800020E030E040E251E4BC01CD010E94277CA1
:10989000DC01CB01BC01CD010E948B7CDC01CB0142
:1098A0008093EF078091A6018093C8078091A5015E
:1098B0009927AA2797FDA095BA2FBC01CD010E9438
:1098C000B97CDC01CB0120E030E040E251E4BC0196
:1098D000CD010E94277CDC01CB01BC01CD010E949F
:1098E0008B7CDC01CB018093A3078091A401809342
:1098F000B8078091670480FF59C08091F8078138CC
:1099000008F454C080916004992787FD9095292D13
:109910003327829FA001839F500D929F500D1124E9
:10992000C40ED51ED0921A03C0921903809161040F
:10993000992787FD9095829FB001839F700D929F1C
:10994000700D1124060F171F1093180300931703AF
:1099500080916204282F332727FD309580911503CD
:1099600090911603820F931F909316038093150313
:1099700080916404282F332727FD309580911506A8
:109980009927289FD001299FB00D389FB00D112431
:10999000B0939A01A09399018091630499278E1541
:1099A0009F0524F490931403809313038091130371
:1099B0009091140397FF04C01092140310921303A4
:1099C0008091100682FF02C01092C80740911903CF
:1099D00050911A03CA0157FD03969C0135952795AE
:1099E0003595279537FF03C0309521953F4F8091DE
:1099F000EC029091ED0282179307B4F4CA0157FF6D
:109A000003C0909581959F4F97FD039695958795F7
:109A1000959587959093ED028093EC02853691059C
:109A200044F084E690E001C001979093ED028093AA
:109A3000EC024091170350911803CA0157FD039699
:109A40009C01359527953595279537FF03C03095AF
:109A500021953F4F8091EA029091EB028217930784
:109A6000B4F4CA0157FF03C0909581959F4F97FDAD
:109A7000039695958795959587959093EB0280939E
:109A8000EA028536910544F084E690E001C0019732
:109A90009093EB028093EA028091E70284FF08C072
:109AA0001092ED021092EC021092EB021092EA0278
:109AB000EB2DFF27EE0FFF1FE55DF84F40913D06B0
:109AC000242F3327808191812817390744F480910E
:109AD000640682FF04C081E08093000313C0EB2D75
:109AE000FF27EE0FFF1FE55DF84F842F9927209188
:109AF0003E06821B9109208131812817390714F411
:109B00001092000340910506E42FFF27EE0FFF1F80
:109B1000E55DF84F50913D06852F99272227332781
:109B2000281B390B808191818217930744F480911F
:109B3000640683FF04C081E08093FF0216C0809119
:109B4000FF02882391F0E42FFF27EE0FFF1FE55D52
:109B5000F84F80913E069927851B9109208131811C
:109B60008217930714F41092FF02EA2DFF27EE0FDD
:109B7000FF1FE55DF84F40913D06242F332780817C
:109B800091812817390744F48091640680FF04C04E
:109B900081E08093FD0217C08091FD02882399F037
:109BA000EA2DFF27EE0FFF1FE55DF84F842F992761
:109BB00020913E06821B91092081318128173907A7
:109BC00014F41092FD0240910406E42FFF27EE0FDB
:109BD000FF1FE55DF84F50913D06852F99272227FD
:109BE0003327281B390B808191818217930744F416
:109BF0008091640681FF04C081E08093FE0216C05C
:109C00008091FE02882391F0E42FFF27EE0FFF1FC3
:109C1000E55DF84F80913E069927851B91092081CB
:109C200031818217930714F41092FE028091000391
:109C3000882319F48091FF02811181E08093010350
:109C40008091FD02882321F48091FE02882351F047
:109C500081E080930203109201031092000310929E
:109C6000FF0202C08093020380910103882321F444
:109C700080910203882369F080913C069927E8A12E
:109C8000F9A18E179F0714F499A388A381E080930C
:109C900027038091E70284FF1AC0109216031092E6
:109CA000150310921A0310921903109218031092C0
:109CB00017039AE59093EF0788E78093C80790937E
:109CC000A3078093B80710920103109202038091BA
:109CD000BB079091BC07A091BD07B091BE07209132
:109CE0006F03309170034091710350917203820FA2
:109CF000931FA41FB51F8093BB079093BC07A0932D
:109D0000BD07B093BE078091C3079091C407A0918F
:109D1000C507B091C6072090670330906803409054
:109D2000690350906A03820D931DA41DB51D809395
:109D3000C3079093C407A093C507B093C60780914B
:109D4000B2079091B307A091B407B091B507E09026
:109D50006B03F0906C0300916D0310916E03EAA207
:109D6000FBA20CA31DA38E0D9F1DA01FB11F8093EE
:109D7000B2079093B307A093B407B093B50780914F
:109D8000A4079091A507A091A607B091A707E0901E
:109D90006303F09064030091650310916603EEA2E3
:109DA000FFA208A719A78E0D9F1DA01FB11F8093AA
:109DB000A4079093A507A093A607B093A707F090D8
:109DC0000203FAA6FF2029F480910103882309F4F5
:109DD00060C010925F0310926003109261031092B2
:109DE000620310925B0310925C0310925D03109269
:109DF0005E031092BB071092BC071092BD07109231
:109E0000BE071092C3071092C4071092C5071092A4
:109E1000C6071092B2071092B3071092B4071092BF
:109E2000B5071092A4071092A5071092A6071092EA
:109E3000A70780914F0390915003A0915103B091D7
:109E4000520380934B0390934C03A0934D03B09324
:109E50004E038091470390914803A0914903B0912C
:109E60004A038093430390934403A0934503B09324
:109E7000460310923302109232021092060310929F
:109E8000050310920803109207030AA5002309F0A6
:109E9000F2C180910103882309F0EDC18091F5059D
:109EA0009091F605815092402CF480911203882302
:109EB00009F4E1C190906308A0901F066091E50746
:109EC0007091E6077BAB6AAB8091F5079091F6073E
:109ED0009DAB8CAB9FEF991609F4D9C0BB24CC2461
:109EE000DD24CA01B901A60195010E94B97D79015D
:109EF0008A01EAA9FBA9CF01AA2797FDA095BA2F4D
:109F0000E81AF90A0A0B1B0BC201B101A60195015F
:109F10000E94B97D59016A012CA93DA9C901AA274E
:109F200097FDA095BA2FA81AB90ACA0ADB0A292CEC
:109F3000332427FC3094432C532CC801B701A201D1
:109F400091010E94457D97FF04C061507E4F8F4F65
:109F50009F4F3B014C0109E0959487947794679457
:109F60000A95D1F7C601B501A20191010E94457D74
:109F700097FF04C061507E4F8F4F9F4F5B016C0174
:109F800019E0D594C794B794A7941A95D1F7809106
:109F9000EC029091ED02813491053CF48091EA024B
:109FA0009091EB0281349105D4F0D401C30197FE66
:109FB00003C00196A11DB11D3C014D0195948794EC
:109FC00077946794D601C501D7FE03C00196A11D01
:109FD000B11D5C016D01D594C794B794A79480918D
:109FE0000706E82FFF27EE0FFF1FE55DF84F808182
:109FF00091810190F081E02DF7FF03C0F095E1958C
:10A00000FF4F7A97A4F0C401B30123E030E040E0B1
:10A0100050E00E94B97D39014A01C601B50123E033
:10A0200030E040E050E00E94B97D59016A01809122
:10A030006508282F332727FD3095432F532F2615EA
:10A0400037054805590514F439014A01992787FD58
:10A050009095909581959F4FAA2797FDA095BA2F2F
:10A06000681679068A069B0614F43C014D012A15F0
:10A070003B054C055D0514F459016A01A816B906A3
:10A08000CA06DB060CF0CFC05C016D01CCC0EA2C27
:10A09000FF2400271127CA01B901A80197010E94D6
:10A0A000B97D39014A014AA95BA9CA01AA2797FDCE
:10A0B000A095BA2F681A790A8A0A9B0AC201B101CF
:10A0C000A80197010E94B97D59016A016CA97DA977
:10A0D000CB01AA2797FDA095BA2FA81AB90ACA0AD8
:10A0E000DB0AD401C30197FE03C00F96A11DB11D69
:10A0F0003C014D01F4E09594879477946794FA9528
:10A10000D1F7D601C501D7FE03C00F96A11DB11D21
:10A110005C016D01E4E0D594C794B794A794EA95E7
:10A12000D1F78091EC029091ED02813491053CF4DD
:10A130008091EA029091EB0281349105A4F0C40170
:10A14000B30123E030E040E050E00E94B97D3901E6
:10A150004A01C601B50123E030E040E050E00E9432
:10A16000B97D59016A0180910706E82FFF27EE0F9C
:10A17000FF1FE55DF84F808191810190F081E02D16
:10A18000F7FF03C0F095E195FF4F7A97A4F0C40163
:10A19000B30123E030E040E050E00E94B97D390196
:10A1A0004A01C601B50123E030E040E050E00E94E2
:10A1B000B97D59016A0171E2671671048104910445
:10A1C0002CF070E2672E712C812C912C80EE681699
:10A1D0008FEF78068FEF88068FEF980644F460EED5
:10A1E000662E6FEF762E6FEF862E6FEF962E91E232
:10A1F000A916B104C104D1042CF050E2A52EB12C53
:10A20000C12CD12CA0EEAA16AFEFBA06AFEFCA064A
:10A21000AFEFDA0644F440EEA42E4FEFB42E4FEF2A
:10A22000C42E4FEFD42E80914F0390915003A091F4
:10A230005103B091520386199709A809B90980936F
:10A240004F0390935003A0935103B0935203809116
:10A25000470390914803A0914903B0914A038A199A
:10A260009B09AC09BD098093470390934803A093D1
:10A270004903B0934A0380913202909133028F3F99
:10A28000910509F008F4C4C5BAA5BB2309F04EC571
:10A2900080910103882309F049C580912703882311
:10A2A00009F044C5E0914506EBA7EE2309F43EC54D
:10A2B0008091BB079091BC07A091BD07B091BE07EC
:10A2C000B7FF04C081509F4FAF4FBF4FE92EFA2E0A
:10A2D0000B2F112707FD1A95E092BB07F092BC07E0
:10A2E0000093BD071093BE078091C3079091C407E8
:10A2F000A091C507B091C607B7FF04C081509F4F1A
:10A30000AF4FBF4F892F9A2FAB2FBB27A7FDBA9511
:10A310008CA79DA7AEA7BFA78093C3079093C40740
:10A32000A093C507B093C60780911F06A82EBB2433
:10A33000CC24DD2420915F033091600340916103C0
:10A3400050916203C601B5010E94457D97FF04C08C
:10A3500061507F4F8F4F9F4F672E782E892E992403
:10A3600087FC9A9460925F0370926003809261030D
:10A370009092620320915B0330915C0340915D03F6
:10A3800050915E03C601B5010E94457D97FF04C050
:10A3900061507F4F8F4F9F4F272E382E492E5524C7
:10A3A00047FC5A9420925B0330925C0340925D0319
:10A3B00050925E038091570390915803A0915903E6
:10A3C000B0915A03B7FF04C081509F4FAF4FBF4FAA
:10A3D000892F9A2FAB2FBB27A7FDBA9580935703E0
:10A3E00090935803A0935903B0935A03D801C7011F
:10A3F00086199709A809B9098093AC039093AD0316
:10A40000A093AE03B093AF0320914406E22EFF2445
:10A4100000271127BC01CD01A80197010E94B97D39
:10A4200059016A012093BB033093BC034093BD03E1
:10A430005093BE038CA59DA5AEA5BFA58219930917
:10A44000A409B5098093B0039093B103A093B2031C
:10A45000B093B303BC01CD01A80197010E94B97D5F
:10A460002093BF033093C0034093C1035093C203B2
:10A47000D601C501D7FE04C081509F4FAF4FBF4FDB
:10A48000892F9A2FAB2FBB27A7FDBA959093060370
:10A490008093050357FF04C021503F4F4F4F5F4F3C
:10A4A000BB2757FDBA95A52F942F832F90930803B0
:10A4B000809307038091EC029091ED028134910525
:10A4C000DCF48091EA029091EB0281349105A4F4CE
:10A4D00080910706E82FFF27EE0FFF1FE55DF84F7D
:10A4E000808191810190F081E02DF7FF03C0F0950C
:10A4F000E195FF4F7A97E4F0809163088F3FC1F4B4
:10A50000809105039091060397FD01969595879597
:10A5100090930603809305038091070390910803AD
:10A5200097FD01969595879590930803809307036F
:10A530008091B2079091B307A091B407B091B5078D
:10A54000B7FF04C081509F4FAF4FBF4F892F9A2F45
:10A55000AB2FBB27A7FDBA958093B2079093B307A3
:10A56000A093B407B093B5078091A4079091A50775
:10A57000A091A607B091A707B7FF04C081509F4FD5
:10A58000AF4FBF4F892F9A2FAB2FBB27A7FDBA958F
:10A590008093A4079093A507A093A607B093A7075D
:10A5A00080916F0390917003A0917103B091720339
:10A5B0002AA13BA14CA15DA1281B390B4A0B5B0BC7
:10A5C0002093A4033093A5034093A6035093A703BD
:10A5D0008091670390916803A0916903B0916A0329
:10A5E000EEA0FFA008A519A5E81AF90A0A0B1B0B93
:10A5F000E092A803F092A9030093AA031093AB037F
:10A600002093AC033093AD034093AE035093AF035C
:10A61000E092B003F092B1030093B2031093B3033E
:10A6200080914B0390914C03A0914D03B0914E0348
:10A63000821B930BA40BB50B80934B0390934C039D
:10A64000A0934D03B0934E03809143039091440334
:10A65000A0914503B09146038E199F09A00BB10B41
:10A660008093430390934403A0934503B093460320
:10A67000FBA5FF23E1F0209125033091260321382B
:10A6800031054CF080918003909181030196909365
:10A6900081038093800320583F4F4CF480918003C6
:10A6A000909181030197909381038093800310928E
:10A6B00026031092250381E090E09093C8038093D5
:10A6C000C703A090AC03B090AD03C090AE03D09090
:10A6D000AF03D601C501D7FE07C088279927DC0143
:10A6E0008A199B09AC09BD0981509240A040B04035
:10A6F00034F084E090E09093C8038093C703809186
:10A70000CD039091CE03A091CF03B091D0032091BF
:10A71000BB073091BC074091BD075091BE07821B1B
:10A72000930BA40BB50B815E914BAF4FBF4F8F5373
:10A730009C49A040B04028F08091640889310CF415
:10A74000FFC031E0A31630E1B30630E0C30630E0CD
:10A75000D3060CF473C08091C903882309F46AC03E
:10A76000D601C501D7FE07C088279927DC018A19C1
:10A770009B09AC09BD099C01AD01B7FF04C0215084
:10A780003E4F4F4F5F4FF9E05595479537952795C9
:10A79000FA95D1F78091C7039091C803820F931F58
:10A7A0009093C8038093C703D601C501D7FE03C0A9
:10A7B0000796A11DB11DE3E0B595A79597958795DF
:10A7C000EA95D1F78093BB039093BC03A093BD039C
:10A7D000B093BE0389589341A040B04064F088E82C
:10A7E00093E1A0E0B0E08093BB039093BC03A093FF
:10A7F000BD03B093BE032091BB033091BC034091D5
:10A80000BD035091BE0357FF04C021503F4F4F4F2F
:10A810005F4F232F342F452F552747FD5A958091A1
:10A82000050390910603820F931F90930603809374
:10A83000050306C081E08093C90302C01092C903DA
:10A8400050E0A51650EFB5065FEFC5065FEFD506E1
:10A850000CF073C08091CA03882309F46AC0D60142
:10A86000C501D7FE07C088279927DC018A199B09F3
:10A87000AC09BD099C01AD01B7FF04C021503E4F9A
:10A880004F4F5F4F69E055954795379527956A95E6
:10A89000D1F78091C7039091C803820F931F9093C3
:10A8A000C8038093C703D601C501D7FE03C007962E
:10A8B000A11DB11D23E0B595A795979587952A957C
:10A8C000D1F78093BB039093BC03A093BD03B093D7
:10A8D000BE0388579C4EAF4FBF4F64F488E79CEE91
:10A8E000AFEFBFEF8093BB039093BC03A093BD0376
:10A8F000B093BE032091BB033091BC034091BD03D4
:10A900005091BE0357FF04C021503F4F4F4F5F4F40
:10A91000232F342F452F552747FD5A958091050346
:10A9200090910603820F931F909306038093050373
:10A9300011C081E08093CA030DC01092CA030AC0FF
:10A940001092C8031092C70388EE93E09093BA0167
:10A950008093B9017BA5272F33278091C70390915E
:10A96000C8032817390724F43093C8032093C7037A
:10A97000E0916408EE2379F02E2F332727FD3095E0
:10A980008091C7039091C8032817390724F43093A6
:10A99000C8032093C7034091AC035091AD0360916D
:10A9A000AE037091AF03413851056105710574F034
:10A9B00080918403909185032091C7033091C8034F
:10A9C000820F931F909385038093840340585F4FB9
:10A9D0006F4F7F4F74F48091840390918503209191
:10A9E000C7033091C803821B930B90938503809318
:10A9F000840381E090E09093C8038093C703A09004
:10AA0000B003B090B103C090B203D090B303D601AD
:10AA1000C501D7FE07C088279927DC018A199B0941
:10AA2000AC09BD0981509240A040B04034F084E0B0
:10AA300090E09093C8038093C7038091D1039091D5
:10AA4000D203A091D303B091D4032091C3073091D6
:10AA5000C4074091C5075091C607821B930BA40BF6
:10AA6000B50B815E914BAF4FBF4F8F539C49A040B8
:10AA7000B04018F0E9310CF4FFC011E0A11610E16C
:10AA8000B10610E0C10610E0D1060CF473C080914D
:10AA9000CB03882309F46AC0D601C501D7FE07C0DD
:10AAA00088279927DC018A199B09AC09BD099C01FB
:10AAB000AD01B7FF04C021503E4F4F4F5F4F09E03B
:10AAC00055954795379527950A95D1F78091C703F6
:10AAD0009091C803820F931F9093C8038093C7037C
:10AAE000D601C501D7FE03C00796A11DB11D13E015
:10AAF000B595A795979587951A95D1F78093BF033C
:10AB00009093C003A093C103B093C20389589341AB
:10AB1000A040B04064F088E893E1A0E0B0E080930A
:10AB2000BF039093C003A093C103B093C2032091CD
:10AB3000BF033091C0034091C1035091C20357FF3E
:10AB400004C021503F4F4F4F5F4F232F342F452FCD
:10AB5000552747FD5A958091070390910803820F6E
:10AB6000931F909308038093070306C081E08093AE
:10AB7000CB0302C01092CB0330E0A31630EFB30634
:10AB80003FEFC3063FEFD3060CF073C08091CC03B8
:10AB9000882309F46AC0D601C501D7FE07C08827FB
:10ABA0009927DC018A199B09AC09BD099C01AD01FB
:10ABB000B7FF04C021503E4F4F4F5F4FE9E055951E
:10ABC000479537952795EA95D1F78091C7039091DE
:10ABD000C803820F931F9093C8038093C703D601C5
:10ABE000C501D7FE03C00796A11DB11D73E0B59541
:10ABF000A795979587957A95D1F78093BF03909302
:10AC0000C003A093C103B093C20388579C4EAF4FBB
:10AC1000BF4F64F488E79CEEAFEFBFEF8093BF03B4
:10AC20009093C003A093C103B093C2032091BF03CC
:10AC30003091C0034091C1035091C20357FF04C03B
:10AC400021503F4F4F4F5F4F232F342F452F552714
:10AC500047FD5A958091070390910803820F931F37
:10AC6000909308038093070311C081E08093CC0385
:10AC70000DC01092CC030AC01092C8031092C703F3
:10AC800088EE93E09093BA018093B9015BA5252FDC
:10AC900033278091C7039091C8032817390724F4FC
:10ACA0003093C8032093C70380916408882379F008
:10ACB000282F332727FD30958091C7039091C80333
:10ACC0002817390724F43093C8032093C703409111
:10ACD000B0035091B1036091B2037091B303413856
:10ACE00051056105710574F0809182039091830391
:10ACF0002091C7033091C803820F931F9093830361
:10AD00008093820340585F4F6F4F7F4FCCF4809108
:10AD10008203909183032091C7033091C803821B63
:10AD2000930B90938303809382030AC010920803CD
:10AD30001092070310920603109205031092270346
:10AD40008091C807882341F41092080310920703EA
:10AD500010920603109205038091BB079091BC07E7
:10AD6000A091BD07B091BE078093CD039093CE0311
:10AD7000A093CF03B093D0038091C3079091C407F1
:10AD8000A091C507B091C6078093D1039093D203D9
:10AD9000A093D303B093D40310925F031092600387
:10ADA000109261031092620310925B0310925C0395
:10ADB00010925D0310925E03109257031092580395
:10ADC0001092590310925A031092BB071092BC07BD
:10ADD0001092BD071092BE071092C3071092C407CD
:10ADE0001092C5071092C6071092B2071092B307CF
:10ADF0001092B4071092B5071092A4071092A507FD
:10AE00001092A6071092A7071092330210923202F6
:10AE10000091150310911603C80117FF04C088277D
:10AE20009927801B910B40976CF088EE93E09093EC
:10AE3000BA018093B9018091100684FD03C081E0BE
:10AE40008093BA03F0901C06AF2CBB24CC24DD24E5
:10AE5000B801882777FD8095982F980117FF04C0C7
:10AE600022273327201B310B442737FD4095542FD1
:10AE70000E94457D9B01AC01C601B5010E94457D44
:10AE800097FF04C061507E4F8F4F9F4F59E09595BB
:10AE90008795779567955A95D1F79B018F2D9927BF
:10AEA000809FD001819FB00D909FB00D1124CD01E6
:10AEB000B7FD03969595879595958795280F391F2A
:10AEC000442737FD4095542F2093A0033093A103CE
:10AED0004093A2035093A30380913F0390914003BA
:10AEE000A0914103B0914203821B930BA40BB50BBD
:10AEF00080933F0390934003A0934103B093420398
:10AF00008155934CA040B04064F080E593ECA0E004
:10AF1000B0E080933F0390934003A0934103B0932C
:10AF2000420380913F0390914003A0914103B0916F
:10AF30004203805B9C43AF4FBF4F64F480EB9CE3C4
:10AF4000AFEFBFEF80933F0390934003A093410383
:10AF5000B0934203A0902D03B0902E03A114B1042E
:10AF600009F478C18091100683FF74C180916F034A
:10AF700090917003A0917103B0917203B7FF04C068
:10AF800081509E4FAF4FBF4F29E0B595A79597953C
:10AF900087952A95D1F76C0197FF04C0D094C1948E
:10AFA000D108D3948091670390916803A0916903BD
:10AFB000B0916A03B7FF04C081509E4FAF4FBF4F9F
:10AFC00009E0B595A795979587950A95D1F7BC01A6
:10AFD00097FF03C0709561957F4FC616D7060CF496
:10AFE0006B01B601D7FE02C0695F7F4F2B0113E0F2
:10AFF000559447941A95E1F7B2E0EB2EF12C4E0CE4
:10B000005F1C0CE112E0A00EB11E75010027F7FCD9
:10B010000095102F24EE3DEFA20EB31E8091F10794
:10B020009091F207A091F307B091F4076090950119
:10B03000709096018090970190909801BC01CD018D
:10B04000A40193010E94B97DE21AF30A040B150BC7
:10B05000C801B70128E631E040E050E00E94B97D28
:10B06000DC01CB01ACE4EA2EAFEFFA2EE80EF91EBC
:10B070000091B9011091BA010115110589F539E165
:10B08000C316D1046CF580912503909126038E0D93
:10B090009F1D90932603809325038091BA038823F4
:10B0A000F9F0C501AA2797FDA095BA2FBC01CD01E3
:10B0B000A40193010E94457DDC01CB018093F1073F
:10B0C0009093F207A093F307B093F407BC01CD016E
:10B0D0000E94B97D30932C0320932B031092BA0366
:10B0E000C701F4E0880F991FFA95E1F7B2010E94B9
:10B0F000847DCB01AA2797FDA095BA2F2091F10757
:10B100003091F2074091F3075091F407280F391F4F
:10B110004A1F5B1F2093F1073093F2074093F30718
:10B120005093F407F090AA016F2D7727C69EC001B7
:10B13000C79E900DD69E900D112497FD4F966C01E1
:10B14000E5E0D594C794EA95E1F76C197D096B01A8
:10B1500077FD7AC00115110509F06FC00091EC026E
:10B160001091ED028091EA029091EB02080F191FF5
:10B1700017FF02C0095F1F4F73E0159507957A9579
:10B18000E1F7005C1F4FCA01B901A40193010E94BD
:10B19000B97DDA01C90120912B0330912C0344279A
:10B1A00037FD4095542F821B930BA40BB50B845E87
:10B1B0009D4FAF4FBF4FBC01CD0128E631E040E0CD
:10B1C00050E00E94B97DDC01CB01845B90408C9DF6
:10B1D000A0018D9D500D9C9D500D1124CA01B801F8
:10B1E0000E94847D83E0F89E60011124C616D70674
:10B1F00014F4B60108C0882799278C199D0968178F
:10B2000079070CF4BC019B01442737FD4095542F6E
:10B2100080913F0390914003A0914103B09142037C
:10B22000820F931FA41FB51F80933F039093400389
:10B23000A0934103B09342030DC0015010401093FE
:10B24000BA010093B90106C084EF91E09093BA016E
:10B250008093B90180912703882381F010923303F2
:10B260001092340310923503109236031092370374
:10B27000109238031092390310923A03709002032F
:10B280007720F1F48091C807282F332744275527CA
:10B2900080916F0390917003A0917103B09172033C
:10B2A000BC01CD010E94457DDC01CB01BC01CD017B
:10B2B00028EF3AE240E050E00E94B97D290102C047
:10B2C00044245524909001039920F1F48091C807FB
:10B2D000282F3327442755278091670390916803CF
:10B2E000A0916903B0916A03BC01CD010E94457D24
:10B2F000DC01CB01BC01CD0128EF3AE240E050E097
:10B300000E94B97D190102C02224332480919E0736
:10B3100090919F07893C91051CF088EC90E005C056
:10B3200088539F4F34F488E39FEF90939F07809357
:10B330009E078091A9079091AA07893C91051CF06E
:10B3400088EC90E005C088539F4F34F488E39FEF6A
:10B350009093AA078093A9078091AB079091AC07BF
:10B36000AA2797FDA095BA2F2091EF07A22EBB2404
:10B37000CC24DD24BC01CD01A60195010E94457DB0
:10B380009B01AC0180919E0790919F07AA2797FD92
:10B39000A095BA2F67E0880F991FAA1FBB1F6A9557
:10B3A000D1F7280F391F4A1F5B1F57FF04C0215CCC
:10B3B0003F4F4F4F5F4F06E055954795379527957F
:10B3C0000A95D1F77201E20EF31EF092AC07E092FB
:10B3D000AB0780919C0790919D07AA2797FDA095A8
:10B3E000BA2FBC01CD01A60195010E94457D9B01AC
:10B3F000AC018091A9079091AA07AA2797FDA09573
:10B40000BA2F17E0880F991FAA1FBB1F1A95D1F7F3
:10B41000280F391F4A1F5B1F57FF04C0215C3F4F95
:10B420004F4F5F4FB6E05595479537952795BA959D
:10B43000D1F78101020F131F10939D0700939C0702
:10B440008091EA079091EB07880F991FAA2797FD33
:10B45000A095BA2F2091A307332744275527BC0175
:10B46000CD010E94457D5B016C0197FF08C08FE311
:10B4700090E0A0E0B0E0A80EB91ECA1EDB1EA6E058
:10B48000D594C794B794A794AA95D1F78091B8079B
:10B49000282F332744275527809153039091540335
:10B4A000A0915503B0915603BC01CD010E94457D8A
:10B4B000DC01CB01BC01CD0120EF35E540E050E0DF
:10B4C0000E94B97DB501620F731F7093EB07609303
:10B4D000EA0791E0E91690E1F90634F080E090E1A6
:10B4E0009093AC078093AB078091AB079091AC072A
:10B4F0008050904F34F480E090EF9093AC078093AD
:10B50000AB070150104134F080E090E190939D072B
:10B5100080939C0780919C0790919D078050904F4D
:10B5200034F480E090EF90939D0780939C076150E6
:10B53000704134F080E090E19093EB078093EA074C
:10B540008091EA079091EB078050904F34F480E0AF
:10B5500090EF9093EB078093EA0780910001482FCA
:10B56000552780911D0190911E014817590794F4A9
:10B5700020911D0130911E0168A179A1649FC00135
:10B58000659F900D749F900D1124B9010E94707DEC
:10B5900079A368A388A199A1880F991F880F991F83
:10B5A00099A388A34091100640FFA7C6992009F0EF
:10B5B000A4C6772009F0A1C6CC24DD2446018091E1
:10B5C0000303909104039093D9058093D8052091AB
:10B5D0008603309187032115310509F03FC0809122
:10B5E0001301909114018959934058F087B5803F19
:10B5F00020F480913602815011C081E08093E003F5
:10B600004EC080911301909114018436910508F584
:10B6100087B58031D0F0809136028F5F80933602FB
:10B620009FE08902900111248091FF05821B87BD54
:10B630008CE291E090932202809321028EE591E0CA
:10B6400090938703809386032AC081E08093DF0371
:10B6500026C07092DF037092E00321C080910D0339
:10B6600090910E03A0910F03B0911003E4E0880FB6
:10B67000991FAA1FBB1FEA95D1F7809337029093B9
:10B680003802A0933902B0933A02D0923502C092A8
:10B690003402215030403093870320938603209159
:10B6A000AD0141FF24C02233D8F48091BF01815005
:10B6B0008093BF018F3FD9F51092280380910D032D
:10B6C00090910E03A0910F03B09110038093090392
:10B6D00090930A03A0930B03B0930C0381E004C082
:10B6E00081E08093280388EC8093BF0120C0809183
:10B6F000990190919A01820F911D2091150633278F
:10B70000829FF001839FF00D929FF00D1124CF01D5
:10B71000AA2797FDA095BA2F8093090390930A0357
:10B72000A0930B03B0930C0381E0809328038091D6
:10B730006F0390917003A0917103B0917203E09038
:10B740009501F09096010091970110919801BC012C
:10B75000CD01A80197010E94B97D59016A0180912C
:10B76000670390916803A0916903B0916A03BC01DB
:10B77000CD01A80197010E94B97DB901C5010E94C0
:10B78000B0733C01CC971CF07CE3672E712CC30195
:10B790000E94BF6C3C0180E2809394018091280359
:10B7A000882309F436C48091E70299279C0120710F
:10B7B000307084FD2EC46091660660FD04C08091E7
:10B7C000100681FD07C008A119A13093D60320936C
:10B7D000D50397C18091E70281FF69C14091BB0108
:10B7E0005091BC01CA010F962091130330911403AC
:10B7F00082179307ACF58091DF03882389F5809148
:10B80000E10381FF13C08D7F8093E10380910D03DD
:10B8100090910E03A0910F03B09110038093090340
:10B8200090930A03A0930B03B0930C038091E10360
:10B8300081608093E103241B350B2F50304037FF8C
:10B8400003C0309521953F4F8091D5039091D60349
:10B85000820F931F9093D6038093D5038BE26EC023
:10B86000CA010F9728173907ACF58091E0038823A8
:10B8700089F58091E10380FF13C08E7F8093E103FF
:10B8800080910D0390910E03A0910F03B0911003CE
:10B890008093090390930A03A0930B03B0930C03C6
:10B8A0008091E10382608093E103241B350B215FCB
:10B8B0003F4F37FF03C0309521953F4F8091D5030F
:10B8C0009091D603821B930B9093D6038093D5035C
:10B8D0008DE234C02091E103822F9927837090700C
:10B8E000892B59F12C7F2093E1031092D6031092FB
:10B8F000D50320910D0330910E0340910F03509119
:10B9000010032093090330930A0340930B035093D1
:10B910000C0361FF06C084EF91E0909322028093B4
:10B92000210280911103882341F42333310541051D
:10B9300051051CF081E0809311038DE38093940105
:10B940002091D5033091D603C90137FF04C0882761
:10B950009927821B930B815092400CF491C08091E7
:10B9600015069927289FA001299F500D389F500D3B
:10B970001124CA0160E075E00E94847DCB01AA27F2
:10B9800097FDA095BA2F2091090330910A034091A9
:10B990000B0350910C03280F391F4A1F5B1F209384
:10B9A000090330930A0340930B0350930C03109246
:10B9B000D6031092D503A0900D03B0900E03C09053
:10B9C0000F03D0901003D601C50180509440A040D1
:10B9D000B04082179307A407B5075CF4D601C501F0
:10B9E00080509C4FAF4FBF4F281739074A075B075E
:10B9F00044F08093090390930A03A0930B03B09340
:10BA00000C038091660681FF06C084E690E0909367
:10BA100022028093210280911906882389F54091A2
:10BA200003035091040357FF02C04D5F5F4F5595CC
:10BA300047955595479580911D0190911E01209144
:10BA400000013327489FB001499F700D589F700D2A
:10BA50001124CB01B9010E94847D7093BC016093D5
:10BA6000BB01663471051CF486E490E005C06739BB
:10BA7000710534F086E990E09093BC018093BB019E
:10BA80008091860390918703892BB9F180910D03F2
:10BA900090910E03A0910F03B091100380930903BE
:10BAA00090930A03A0930B03B0930C0326C08091DC
:10BAB0000D0390910E03A0910F03B09110038059D4
:10BAC0009140A040B0408093090390930A03A09353
:10BAD0000B03B0930C0380911906882311F099276A
:10BAE00002C088E790E09093BC018093BB0188A1DD
:10BAF00099A1909304038093030300910303109191
:10BB00000403A0900D03B0900E03C0900F03D090DB
:10BB100010032091090330910A0340910B035091C7
:10BB20000C032A153B054C055D0524F08091660643
:10BB300080FDB1C28091860390918703892B39F0F3
:10BB40000091030310910403CC24DD24D7C0D60157
:10BB5000C501821B930BA40BB50B8093A403909398
:10BB6000A503A093A603B093A7038230E0E89E0745
:10BB7000EFEFAE07EFEFBE072CF481E090E8AFEFF8
:10BB8000BFEF09C08F5F9F47A040B04064F08FEFC8
:10BB90009FE7A0E0B0E08093A4039093A503A09357
:10BBA000A603B093A703C090A403D090A5038091EF
:10BBB000AC01282F3327442755278091A403909167
:10BBC000A503A091A603B091A703BC01CD010E94DB
:10BBD000457D97FF04C0615E7F4F8F4F9F4F55E0BB
:10BBE00095958795779567955A95D1F76093A403B6
:10BBF0007093A5038093A6039093A70365302EEF5F
:10BC000072072FEF82072FEF92072CF484E09EEF4C
:10BC1000AFEFBFEF09C0605074408040904064F0C7
:10BC200080E094E0A0E0B0E08093A4039093A503AB
:10BC3000A093A603B093A7038090A4039090A503BC
:10BC4000209134023091350237FF02C0295F3F4F07
:10BC500043E0359527954A95E1F74FEF22383407B1
:10BC60001CF421E83FEF05C02038310514F020E82E
:10BC700030E0C901AA2797FDA095BA2F2091AE0107
:10BC8000332744275527BC01CD010E94457D97FFEE
:10BC900004C06D5F7F4F8F4F9F4F22E09595879532
:10BCA000779567952A95D1F79B015FEF613075070E
:10BCB0001CF420E03FEF06C06F3F710519F014F04F
:10BCC00020E031E08091E103882349F0C90137FD8C
:10BCD00003969C0135952795359527950DC0809144
:10BCE000660680FF09C0C90137FD07969C01A3E0E5
:10BCF00035952795AA95E1F7820E931E2091AB0109
:10BD0000222309F454C060912F0370913003809175
:10BD100031039091320397FF04C061587F4F8F4FDA
:10BD20009F4FF7E09595879577956795FA95D1F7A9
:10BD30003327442755270E94457D97FF04C0615E45
:10BD40007F4F8F4F9F4FE5E0959587957795679546
:10BD5000EA95D1F76093A4037093A5038093A6039B
:10BD60009093A7036138AFEF7A07AFEF8A07AFEF81
:10BD70009A072CF480E89FEFAFEFBFEF0AC06F3F48
:10BD800071058105910569F064F080E091E0A0E023
:10BD9000B0E08093A4039093A503A093A603B0936F
:10BDA000A7038091A4039091A503880E991E80910A
:10BDB000A901282F332780916708992787FD90953F
:10BDC000289FF001299FF00D389FF00D11249F014D
:10BDD000F7FF02C021583F4F220F232F221F330BA2
:10BDE000FFEF21383F071CF420E83FEF06C02F3F4C
:10BDF000310519F014F020E031E0820E931EC401E9
:10BE0000AA2797FDA095BA2FE0900303F0900403B2
:10BE10009701442737FD4095542FBC01CD010E9466
:10BE2000457D97FF04C061507E4F8F4F9F4F59E073
:10BE300095958795779567955A95D1F7061B170BBA
:10BE40008091D5039091D603892B09F060C01E1410
:10BE50001F040CF05CC09601D7FE03C030952195FD
:10BE60003F4F2D33310540F48091D9039091DA038F
:10BE70008017910774F526C02C53304045E0369565
:10BE800027954A95E1F72031310510F02FE030E099
:10BE90004091D9035091DA031C141D04E4F480E1AD
:10BEA00090E0821B930B489F9001499F300D589F53
:10BEB000300D112494E0369527959A95E1F72017D7
:10BEC000310720F58091BD019091BE010817190737
:10BED000F4F08C011CC0205F3F4F8091BD01909118
:10BEE000BE01829FB001839F700D929F700D11243F
:10BEF0009B0184E0369527958A95E1F74017510715
:10BF000014F08A0104C00217130708F08901C80160
:10BF1000AA2797FDA095BA2F1DE0880F991FAA1F89
:10BF2000BB1F1A95D1F79301442737FD4095542F35
:10BF3000BC01CD010E94B97D2093A8033093A903D1
:10BF40004093AA035093AB030091A8031091A90357
:10BF50008091D7039091D8039C01220F331F280FA3
:10BF6000391F200F311F37FF02C02D5F3F4FA9013E
:10BF700055954795559547955093D8034093D703CA
:10BF800080911106282F3327220F331F220F331FD2
:10BF9000241735076CF48091E907282F3327220FE7
:10BFA000331F220F331F205530404217530724F010
:10BFB0003093D8032093D7038091660680FF14C086
:10BFC0008091D7039091D803A8A1B9A18A179B07A4
:10BFD00024F0B093D803A093D703E091D703F09156
:10BFE000D803F9A3E8A357C028A139A12E193F0906
:10BFF00037FF02C02D5F3F4F359527953595279523
:10C00000E090D703F090D803E20EF31EF9A2E8A265
:10C0100042C080911906882301F560910303709155
:10C02000040377FF02C06D5F7F4F75956795759527
:10C03000679540911D0150911E0180910001282FAC
:10C040003327649FC001659F900D749F900D11244C
:10C05000B9010E94847DCB0101C099279093BC0156
:10C060008093BB018091BB019091BC018734910505
:10C070001CF486E490E005C08639910534F086E929
:10C0800090E09093BC018093BB0108A119A110938B
:10C09000D8030093D7038091E70299279C0122706F
:10C0A000307081FF1CC18091DB039091DC03A09173
:10C0B000DD03B091DE030097A105B10521F0809169
:10C0C00011038130B1F428A139A1C901AA2797FD34
:10C0D000A095BA2F2EE0880F991FAA1FBB1F2A9583
:10C0E000D1F78093DB039093DC03A093DD03B0933F
:10C0F000DE0380911103813019F482E080931103F3
:10C1000048A159A1CA01AA2797FDA095BA2F93016A
:10C11000442737FD4095542FBC01CD010E94457D39
:10C12000DC01CB018093A8039093A903A093AA03F9
:10C13000B093AB03B7FF04C08150904EAF4FBF4FD9
:10C140005C016D018DE0D594C794B794A7948A954E
:10C15000D1F7A092A803B092A903C092AA03D092EB
:10C16000AB036091E8027091E9025FE0603A750705
:10C1700050F58091DB039091DC03A091DD03B09139
:10C18000DE039C01AD010AE056954795379527954A
:10C190000A95D1F7821B930BA40BB50BA601950151
:10C1A00014E0220F331F441F551F1A95D1F7820F39
:10C1B000931FA41FB51F8093DB039093DC03A09310
:10C1C000DD03B093DE0360547F4118F58091DB03FB
:10C1D0009091DC03A091DD03B091DE039C01AD01E1
:10C1E000FCE05695479537952795FA95D1F7821B30
:10C1F000930BA40BB50BA6019501E2E0220F331FB0
:10C20000441F551FEA95D1F7820F931FA41FB51F36
:10C2100029C080913402909135028091340290912E
:10C22000350297FF03C0909581959F4F8436910505
:10C230000CF58091DB039091DC03A091DD03B091BC
:10C24000DE039C01AD017EE0569547953795279515
:10C250007A95D1F7821B930BA40BB50B8A0D9B1D0E
:10C26000AC1DBD1D8093DB039093DC03A093DD0325
:10C27000B093DE038091DB039091DC03A091DD039A
:10C28000B091DE036EE0B695A795979587956A9570
:10C29000D1F790930403809303034091170644233E
:10C2A00099F055279C01BA010E94847DC901861B23
:10C2B000970B9093DA038093D903260F371F30939F
:10C2C000BE012093BD0119C01092DA031092D90368
:10C2D0008FEF93E09093BE018093BD010EC010924A
:10C2E00011031092DB031092DC031092DD03109215
:10C2F000DE0330930403209303039091B00798ABBF
:10C30000292F3327220F331F220F331F285D3F4F62
:10C31000A8A1B9A12A173B0714F039A328A3B0910B
:10C32000E907B9AB8B2F9927880F991F880F991FA1
:10C3300080559040E8A1F9A18E179F0714F499A3A6
:10C3400088A380916C02882321F480916E088F3F2E
:10C35000A1F08091E8029091E9020297C09768F4F9
:10C36000E8A0F9A01E141F0444F481E090E090932B
:10C37000E9028093E80239A328A308A119A1109328
:10C38000BD050093BC058091A0039091A103A091ED
:10C39000A203B091A30322E0880F991FAA1FBB1F1D
:10C3A0002A95D1F7C090EA07D090EB07C81AD90AAE
:10C3B000013A11058CF0C80117FD019695958795F6
:10C3C0008C159D050CF46C01909581959F4FC816B6
:10C3D000D90694F46C0110C011E5C116D1041CF00B
:10C3E000E0E5CE2ED12C20EBC2162FEFD20624F49E
:10C3F00070EBC72E7FEFD72E49A9242F3327220FAA
:10C40000331F220F331FC90168A179A1861B970B27
:10C410008C159D050CF46C0188A199A1821B930BCE
:10C42000C816D9060CF46C018091AB079091AC074B
:10C430006091190370911A03861B970B9093BA07AA
:10C440008093B907A090C807209137033091380333
:10C450004091390350913A03AA2041F0461A570AF5
:10C46000C201AA2797FDA095BA2F04C0AA2797FD5D
:10C47000A095BA2F280F391F4A1F5B1F209337033F
:10C48000309338034093390350933A038091370334
:10C4900090913803A0913903B0913A0381509A4F9B
:10C4A000A040B04064F080E09AEFA0E0B0E080935C
:10C4B000370390933803A0933903B0933A038091E4
:10C4C000370390913803A0913903B0913A0380501B
:10C4D0009640AF4FBF4F64F480E096E0AFEFBFEF00
:10C4E0008093370390933803A0933903B0933A03B2
:10C4F000B09026062B2D33278091B9079091BA076B
:10C50000289F7001299FF00C389FF00C112497018F
:10C51000F7FE02C0295F3F4F790153E0F594E7949D
:10C520005A95E1F70091AF011091B00198014427AD
:10C5300037FD4095542F8091370390913803A09197
:10C540003903B0913A03BC01CD010E94B97DE20EDE
:10C55000F31E90909B01692D7727882799279601D4
:10C56000D7FE04C0222733272C193D0937FF02C00C
:10C570002F5F3F4F3595279548A159A1240F351FAF
:10C58000442737FD4095542F0E94457D97FF04C0F6
:10C59000615C7F4F8F4F9F4F26E0959587957795EC
:10C5A00067952A95D1F79B016E157F050CF47B01E9
:10C5B000309521953F4FE216F3060CF479018091F6
:10C5C0009C0790919D076091170370911803861B3B
:10C5D000970B90939B0780939A0720913303309198
:10C5E00034034091350350913603AA2041F0261AB6
:10C5F000370AC101AA2797FDA095BA2F04C0AA2720
:10C6000097FDA095BA2F280F391F4A1F5B1F209353
:10C6100033033093340340933503509336038091B2
:10C62000330390913403A0913503B09136038150C8
:10C630009A4FA040B04064F080E09AEFA0E0B0E0F4
:10C640008093330390933403A0933503B093360360
:10C650008091330390913403A0913503B091360358
:10C6600080509640AF4FBF4F64F480E096E0AFEF4C
:10C67000BFEF8093330390933403A0933503B093BB
:10C6800036032B2D332780919A0790919B07289F83
:10C69000D001299FB00D389FB00D11249D01B7FF27
:10C6A00002C0295F3F4F5901B3E0B594A794BA95F2
:10C6B000E1F79801442737FD4095542F80913303CB
:10C6C00090913403A0913503B0913603BC01CD01A4
:10C6D0000E94B97DA20EB31E692D7727882799275E
:10C6E0009601D7FE04C0222733272C193D0937FFB6
:10C6F00002C02F5F3F4F35952795E8A1F9A12E0F76
:10C700003F1F442737FD4095542F0E94457D97FFDA
:10C7100004C0615C7F4F8F4F9F4FF6E095958795E2
:10C7200077956795FA95D1F79B016A157B050CF40F
:10C730005B01309521953F4FA216B3060CF45901C9
:10C74000EAEC6E2EE6E07E2E71E8872E76E0972EDC
:10C750006BE0362E59EC452E57E0552ED4012C9126
:10C7600012160CF0DFC0203419F408A119A11EC064
:10C77000E8A1F9A1CF01AA2797FDA095BA2F3327E9
:10C7800027FD3095432F532FBC01CD010E94457DDD
:10C7900097FF04C0615C7F4F8F4F9F4F46E0959598
:10C7A0008795779567954A95D1F78B01F40121819B
:10C7B000203419F40E0D1F1D22C0203C19F40E194F
:10C7C0001F091DC0C701AA2797FDA095BA2F3327BF
:10C7D00027FD3095432F532FBC01CD010E94457D8D
:10C7E00097FF04C0615C7F4F8F4F9F4F36E0959558
:10C7F0008795779567953A95D1F7060F171FF4013E
:10C800002281203419F40A0D1B1D22C0203C19F48A
:10C810000A191B091DC0C501AA2797FDA095BA2FAB
:10C82000332727FD3095432F532FBC01CD010E94A4
:10C83000457D97FF04C0615C7F4F8F4F9F4F26E07F
:10C8400095958795779567952A95D1F7060F171FC8
:10C85000F4012381203419F40C0D1D1D22C0203C4D
:10C8600019F40C191D091DC0C601AA2797FDA09532
:10C87000BA2F332727FD3095432F532FBC01CD010D
:10C880000E94457D97FF04C0615C7F4F8F4F9F4F93
:10C89000B6E09595879577956795BA95D1F7060F88
:10C8A000171FD2018D919C91801791075CF4BC01F8
:10C8B000600F711F77FF02C06F5F7F4F8B0115956F
:10C8C000079504C0000F111F081B190BB8A98B2F67
:10C8D0009927880F991F880F991F8017910754F483
:10C8E000E9A98E2F9927880F991F880F991F08177C
:10C8F00019070CF08C01C80117FD039695958795D3
:10C9000095958795F3018183880F991F880F991F4B
:10C910009801281B390BC901880F8283D2010D931E
:10C920001C9303C0F301118212823A9402E010E0DA
:10C93000400E511E24E030E0820E931E48E050E08D
:10C94000640E751E37FE0ACFE2E1CB5C0C94F07DDD
:10C950008091EE039091EF03A091F003B091F10369
:10C960008093E6039093E703A093E803B093E90371
:10C970008091EA039091EB03A091EC03B091ED0359
:10C980008093E2039093E303A093E403B093E50361
:10C9900008951092F9031092F8031092F703109281
:10C9A000F603089584B1806A84B93D9A82E58CBD0E
:10C9B0001DBC459A81E08093FB078AEA80930C08AE
:10C9C00083E880930D088AE080930E081092100887
:10C9D00010920F0810921208109211081092660817
:10C9E00010922E0808953091FB07332309F085C07B
:10C9F0000DB407FE82C084E080932002459A2EB5D4
:10CA00008091FD0399278130910589F0823091054D
:10CA10001CF4892B21F03EC00297B9F03BC0309343
:10CA20002D082093FE032138A9F581E008C02535A3
:10CA300049F48091FE03820F8093FE0382E080938D
:10CA4000FD0328C03093FD0325C080912D08E82FF9
:10CA5000FF27E75BF74F20838F5F80932D0890912E
:10CA6000FE038A31A0F0291769F48AE1A9E4B8E04D
:10CA7000EFE2F8E00D9001928A95E1F781E0809372
:10CA80002E0802C030932E081092FD0303C0920FAF
:10CA90009093FE0320910B08203208F028C045989F
:10CAA0000000000000000000000000000000000086
:10CAB0000000000000000000000000000000000076
:10CAC0000000000000000000000000000000000066
:10CAD000E0910408F0910508E20FF11D80818EBD00
:10CAE00080912B089081890F80932B0803C081E0EF
:10CAF0008093FB072F5F20930B080895EF92FF921E
:10CB00000F931F9380911F069927880F991F880FF5
:10CB1000991F7C010027F7FC0095102F80916F036F
:10CB200090917003A0917103B0917203BC01CD018B
:10CB3000A80197010E94B97D3093100820930F0837
:10CB40008091670390916803A0916903B0916A0393
:10CB5000BC01CD01A80197010E94B97D3093120854
:10CB6000209311082091F1073091F2074091F307CB
:10CB70005091F407DA01C901E3E0880F991FAA1F59
:10CB8000BB1FEA95D1F7820F931FA41FB51F820F19
:10CB9000931FA41FB51F20919501309196014091DC
:10CBA000970150919801BC01CD010E94B97D30934D
:10CBB0001808209317088091800390918103209199
:10CBC000420230914302821B930B90931E08809384
:10CBD0001D08E0917603F09177038091C007909152
:10CBE000C107BF010E94847DCB019B01220F331F2F
:10CBF000220F331F280F391F280F391F37FF02C09C
:10CC00002D5F3F4F3595279535952795309314081F
:10CC1000209313088091ED079091EE07BF010E94C9
:10CC2000847D9B01220F331F220F331F260F371FD6
:10CC3000260F371F37FF02C02D5F3F4F35952795D1
:10CC40003595279530931608209315081092770391
:10CC5000109276031092C1071092C0071092EE074F
:10CC60001092ED0780910E0899278D30910509F4F7
:10CC700066C08E3091055CF48B30910509F48EC04E
:10CC80008C3091050CF00FC10A9761F0A8C18F306C
:10CC9000910509F47CC18F3091050CF45CC140977B
:10CCA00099F19DC18091FC0280931F088091FB0245
:10CCB000809320088091FA02809321088091F902E4
:10CCC000809322088091F802809323088091F702D4
:10CCD000809324088091F602809325088091F502C4
:10CCE000809326088091E702809327088091E702CD
:10CCF000837F8093E7020E944730809328088091C9
:10CD00007303809329086BC180916808909169082A
:10CD10009093200880931F0880916C0890916D0873
:10CD2000909322088093210880911D0190911E010B
:10CD300080932308809100018093240850C1809142
:10CD4000510680931F08809152068093200880919D
:10CD50005306809321088091540680932208809185
:10CD6000550680932308809159068093240880916A
:10CD70005A068093250880915B068093260880914F
:10CD80005E068093270880915C0680932808809136
:10CD90005D068093290880915F06DAC0F89480913F
:10CDA0000606E82FFF27EE0FFF1FE55DF84F019005
:10CDB000F081E02DE038F1051CF0EFE7F0E006C06F
:10CDC0002FEFE138F20714F4E1E8FFEFE0931F08DA
:10CDD00080910706E82FFF27EE0FFF1FE55DF84F54
:10CDE0000190F081E02DE038F1051CF0EFE7F0E074
:10CDF00006C06FEFE138F60714F4E1E8FFEFE093C7
:10CE0000200880910506E82FFF27EE0FFF1FE55D44
:10CE1000F84F0190F081E02DE038F1051CF0EFE7CC
:10CE2000F0E006C08FEFE138F80714F4E1E8FFEF17
:10CE3000E093210880910406E82FFF27EE0FFF1FE3
:10CE4000E55DF84F0190F081E02DE038F1051CF030
:10CE5000EFE7F0E006C02FEFE138F20714F4E1E865
:10CE6000FFEF7894E093220880911C0380932308BD
:10CE700080911D038093240880911E0380932508D0
:10CE800080911F03809326088091200380932708B8
:10CE900080912103809328088091220380932908A0
:10CEA0008091230355C080915B04863018F0109266
:10CEB0005B0485E080931F088091600680932008C2
:10CEC00080910D0390910E03A0910F03B091100378
:10CED000BC01CD0125E030E040E050E00E94B97D8A
:10CEE00030932208209321088091090390910A032E
:10CEF000A0910B03B0910C03BC01CD0125E030E003
:10CF000040E050E00E94B97D30932408209323082C
:10CF100080915606809325088091570680932608B5
:10CF2000809158068093270880911B0380932808DE
:10CF300080912B0790912C07809329088091BC0544
:10CF40009091BD0597FD0396959587959595879545
:10CF500080932A0844C010921F0880E5809320081F
:10CF600086E0809321088EE0809322088091020160
:10CF70008093230880914004809324088091410489
:10CF800080932508809142048093260828C08091D0
:10CF9000380680931F088091650680932008809151
:10CFA000A10180932108809131068093220880910D
:10CFB0003206809323088091330680932408809161
:10CFC000A0018093250880913506809326088091E2
:10CFD0003606809327088091370680932808809131
:10CFE0002E08882309F4CFC08AEF8093E80140918E
:10CFF000300850913108CA0181509E4F8F5F934095
:10D00000B0F42091320830913308C90181509E4F0D
:10D010008F5F934060F48091100685FF08C05093A5
:10D02000F9034093F8033093F7032093F6038091BC
:10D0300036089091370821E08936920724F49093BE
:10D040002E0380932D0380912D0390912E03209128
:10D050002B0330912C03821B930B845E9D4F68E65B
:10D0600071E00E94847D845B904090932A038093BA
:10D07000290320913A0830913B0880912102909138
:10D0800022028217930740F480915B04882321F4E5
:10D09000309322022093210280912F08992788360D
:10D0A000910549F18936910524F48736910531F0CF
:10D0B00072C08936910509F445C06DC080913C0865
:10D0C0008093630880913D088093650880913E08B5
:10D0D0008093640880913F0880936608809140089F
:10D0E00080936708809141088093E901809142080C
:10D0F0008093FC0350C080913C0880930608809187
:10D100003D088093070880913E088093080880912D
:10D110003F08809309088091400880930A08809115
:10D12000AC0590914108892B8093AC059091420801
:10D130009093FA038091AD0583709C70892B809346
:10D14000AD0529C080913C088093FC0780913D0883
:10D150008093FD0780913E088093FE0780913F08F1
:10D160008093FF07809140089091410890930108B7
:10D17000809300088091420890914308909303089F
:10D180008093020808C01092F9031092F8031092DD
:10D19000F7031092F6031F910F91FF90EF900895FF
:10D1A0008091FB07882309F43BC045988CE098E008
:10D1B00090930508809304089091FB03E92FFF27C3
:10D1C000E152FE4F9F5F9093FB03808180930E0896
:10D1D000993010F01092FB031092FB070E947E65BD
:10D1E00081E080930B0800000000000000000000B8
:10D1F000000000000000000000000000000000002F
:10D20000000000000000000000000000000000001E
:10D2100000000000000080910C0880932B088EBD58
:10D22000089587B18C6087B94298439810920004A2
:10D2300080E88093EB011092FF038093EA01089548
:10D24000809105048150809305048F3F09F0F4C05C
:10D2500094E0909305048091E702807BE1F0809157
:10D260004F06882349F080910804882311F4909395
:10D27000000481E080930804809150068823B9F06F
:10D2800080910904882319F484E08093FF0381E0EE
:10D29000809309040CC08093080480930904809152
:10D2A0004B068093060480914D068093070480917D
:10D2B0000804882309F040C080916406282F332792
:10D2C00024FF07C080911203882319F425FD4DC067
:10D2D0004EC090914C06983F50F08091C2078D3D12
:10D2E00030F08091060488230CF43FC040C0983F82
:10D2F00048F08091C2078A3028F480910604882380
:10D30000B4F133C0809100048150809300048F3FBA
:10D3100079F58091C2078150809300048091EB01E0
:10D32000813011F480E801C086958093EB018091F3
:10D33000EB019091060417C0809100048150809306
:10D3400000048F3FA9F489E0809300048091EB01F1
:10D35000813011F480E801C086958093EB018091C3
:10D36000EB0190914F06892311F0429A01C0429837
:10D3700080910904882309F043C080916406282F16
:10D38000332724FF07C080911203882319F426FD58
:10D3900050C034C090914E06983F50F08091E807FD
:10D3A0008D3D30F08091070488230CF442C026C0E4
:10D3B000983F48F08091E8078A3028F4809107046C
:10D3C0008823E4F036C08091FF0381508093FF03EF
:10D3D0008F3F91F58091E80781508093FF03809102
:10D3E000EA01813011F480E801C086958093EA015A
:10D3F0008091EA01909107048923D9F44398089514
:10D400008091FF0381508093FF038F3FA9F489E04F
:10D410008093FF038091EA01813011F480E801C01C
:10D4200086958093EA018091EA01909150068923C4
:10D4300011F0439A0895439808954FB724E130E0DE
:10D44000F8948091C9008F778093C9008091C900BA
:10D450008F7B8093C9008091C9008F7D8093C90024
:10D460005A9A52985B9A539A832F99278093CD00AA
:10D470002093CC008091C80082608093C80080E136
:10D480008093C9008091CA008F778093CA008091F1
:10D49000CA008F7B8093CA008091CA008F7D8093E1
:10D4A000CA008091CA008F7E8093CA008091CA0012
:10D4B000877F8093CA008091C9008B7F8093C900C9
:10D4C0008091CA0084608093CA008091CA00826003
:10D4D0008093CA008091C80087FF03C08091CE006E
:10D4E000F9CF8091C90080688093C9004FBF08952B
:10D4F000FF920F931F93CF93DF9380E197E20E94F7
:10D500002617EC01FF248091C9008F778093C90012
:10D510008091C9008F7E8093C9005A9881E49AE077
:10D520009F938F930FEF12E11F930F93E0912704C6
:10D53000F091280409950F900F900F900F9002C062
:10D540004A996CC0CE010E942F178823C9F3E0913D
:10D550002704F0912804FF2009F468C087E79AE0C7
:10D560009F938F931F930F930995529A0F900F904B
:10D570000F900F90CE010E942F178823D9F383E6D6
:10D5800090E05A9A019797FFFCCF8FE891E05A9864
:10D59000019797FFFCCF89E090E05A9A019797FF97
:10D5A000FCCF89E090E05A98019797FFFCCF8FE875
:10D5B00091E05A9A019797FFFCCF8FE891E05A9833
:10D5C000019797FFFCCF89E090E05A9A019797FF67
:10D5D000FCCF89E090E05A98019797FFFCCF8FE845
:10D5E00091E05A9A019797FFFCCF8FE891E05A9803
:10D5F000019797FFFCCF89E090E05A9A019797FF37
:10D60000FCCF89E090E05A98019797FFFCCF8FE814
:10D6100091E05A9A019797FFFCCF13C08AE590E0FA
:10D620000E942617EC0191E0F92E91CF8DE79AE048
:10D630009F938F931F930F9309950F900F900F90C7
:10D640000F9052985A980E941D6AE5E0CDB7DEB758
:10D650000C94FD7DEF92FF920F931F93CF93DF9376
:10D66000482F00E010E08091EC01813061F41092CD
:10D67000EC0184E480930A0410920C0410920B04D1
:10D6800010920D042BC180910A04882319F421E023
:10D6900030E001C0980190910B04992371F4232B81
:10D6A00011F081E010C084E480930A0490930C048C
:10D6B00090930B0490930D04FAC0913069F4232BDE
:10D6C00009F0EBC082E080930B0480910C048F5F23
:10D6D00080930C0483E0E9C09230D1F4232B09F04D
:10D6E000DCC083E080930A0440930D0490910C0405
:10D6F000923039F410920E0447FF03C081E080930A
:10D700000E0483E080930B049F5F90930C04CFC0C2
:10D71000933009F0C2C0232B09F0BFC090930A04D4
:10D7200082E080930B0480910C048F5F80930C0443
:10D7300020910D04822F9927782F6627842F99270F
:10D74000682B792B80912A06813049F47370CB01C4
:10D750008050924063E070E00E94847D17C0823068
:10D7600061F47770CB018050944066E070E00E94D5
:10D77000847D2695269526950BC07370685671405A
:10D78000CB0177FD0196BC01759567952695269589
:10D79000022F11270F7010700F5F1F4F0D301105F2
:10D7A00008F074C07801E00EF11EF701E55DF84F56
:10D7B000808191819B01281B390BC90137FF03C070
:10D7C000909581959F4F069794F480911B03883C18
:10D7D00030F480911B03865F80931B0308C088ECA4
:10D7E00080931B0380916F008F7D80936F00F70102
:10D7F000E55DF84F808191819C01220F331F280F36
:10D80000391F260F371F37FF02C02D5F3F4FE90139
:10D81000D595C795D595C795CB0101968C179D07D2
:10D8200014F4219706C061507040C617D7070CF456
:10D83000219680911B03843BD0F0F701E55DF84F02
:10D8400080819181FE01E81BF90BCF0163E070E05C
:10D850000E94847DCB01880F991F860F971F2FE5AB
:10D8600037E0E20EF31EF7019183808307C02FE5B6
:10D8700037E0E20EF31EF70111821082000F111F34
:10D88000055D184FF801D183C08311C00231110525
:10D8900070F081E08093EC010AC081E08093EC019C
:10D8A00010920C0410920E0484E480930A04809178
:10D8B0000C04803198F080910E04882331F480911B
:10D8C000EC01882311F48093930110920C041092C0
:10D8D0000E0410920B0484E480930A04E6E0CDB7B2
:10D8E000DEB70C94FC7DCF93FC0197FF05C0CFEF12
:10D8F000F095E195FF4F01C0C1E028E631E0CF018E
:10D90000B9010E94847DFC018B35910554F08B5543
:10D9100090408A35910538F484EB90E08E1B9F0B84
:10D92000FC0141E00DC0CF01855B90408A35910537
:10D9300018F4E45BF04003C02E1B3F0BF9014FEFDE
:10D94000EE0FFF1FE857F54F259134918C2F992743
:10D9500087FD9095289FB001299F700D389F700D0D
:10D960001124842F992787FD9095689FA001699FB6
:10D97000500D789F500D1124CA01CF9108952AE5CA
:10D9800030E0281B390BC9010E94736C0895CF93B6
:10D99000DF9380E00E94947580911D0190911E019B
:10D9A0006AE070E00E94847D9F938F9380911D01B7
:10D9B00090911E016AE070E00E94847D7F936F93D6
:10D9C00086E89BE09F938F93C7E8D5E7DF93CF93DB
:10D9D000E0912704F091280409952DB73EB7285F00
:10D9E0003F4F2DBF8091E8018823B9F186E00E9466
:10D9F000947580910008909101086AE070E00E949F
:10DA0000707D7F936F938FED90E09F938F938091C4
:10DA1000F1079091F207A091F307B091F4072091DC
:10DA20009501309196014091970150919801BC0168
:10DA3000CD010E94B97D3F932F938FE89BE09F9388
:10DA40008F93DF93CF93E0912704F09128040995F9
:10DA50008DB79EB70A968DBF12C086E00E9494755E
:10DA60008BE99BE09F938F93DF93CF93E091270403
:10DA7000F091280409950F900F900F900F908091CE
:10DA8000FA038823C1F086E00E9494758091FA031E
:10DA900099279F938F9382EA9BE09F938F93DF93C5
:10DAA000CF93E0912704F091280409952DB73EB754
:10DAB0002A5F3F4F2DBF80E10E9494758091F30152
:10DAC0009091F4016CE370E00E94707D9F938F93BE
:10DAD0008091F3019091F4016CE370E00E94707DFD
:10DAE0007F936F9380916C0890916D089F938F93B3
:10DAF0008DEA9BE09F938F93C7E8D5E7DF93CF93A1
:10DB0000E0912704F09128040995809110062DB723
:10DB10003EB7265F3F4F2DBF80FF29C08AE10E949C
:10DB200094758091940199279F938F9380910D0311
:10DB300090910E03A0910F03B0911003BC01CD0191
:10DB400024E630E040E050E00E94B97D3F932F93FF
:10DB50008AEB9BE09F938F93DF93CF93E091270411
:10DB6000F091280409958DB79EB708968DBFDF9177
:10DB7000CF910895CF93DF9380E00E9494758091B8
:10DB8000E906992787FD90959F938F938091E106F1
:10DB9000992787FD90959F938F938091D906992718
:10DBA00087FD90959F938F938091D106992787FD4C
:10DBB00090959F938F9381EC9BE09F938F93C7E801
:10DBC000D5E7DF93CF93E0912704F09128040995DE
:10DBD00080E10E9494752DB73EB7245F3F4F2DBF63
:10DBE00080910907992787FD90959F938F93809146
:10DBF0000107992787FD90959F938F938091F90650
:10DC0000992787FD90959F938F938091F10699278F
:10DC100087FD90959F938F9381ED9BE09F938F93CA
:10DC2000DF93CF93E0912704F09128040995809128
:10DC300002062DB73EB7245F3F4F2DBF853098F4C5
:10DC400080E10E94947581EE9BE09F938F93DF9318
:10DC5000CF93E0912704F091280409950F900F903D
:10DC60000F900F9018C08730B0F488E10E9494752F
:10DC70008FED90E09F938F9382EF9BE09F938F9324
:10DC8000DF93CF93E0912704F091280409958DB795
:10DC90009EB706968DBFDF91CF9108950F931F9386
:10DCA00080E00E9494752AE030E0809168089091AD
:10DCB0006908B9010E94707D9F938F9380916808D5
:10DCC00090916908B9010E94707D7F936F93809154
:10DCD0001D0190911E01B9010E94847D9F938F9335
:10DCE00080911D0190911E01B9010E94847D7F9356
:10DCF0006F938BEF9BE09F938F9307E815E71F933C
:10DD00000F93E0912704F0912804099580E10E9487
:10DD100094758DB79EB70C968DBF80916C089091CD
:10DD20006D089F938F9380916A0890916B089F93E1
:10DD30008F938EE09CE09F938F931F930F93E091BE
:10DD40002704F091280409958DB79EB708968DBFDA
:10DD50001F910F9108950F931F93CF93DF9380919D
:10DD6000E801C7E8D5E7882309F478C080E00E947D
:10DD700094758091FD0799279F938F938091FF075A
:10DD800099279F938F938AE19CE09F938F938E01B5
:10DD9000DF93CF93E0912704F091280409958DB784
:10DDA0009EB708968DBF8091FE07833031F48CE0DA
:10DDB0000E94947589E29CE005C08CE00E949475F5
:10DDC0008EE29CE09F938F93DF93CF93E0912704A3
:10DDD000F091280409950F900F900F900F9080916B
:10DDE000FC0781FF12C08CE00E94947583E39CE0E5
:10DDF0009F938F931F930F93E0912704F091280432
:10DE000009950F900F900F900F9080E10E949475EC
:10DE10008FED90E09F938F9380910208909103087B
:10DE20009F938F9380910008909101086AE070E0C1
:10DE30000E94707D7F936F9388E39CE09F938F9304
:10DE400087E895E79F938F93E0912704F09128044A
:10DE500009958DB79EB70A968DBF12C082E00E94C9
:10DE6000947588E49CE09F938F93DF93CF93E09128
:10DE70002704F091280409950F900F900F900F90B0
:10DE8000DF91CF911F910F910895CF93DF9380E0A1
:10DE90000E9494758091E70699270C979F938F9322
:10DEA0008091DF0699270C979F938F938091D706D7
:10DEB00099270C979F938F938091CF0699270C9762
:10DEC0009F938F9385E59CE09F938F93C7E8D5E759
:10DED000DF93CF93E0912704F0912804099580E126
:10DEE0000E9494752DB73EB7245F3F4F2DBF8091A0
:10DEF000070799270C979F938F938091FF06992787
:10DF00000C979F938F938091F70699270C979F9377
:10DF10008F938091EF0699270C979F938F9385E6B7
:10DF20009CE09F938F93DF93CF93E0912704F09130
:10DF300028040995809102062DB73EB7245F3F4F14
:10DF40002DBF853098F480E10E94947585E79CE0B0
:10DF50009F938F93DF93CF93E0912704F091280450
:10DF600009950F900F900F900F9028C0873030F5D3
:10DF700088E10E94947580916808909169086AE030
:10DF800070E00E94707D9F938F93809168089091BC
:10DF900069086AE070E00E94707D7F936F9382E869
:10DFA0009CE09F938F93DF93CF93E0912704F091B0
:10DFB000280409958DB79EB708968DBFDF91CF9144
:10DFC0000895CF93DF9380E00E9494758091E306DB
:10DFD00099279F938F938091DB0699279F938F9327
:10DFE0008091D30699279F938F938091CB06992791
:10DFF0009F938F938CE89CE09F938F93C7E8D5E71E
:10E00000DF93CF93E0912704F0912804099580E1F4
:10E010000E9494752DB73EB7245F3F4F2DBF80916E
:10E02000030799279F938F938091FB0699279F93CE
:10E030008F938091F30699279F938F938091EB069E
:10E0400099279F938F938CE99CE09F938F93DF9305
:10E05000CF93E0912704F09128040995809102065E
:10E060002DB73EB7245F3F4F2DBF853030F480E1A0
:10E070000E9494758CEA9CE007C0873090F488E198
:10E080000E9494758DEB9CE09F938F93DF93CF93C9
:10E09000E0912704F091280409950F900F900F90BC
:10E0A0000F90DF91CF9108956F927F928F929F9200
:10E0B000AF92BF92CF92DF92EF92FF920F931F9396
:10E0C000A0903703B0903803C0903903D0903A0342
:10E0D00029E0D594C794B794A7942A95D1F7E090F6
:10E0E0003303F0903403009135031091360399E027
:10E0F00015950795F794E7949A95D1F760903F03AB
:10E1000070904003809041039090420389E0959481
:10E110008794779467948A95D1F780E00E949475EC
:10E12000FF92EF92BF92AF9286EC9CE09F938F9309
:10E1300007E815E71F930F93E0912704F091280457
:10E14000099580E10E9494758DB79EB708968DBFA2
:10E150007F926F9284ED9CE09F938F931F930F9318
:10E16000E0912704F091280409958DB79EB7069693
:10E170008DBF1F910F91FF90EF90DF90CF90BF90D8
:10E18000AF909F908F907F906F900895CF93DF9383
:10E1900080E00E94947580910303909104039F9303
:10E1A0008F9385EE9CE09F938F93C7E8D5E7DF932D
:10E1B000CF93E0912704F0912804099580E10E9413
:10E1C00094758DB79EB706968DBF8091130390917D
:10E1D00014039F938F93809103039091040397FD01
:10E1E000039695958795959587959F938F9382EF45
:10E1F0009CE09F938F93DF93CF93E0912704F0915E
:10E20000280409958DB79EB708968DBFDF91CF91F1
:10E2100008950F931F93CF93C82F80E00E949475A9
:10E2200080914507909146079F938F9383E09DE0EF
:10E230009F938F9307E815E71F930F93E0912704AF
:10E24000F0912804099580E10E9494758DB79EB7DE
:10E2500006968DBF80914707909148079F938F93B3
:10E2600083E19DE09F938F931F930F93E091270489
:10E27000F091280409958DB79EB706968DBFCF32D1
:10E2800031F48091450790914607019607C0CF343D
:10E2900049F480914507909146070197909346076E
:10E2A00080934507CF911F910F9108950F931F936E
:10E2B000CF93C82F80E00E9494758091450790917C
:10E2C00046079F938F9383E29DE09F938F9307E888
:10E2D00015E71F930F93E0912704F0912804099507
:10E2E00080E10E9494758DB79EB706968DBF8C2FE6
:10E2F00099279F938F9380914707909148079F9309
:10E300008F9383E39DE09F938F931F930F93E091EF
:10E310002704F091280409958DB79EB708968DBF04
:10E32000CF3231F48091470790914807059607C096
:10E33000CF3449F48091470790914807059790930F
:10E34000480780934707CF911F910F9108950F932E
:10E350001F93CF93C82F80E00E949475809112067E
:10E3600099279F938F9383E49DE09F938F9307E872
:10E3700015E71F930F93E0912704F0912804099566
:10E3800080E10E9494758DB79EB706968DBF8091EF
:10E39000140699279F938F938BE49DE09F938F930F
:10E3A0001F930F93E0912704F091280409958DB7EE
:10E3B0009EB706968DBFCF3221F4809112068F5FF3
:10E3C00005C0CF3429F48091120681508093120643
:10E3D000CF911F910F9108950F931F93CF93C82F43
:10E3E00080E00E9494758091120699279F938F93E5
:10E3F00083E59DE09F938F9307E815E71F930F93A5
:10E40000E0912704F0912804099580E10E94947519
:10E410008DB79EB706968DBF8091140699279F935E
:10E420008F938BE59DE09F938F931F930F93E091C4
:10E430002704F091280409958DB79EB706968DBFE5
:10E44000CF3221F4809114068F5F05C0CF3429F4B8
:10E4500080911406815080931406CF911F910F91E3
:10E460000895CF93C82F20910F042093100499276B
:10E470008F32910509F1803391051CF44F97A1F07B
:10E480002CC08F34910501F18F38910531F522238D
:10E4900019F481E090E038C086E0289FF001112453
:10E4A000E25CF44F849117C086E0289FF0011124AC
:10E4B000E15CF44F84910FC086E0289FF0011124A5
:10E4C000E05CF44F849107C086E0289FF00111249E
:10E4D000EF5BF44F849180930F0490910F0480912F
:10E4E00010049813C0E00E949A7590910F0486E082
:10E4F000989FF0011124EE5BF44F259134918C2FFD
:10E50000F901099580E090E0CF9108951092690893
:10E510001092680810926D0810926C0810926B08A7
:10E5200010926A0810926E088AE090E00E94261706
:10E5300090931204809311040895CF93DF938091F8
:10E540001104909112040E942F17882309F4AFC080
:10E5500080911104909112040A9690931204809372
:10E560001104E0E0F0E09F0190E05FEFAAECB6E07C
:10E570004BE0ED018B8187FF0BC09F5F8D81E80F22
:10E58000F11D8981280F311D8E81851708F4582FC0
:10E590004150189647FFEDCF50936E08232B41F55D
:10E5A00020911704309118044091190450911A04D5
:10E5B000BB27A52F942F832F9093160480931504C7
:10E5C000AA27BB27281B390B4A0B5B0BCF01AA27B5
:10E5D000BB27280F391F4A1F5B1F20931704309356
:10E5E00018044093190450931A04E5E0F0E013C0B6
:10E5F00020911504309116042E173F0718F4E21BE2
:10E60000F30B02C0E0E0F0E0892F9927880F991FF3
:10E61000E80FF91F3596F0936908E0936808EF3F1B
:10E62000F10578F480911D0190911E018E9F90015B
:10E630008F9F300D9E9F300D1124C90164E670E05C
:10E6400013C0CF01969587959695879520911D01CA
:10E6500030911E01289FA001299F500D389F500D19
:10E660001124CA0169E170E00E94707D70936B080B
:10E6700060936A0820911304309114042E0F3F1FF9
:10E6800030931404209313045EE02131350778F0B1
:10E6900080916C0890916D08019690936D0880931D
:10E6A0006C0820513E403093140420931304DF91F2
:10E6B000CF910895002422273327442751E0BB2718
:10E6C000EE27FF27A0E1660F771F881F991F001C08
:10E6D000221F331F441F660F771F881F991F001CBE
:10E6E000221F331F441F2AF4050E2B1F3E1F4F1FEE
:10E6F00004C0051A2B0B3E0B4F0B550FBB1FEE1F13
:10E70000587F556047FD5250AA95E9F6E695B795B2
:10E710005795E695B7955795852F9B2F08952227F6
:10E72000332741E0552768E0880F991F221F331FC8
:10E73000880F991F221F331F1AF4240F351F02C0A0
:10E74000241B350B440F551F487F456037FD425051
:10E750006A9551F75695479556954795842F089594
:10E76000AA2797FF04C0809590958A1F9A1F77FF6C
:10E7700004C0609570956A1F7A1F669F9001779F0D
:10E78000A001679F300D411D5A1F300D411D5A1FBA
:10E79000889FF001999F2E0F3F1F401D511D899F9B
:10E7A000300D411D5A1F300D411D5A1FCA01B901BC
:10E7B000112480CF4FB720E430E0F8948091C90055
:10E7C0008F778093C9008091C9008F7B8093C900A7
:10E7D0008091C9008F7D8093C9005A9A52985B9AA4
:10E7E000539A832F99278093CD002093CC0080915A
:10E7F000C80082608093C80088E18093C90080913E
:10E80000CA008F778093CA008091CA008F7B809363
:10E81000CA008091CA008F7D8093CA008091CA008F
:10E820008F7E8093CA008091CA00877F8093CA0040
:10E830008091C9008B7F8093C9008091CA00846059
:10E840008093CA008091CA0082608093CA00809140
:10E85000C80087FF03C08091CE00F9CF8091C90026
:10E8600080688093C9004FBF08950F931F93CF9383
:10E87000DF93482F4F5F893108F089C080912A07C4
:10E88000841710F440932A07CB0183539B4268E11D
:10E8900070E00E94847DA42FBB27FD01EA0FFB1FBF
:10E8A000E55DF84F808191819B01281B390BC901DF
:10E8B00037FF03C0909581959F4F069794F4809100
:10E8C0001B03883C30F480911B03865F80931B03FD
:10E8D00008C088EC80931B0380916F008F7D80932C
:10E8E0006F00FD01EA0FFB1FE55DF84F808191810C
:10E8F0009C01220F331F280F391F260F371F37FFA8
:10E9000002C02D5F3F4FE901D595C795D595C795B5
:10E91000CB0101968C179D0714F4219706C0615016
:10E920007040C617D7070CF4219680911B03843BD7
:10E93000D8F08D010A0F1B1FF801E55DF84F8081AB
:10E940009181FE01E81BF90BCF0163E070E00E94AA
:10E95000847DCB01880F991F860F971F015A184F8E
:10E96000F8019183808307C0AA0FBB1FA15AB84F3B
:10E9700011961C921E92E42FFF27EE0FFF1FE55DFC
:10E98000F84FD183C083443011F410929301DF918A
:10E99000CF911F910F910895CF93DF9320916F082E
:10E9A000822F9927807F9070409709F06CC02F319B
:10E9B00009F046C08091700880931F04209172086E
:10E9C000209321048091730880932004822F99273B
:10E9D00090932C0780932B07222309F054C0809139
:10E9E0000406282F3327220F331FF901E15AF84F6D
:10E9F0001182108280910506A82FBB27AA0FBB1F8A
:10EA0000FD01E15AF84F1182108280910706E82F2C
:10EA1000FF27EE0FFF1FCF01815A984FEC0119829B
:10EA20001882255D384FE90119821882A55DB84F1B
:10EA300011961C921E92E55DF84F1182108223C040
:10EA4000C22FCF70CA30F8F4809170088093990873
:10EA500080917108809398088091720880939B0838
:10EA60008091730880939A08609198087091990832
:10EA70008C2F0E94357460919A0870919B088C2F9E
:10EA80008F5F0E943574DF91CF910895CF93C82F87
:10EA90008F3F49F4809122048F3F29F4109224047F
:10EAA0001092230432C020912404222339F4CF3160
:10EAB00011F485E001C084E0809325048091250451
:10EAC000909123048217A0F4892F809580932304CA
:10EAD0008F3F19F48EEF8093230480912304C8178D
:10EAE00011F40E94CC7410922404109223040BC0E1
:10EAF000E22FFF27E159F74FC0832F5F20932404B3
:10EB00009C0F90932304C0932204CF910895909179
:10EB10001E04933240F4E92FFF27EB58F74F808310
:10EB20009F5F90931E040895833218F48D5F809345
:10EB30001E04089590E2E8E7F8E08FE19193815098
:10EB400087FFFCCF0895CF93CFB723E031E0F8944F
:10EB50008091C9008F778093C9008091C9008F7B15
:10EB60008093C9008091C9008F7D8093C9005A9A13
:10EB700052985B9A539A832F99278093CD002093C4
:10EB8000CC008091C80082608093C80088E18093A7
:10EB9000C9008091CA008F778093CA008091CA0013
:10EBA0008F7B8093CA008091CA0080628093CA00E4
:10EBB0008091CA0080618093CA008091CA008860F9
:10EBC0008093CA008091C90084608093C9008091BD
:10EBD000CA0084608093CA008091CA0082608093DA
:10EBE000CA008091C80087FF03C08091CE00F9CF92
:10EBF0008091C90080688093C9008091C9008064B9
:10EC00008093C9000E949A75CFBFCF910895282F95
:10EC100099278F709070892B31F4209580911D0475
:10EC2000822B80931D0408958091EF01882309F4BD
:10EC300041C08091E70285FF0AC082E98093750890
:10EC400083E28093760885E58093770802C010926E
:10EC500075088091F0018F3071F480911D040E943D
:10EC60003172882341F081E980937508809376089A
:10EC700081E3809377081092EF018091C80085FFAF
:10EC8000FCCF8091C9008F7E8093C9008091C9001C
:10EC90008E7F8093C90080917508882311F48EEFD0
:10ECA00001C08EE78093CE0080911D048093F00117
:10ECB00010921D0408951F920F920FB60F92112407
:10ECC0008F939F93EF93FF939091EF01992309F016
:10ECD00040C080912604882361F4809175088823C0
:10ECE00011F483E003C0813999F481E08093260414
:10ECF0000FC0833099F480917508882349F0909370
:10ED000075088091C9008E7F8093C9008EEF1EC068
:10ED10008091C90081608093C9000EC0833261F484
:10ED20008091C9008E7F8093C9008FEF8093CE00C1
:10ED300081E08093EF0114C080912604E82FFF2723
:10ED4000EB58F74F8F5F8093260480818093CE002D
:10ED500007C0109226048091C90080618093C90089
:10ED6000FF91EF919F918F910F900FBE0F901F9089
:10ED70001895EF92FF920F931F93CF93DF937C012F
:10ED80008B01EA01452B39F0F80181918F01F701E0
:10ED900009952197C9F7E6E0CDB7DEB70C94FC7D65
:10EDA000EF92FF920F931F93CF93DF937C018B0120
:10EDB000EA01452B41F0F8010F5F1F4F8491F701E5
:10EDC00009952197C1F7E6E0CDB7DEB70C94FC7D3D
:10EDD0000F931F93CF938C01C62F161634F480E245
:10EDE000F8010995C1501C16D4F3CF911F910F91D2
:10EDF00008950F931F93CF938C01C62F161634F4EA
:10EE000080E3F8010995C1501C16D4F3CF911F91EE
:10EE10000F910895A5E3B0E0E0E1F7E70C94D47D0D
:10EE20002E96EEADFFAD2E97882499245401809143
:10EE30001C04882321F42C961FAE1EAE2C975EE492
:10EE4000452E512C4C0E5D1E6F01B60105C01532CA
:10EE500039F00894C11CD11CF60114911123B9F7A3
:10EE6000A601461B570B31F02C968EAD9FAD2C970B
:10EE70000E94D076112309F46AC20894C11CD11CE7
:10EE8000FF24FDA6FCA64FEFE42EF9A6F601089498
:10EE9000C11CD11C1491153721F0812F8062883755
:10EEA000B1F4F0FE0AC0F20124E030E0420E531E3D
:10EEB00080809180A280B3800AC0F20142E050E0DD
:10EEC000440E551E808191814C01AA24BB2410322E
:10EED00021F489A58823D1F61DC0133219F458E016
:10EEE000F52AD4CF1A3211F01D3291F41A3259F4A6
:10EEF000F20182E090E0480E591EE081ECA7EE237B
:10EF00002CF6E195ECA790E1F92AAFEDFA22BECFFD
:10EF10001B3211F419A7BACF1E32C1F5F6010894BD
:10EF2000C11CD11C14911A3279F4F20122E030E0B4
:10EF3000420E531E408151813FEF4F3F530714F45F
:10EF40004FEF5FEFE42EA2CF40E050E0812F8053DF
:10EF50008A30A0F4CA0133E0880F991F3A95E1F78F
:10EF6000840F951F480F591F410F511D40535040AA
:10EF7000F6010894C11CD11C1491E8CF8FEF4F3FCC
:10EF8000580714F44FEF5FEFE42E85CF103329F4C8
:10EF9000F4FC7CCF90E2F92A79CF812F815389301C
:10EFA000D8F440E050E0CA0123E0880F991F2A9569
:10EFB000E1F7840F951F480F591F410F511D405312
:10EFC0005040F6010894C11CD11C1491812F80532C
:10EFD0008A3048F34CA75FCF183619F4A4E0FA2A18
:10EFE00055CF1C3619F4B1E0FB2A50CF133661F42B
:10EFF0003E010894611C711CF20122E030E0420ED7
:10F00000531E808189833CC1143421F0143611F0E1
:10F01000193651F5143411F431E0F32AF0FE0AC028
:10F02000F20144E050E0440E551E80809180A280A1
:10F03000B3800CC0F20182E090E0480E591E80813E
:10F0400091814C01AA2497FCA094BA2CB7FE0AC067
:10F05000B094A09490948094811C911CA11CB11C2C
:10F060008DE289A70AE06FC01F3411F01F3631F41A
:10F070001F3411F491E0F92A08E064C0103779F4E4
:10F08000F201A2E0B0E04A0E5B1E808191814C014A
:10F09000AA24BB2400E1B0E4FB2A18E753C01337CD
:10F0A000C1F5F20122E030E0420E531E6080718013
:10F0B0006114710489F43E010894611C711C88E29A
:10F0C00089838EE6F301818385E78B838CE68C83CD
:10F0D0008D8389E28E831F82E7FC13C08E2D9927D2
:10F0E00087FD9095AC0160E070E0C3010E94A17BB8
:10F0F000009729F0382E3618E3140CF0C3C03E2CCC
:10F10000C1C0F30101900020E9F731973E2E361877
:10F11000B9C0153511F0153731F4153511F4F1E09A
:10F12000FF2A0AE00FC0183519F0183709F0A0C0FF
:10F1300000E1F3FE07C081149104A104B10411F0B1
:10F1400020E4F22A19A6EDA6E7FC02C03FEDF32267
:10F1500089E2682E712C6C0E7D1E81149104A1042D
:10F16000B10421F44DA5442309F47BC0802F9927D5
:10F17000AA27BB278EA79FA7A8ABB9AB202E332405
:10F1800090E0891690E0990691E0A90690E0B90612
:10F1900048F0C501B4012EA53FA548A959A90E9470
:10F1A000977D17C0AFEF8A169104A104B10449F00E
:10F1B00040F0C401B1010E94707D9B014427552796
:10F1C00008C0882D602F0E94647D282F3327442794
:10F1D00055272AAB3BAB4CAB5DAB0A3059F48AA93F
:10F1E000880F880F880F9AA9990F890F382D381B1F
:10F1F000832F10C0003139F48AA98295807F482D71
:10F20000481B842F07C08AA9880F880F880F582DA4
:10F21000581B852F90E02EA53FA548A959A9821615
:10F220009306A406B50608F091E08AA89BA8ACA8AE
:10F23000BDA88A3010F4805D04C0895A183509F4DD
:10F240008F7DD3018E933D01992309F099CF08302A
:10F2500041F4F3FE06C0803321F080E3FD01829388
:10F260003F01CE010196382E3618F8E23F0E0BC052
:10F27000112309F46CC03E010894611C711C1983B0
:10F28000B1E03B2E19A6032D2DA4231827FC222420
:10F2900089A5882311F00F5F02C0F6FC0E5F020DF6
:10F2A000EF2CFF24C70180739070892B49F48CA543
:10F2B000801B682F2C968EAD9FAD2C970E94E87610
:10F2C00089A5882331F041E050E0BE01675D7F4FA2
:10F2D0000AC0E6FE0EC080E38AA71BA742E050E00A
:10F2E000BE01665D7F4F2C968EAD9FAD2C970E9420
:10F2F000B976C70180739070809749F48CA5801B04
:10F30000682F2C968EAD9FAD2C970E94F976622DBA
:10F310002C968EAD9FAD2C970E94F976832D992760
:10F3200087FD9095AC01B3012C968EAD9FAD2C97C7
:10F330000E94B976E4FE89CD2CA5201B2CA7622F54
:10F340002C968EAD9FAD2C970E94E8767ECDE2E1A3
:10F35000CB5C0C94F07D2FB740E0F894E0E0F0E057
:10F3600081E2809357009491E2E0F0E080935700AF
:10F370003491E4E0F0E08093570084912FBF9E31F8
:10F3800099F4363941F4893011F441E00DC08A30E6
:10F3900059F442E009C0373939F4863011F443E0BA
:10F3A00003C0853009F444E0842F992708959FB75E
:10F3B000F8948091C900877F8093C9008091C9002B
:10F3C0008F7E8093C9008091C9008F778093C90098
:10F3D0008091C9008F7B8093C9008091C9008F7D87
:10F3E0008093C90052985A9A53985B9A9FBF089588
:10F3F0001F93CF93DF93182F80911C04882309F467
:10F400008DC08091EE01181709F488C080911B040B
:10F41000882321F40E94AB7980931B048FE49EE043
:10F420009F938F93CFEFD2E1DF93CF93E0912704A7
:10F43000F091280409950F900F900F900F90812F55
:10F4400099278230910501F1833091052CF40097C2
:10F4500061F0019769F024C084309105D9F08430BF
:10F460009105ACF00597C9F01BC08FE39EE002C088
:10F470008DE29EE09F938F93DF93CF93E0912704DB
:10F48000F0912804099518C084E19EE0F3CF81EF44
:10F490009DE0F0CF83EE9DE0EDCF8BED9DE0EACFD8
:10F4A0008CE59EE09F938F93DF93CF93E0912704A9
:10F4B000F0912804099510E00F900F900F900F9095
:10F4C00080911B04843011F0823099F40E94D77926
:10F4D000812F8150833018F40E941D6A1DC01430A2
:10F4E00019F40E94A37518C01530B1F40E94DA73A4
:10F4F00013C0112389F082E79EE09F938F938FEFD3
:10F5000092E19F938F93E0912704F091280409954D
:10F510000F900F900F900F901093EE01DF91CF910D
:10F520001F9108950F931F9381E080931C044091D5
:10F53000ED01EBE8FDE020E030E05FE48491992705
:10F540002F5F3F4F829FB001839F700D929F700D80
:10F55000112446275150319657FFF0CF4093ED01CB
:10F56000E3E6FDE020E030E057E2849199272F5F49
:10F570003F4F829FB001839F700D929F700D1124A9
:10F5800046275150319657FFF0CF4093ED018091BF
:10F590001B04882321F40E94AB7980931B04809183
:10F5A000ED01833459F088E190E029E20FB6F89438
:10F5B000A895809360000FBE209360008AE097E7D3
:10F5C00090932804809327048DE89EE09F938F9367
:10F5D0000FEF12E11F930F93E0912704F09128049D
:10F5E00009950F900F900F900F9087E690E09F93F2
:10F5F0008F9380E590E09F938F931F921F9280914D
:10F6000002016AE00E94647D892F99279F938F935E
:10F61000809102010E94647D99279F938F9383EBD1
:10F620009EE09F938F931F930F93E0912704F09197
:10F63000280409958BE89DE09F938F931F930F9368
:10F64000E0912704F0912804099583E69DE09F93BB
:10F650008F931F930F93E0912704F091280409954D
:10F660008DB79EB746968DBF87EE9EE09F938F9392
:10F670001F930F93E0912704F0912804099583ECE0
:10F680008093810080916F00806280936F000F9063
:10F690000F900F900F901F910F91089580911C046F
:10F6A000882361F08091EE01843011F40E94147679
:10F6B0008091ED01833411F010921C0408951F9283
:10F6C0000F920FB60F9211242F933F934F935F9396
:10F6D0006F937F938F939F93AF93BF93EF93FF931A
:10F6E0002091CE009091EE01892F8150833020F43B
:10F6F000822F0E942A6B0BC0943021F4822F0E942B
:10F70000077605C0953019F4822F0E944675FF9147
:10F71000EF91BF91AF919F918F917F916F915F9189
:10F720004F913F912F910F900FBE0F901F90189502
:10F73000FB01DC0102C005900D9241505040D8F70A
:10F740000895FC014150504030F001900616D1F769
:10F750003197CF010895882799270895A0E0B0E058
:10F76000E4EBFBE70C94DC7D6C017B01EA015901C1
:10F7700021978FEFCF3FD80789F086010894C11CED
:10F78000D11CC7010894E11CF11CF5010995F80191
:10F7900080832197FFEFCF3FDF0779F7EAE0CDB70E
:10F7A000DEB70C94F87DCF92DF92EF92FF920F9329
:10F7B0001F937C016B01FB010995082FC70101967E
:10F7C000F6010995182FC8011F910F91FF90EF9036
:10F7D000DF90CF900895A0E0B0E0E1EFFBE70C945C
:10F7E000DE7D8C017B01EA01690121978FEFCF3F1C
:10F7F000D80771F0F70121917F01C8010F5F1F4FFA
:10F80000622FF60109952197FFEFCF3FDF0791F7B0
:10F81000E8E0CDB7DEB70C94FA7DCF92DF92EF929D
:10F82000FF920F931F936C018B017A01FA010995E6
:10F83000812F9927682FC6010196F70109951F911D
:10F840000F91FF90EF90DF90CF9008955058BB2715
:10F85000AA270ED0E0C0D1D030F0D6D020F031F4BD
:10F860009F3F11F41EF4C6C00EF4E095E7FBBCC048
:10F87000E92FE2D080F3BA17620773078407950770
:10F8800018F071F49EF5FAC00EF4E0950B2EBA2F25
:10F89000A02D0B01B90190010C01CA01A001112496
:10F8A000FF27591B99F0593F50F4503E68F11A1642
:10F8B000F040A22F232F342F4427585FF3CF4695D3
:10F8C00037952795A795F0405395C9F77EF41F16F5
:10F8D000BA0B620B730B840BBAF09150A1F0FF0FBF
:10F8E000BB1F661F771F881FC2F70EC0BA0F621FAB
:10F8F000731F841F48F4879577956795B795F7959B
:10F900009E3F08F0B3CF9395880F08F09927EE0F2C
:10F9100097958795089598D088F09F5790F0B92FC4
:10F920009927B751A0F0D1F0660F771F881F991F54
:10F930001AF0BA95C9F712C0B13081F09FD0B1E08A
:10F9400008959CC0672F782F8827B85F39F0B93F9A
:10F95000CCF3869577956795B395D9F73EF4909556
:10F960008095709561957F4F8F4F9F4F0895E894D4
:10F9700009C097FB3EF490958095709561957F4FF7
:10F980008F4F9F4F9923A9F0F92F96E9BB279395A5
:10F99000F695879577956795B795F111F8CFFAF4B5
:10F9A000BB0F11F460FF1BC06F5F7F4F8F4F9F4FE6
:10F9B00016C0882311F096E911C0772321F09EE844
:10F9C000872F762F05C0662371F096E8862F70E0AA
:10F9D00060E02AF09A95660F771F881FDAF7880F84
:10F9E0009695879597F9089597F99F6780E870E055
:10F9F00060E008959FEF80EC089500240A941616A5
:10FA0000170618060906089500240A94121613060C
:10FA1000140605060895092E0394000C11F488239A
:10FA200052F0BB0F40F4BF2B11F460FF04C06F5FB6
:10FA30007F4F8F4F9F4F089557FD9058440F551F8C
:10FA400059F05F3F71F04795880F97FB991F61F060
:10FA50009F3F79F087950895121613061406551FD7
:10FA6000F2CF4695F1DF08C0161617061806991F43
:10FA7000F1CF86957105610508940895E894BB2738
:10FA800066277727CB0197F90895629FD001739F6E
:10FA9000F001829FE00DF11D649FE00DF11D929F2A
:10FAA000F00D839FF00D749FF00D659FF00D992769
:10FAB000729FB00DE11DF91F639FB00DE11DF91F8D
:10FAC000BD01CF0111240895991B79E004C0991F4D
:10FAD000961708F0961B881F7A95C9F780950895A8
:10FAE000AA1BBB1B51E107C0AA1FBB1FA617B70764
:10FAF00010F0A61BB70B881F991F5A95A9F7809580
:10FB00009095BC01CD01089597FB092E07260AD0D8
:10FB100077FD04D0E5DF06D000201AF470956195DA
:10FB20007F4F0895F6F7909581959F4F0895A1E234
:10FB30001A2EAA1BBB1BFD010DC0AA1FBB1FEE1F67
:10FB4000FF1FA217B307E407F50720F0A21BB30BB2
:10FB5000E40BF50B661F771F881F991F1A9469F72E
:10FB600060957095809590959B01AC01BD01CF018A
:10FB7000089597FB092E05260ED057FD04D0D7DF38
:10FB80000AD0001C38F450954095309521953F4F90
:10FB90004F4F5F4F0895F6F790958095709561955A
:10FBA0007F4F8F4F9F4F08952F923F924F925F92BA
:10FBB0006F927F928F929F92AF92BF92CF92DF927D
:10FBC000EF92FF920F931F93CF93DF93CDB7DEB7E2
:10FBD000CA1BDB0B0FB6F894DEBF0FBECDBF099476
:10FBE0002A88398848885F846E847D848C849B84CD
:10FBF000AA84B984C884DF80EE80FD800C811B81DB
:10FC0000AA81B981CE0FD11D0FB6F894DEBF0FBE09
:10FC1000CDBFED010895EE0FFF1F0590F491E02D8B
:04FC20000994FFCF75
:10FC24005E010A010164FF01FFFF01FC01FC010107
:10FC3400737373FF03007D0000C409C409640011D9
:10FC440048656C6C6F20576F726C64000000000094
:10FC540000000000000000000000000000000000A0
:10FC64000000000000000000000000000000000090
:10FC74000000000000000000000000000000000080
:10FC84000000000000000000000000000000000070
:10FC940053706F727400004E6F726D616C0000429D
:10FCA4006567696E6E6572000051756164726F00FC
:10FCB40000640001200B050000ECFF6440415A463B
:10FCC40064640A02969696960840403A10FB3038CF
:10FCD4000190D0030090D00300F4017800FF036486
:10FCE40000020406070808080706040200FEFCFADE
:10FCF400F9F8F8F8F9FAFCFE000204060708080B04
:10FD04000A0D0B0C0E0B0F10FA2001010170FF01FC
:02FD14000F00DE
:00000001FF
